:020000040800F2
:1000000088AF00209D010008AD3D01082D280108A2
:10001000D13A010835380008C5D8010800000000B1
:10002000000000000000000000000000C16A01089C
:10003000B56F000800000000A1460108F174010836
:10004000B7010008B7010008B7010008B7010008B0
:10005000B7010008B7010008B96F0008B701000830
:10006000B7010008C56F0008D16F0008B70100088C
:10007000156A0008256A0008B7010008B7010008E2
:10008000B7010008B7010008B7010008B701000870
:100090003938000849380008B7010008DD6F00084A
:1000A000E5750108B7010008B7010008B7010008AD
:1000B000B7010008B7010008B7010008B701000840
:1000C000B7010008B7010008B7010008B701000830
:1000D000B7010008D9A60108B7010008B701000858
:1000E000B7010008B7010008B7010008B701000810
:1000F000B7010008B7010008B7010008356A000819
:10010000B7010008B7010008B7010008B7010008EF
:10011000B7010008B7010008B7010008F57501082C
:10012000B7010008456A0008556A0008656A0008BA
:10013000B7010008B7010008B7010008B7010008BF
:100140005938000869380008B70100081D3E010849
:10015000756A0008856A0008956A0008F5A6010816
:10016000B7010008B7010008B7010008B70100088F
:10017000B7010008B7010008B7010008000000003F
:10018000B7010008B7010008DFF80CD000F0FAFB57
:100190000048004755DC010888AF0020064880472A
:1001A00006480047FEE7FEE7FEE7FEE7FEE7FEE75C
:1001B000FEE7FEE7FEE7FEE7C575010889010008D6
:1001C0002DE9F05F0546002092469B46884606468C
:1001D000814640241BE0284641464746224600F01F
:1001E00063FA53465A46C01A914110D31146184635
:1001F000224600F04AFA2D1A67EB01084F462246C4
:100200000120002100F041FA17EB00094E41201EA9
:10021000A4F10104DFDC484631462A464346BDE8E6
:10022000F09F00000649074A0868504343F239022C
:10023000104408604008704701490860704700009A
:10024000000000206D4EC64140EA01039B0703D029
:1002500009E008C9121F08C0042AFAD203E011F805
:10026000013B00F8013B521EF9D27047D2B201E0C7
:1002700000F8012B491EFBD270470022F6E710B5AB
:1002800013460A4604461946FFF7F0FF204610BD04
:1002900010B5044604E00B7800F8013B03B1491C9B
:1002A000521EF8D2204610BD421C10F8011B002936
:1002B000FBD1801A704710B5002200E0521C835C0D
:1002C0008C5CA34201D1002BF8D1D8B2E1B2401A24
:1002D00010BD034611F8012B00F8012B002AF9D1BB
:1002E0001846704730B505460020034600E05B1C09
:1002F000934205D2EC5CC85C201A01D1002CF6D1E7
:1003000030BD2DE9FE4F804681EA0300C00F0C4648
:10031000009021F0004123F00045B8EB0200A94114
:1003200005D24046214690461C460B46024623F025
:100330000040104347D0270DC7F30A00C3F30A510A
:100340000290401A019040286BDAC3F3130040F486
:10035000801B0098924620B10023D2EB030A63EB86
:100360000B0B01985946C0F14002504600F08DF940
:1003700006460D4650465946019A00F0A5F910EB85
:1003800008006141002487EA115284EAE7731A43A6
:1003900040D0009A62B3019A012A4FEA075215DC55
:1003A000001B61EB02014FF0004202EA0752CDE967
:1003B0000042001C41F5801132462B4600F0DCF96A
:1003C00003B0BDE8F08F40462146F9E7001B61EB22
:1003D0000201001C41F5801300185B412018A2F5B2
:1003E000001747EB030140EAD570B6196D4111E0E3
:1003F0006D084FEA360645EAC0754FEA0752001B02
:1004000061EB0201001C41F5801149084FEA300000
:100410000019514132462B4603B0BDE8F04F00F0C1
:100420009CB90098012240000023D0EB020263EB4C
:10043000E073009821464FEAE074B8EB000061EBEE
:100440000401E9E783F000435BE781F0004158E7EE
:100450002DE9FE4F81EA030404F0004421F000413D
:1004600000944FF0000B23F0004350EA01045ED0EB
:1004700052EA03045BD0C3F30A54C1F30A552C4477
:10048000A4F2F3340194A0FB0254C1F3130141F42C
:100490008011C3F3130343F4801301FB024400FBF8
:1004A000034E840A970A44EA815447EA8357A4FB1F
:1004B000076802958D0A05FB07854FEA932C04FB1C
:1004C0000C542705029D4FEA065847EA1637B5EB4C
:1004D00008056EEB070C870E920E47EA811742EA79
:1004E0008312A7FB0201B6EB0B0164EB00042B0D9A
:1004F00043EA0C335E1844EB1C50DA465146E7FBE6
:100500000201C5F313044FEA0B3343EA14534FEAD5
:100510000432019C43EA0603A4F10C040294009CFB
:10052000CDE900B400F028F903B0BDE8F08F002059
:100530000146F9E730B5041E71F1000404DB4FF009
:100540000044404264EB0101141E73F1000405DB1A
:100550001C464FF00043524263EB0403801A99415A
:1005600001D3012030BD002030BD30B5041E71F133
:10057000000404DB4FF00044404264EB0101141E10
:1005800073F1000405DB1C464FF00043524263EB5D
:100590000403101A8B4101D3012030BD002030BD6F
:1005A0000EB5C10F80EAE0700844CA07002140F28E
:1005B00033438DE80E000A460B4600F0DDF803B029
:1005C00000BD70B5C1F30A5201F000450024C1F32B
:1005D000130140F2FF3341F480119A4201DA002006
:1005E00070BD40F233439A42A2F2334203DC5242DE
:1005F00000F05AF800E090402C43F1D0404270BD2A
:1006000000F0004230F000400AD0C10D01F56071E9
:10061000C0F3160042EA0151C20840071143704777
:1006200000200146704701F0004330B421F0004142
:1006300050EA010206D00A0DA2F56072C1F313015F
:10064000002A02DC30BC00207047440F44EAC10499
:10065000C100E01830BC00EBC25000F047B830B524
:100660000B46014600202022012409E021FA02F570
:100670009D4205D303FA02F5491B04FA02F528440A
:10068000151EA2F10102F1DC30BD202A04DB203A64
:1006900000FA02F1002070479140C2F1200320FAD5
:1006A00003F3194390407047202A04DB203A21FAD3
:1006B00002F00021704721FA02F3D040C2F120027B
:1006C0009140084319467047202A06DBCB17203A91
:1006D00041FA02F043EAE07306E041FA02F3D04047
:1006E000C2F1200291400843194670470029A8BF73
:1006F0007047401C490008BF20F00100704710B44B
:10070000B0FA80FC00FA0CF050EA010404BF10BCFF
:10071000704749B1CCF1200421FA04F411FA0CF12C
:1007200018BF012121430843A3EB0C01CB1D4FEA65
:1007300000614FEA102042BF002010BC704700EB60
:10074000C35010440029A4BF10BC7047401C49008E
:1007500008BF20F0010010BC704710B5141E73F1E3
:10076000000408DA401C41F1000192185B411A4371
:1007700001D120F0010010BD2DE9F04D92469B46BD
:1007800011B1B1FA81F202E0B0FA80F22032904663
:10079000FFF77BFF04460F4640EA0A0041EA0B01DF
:1007A00053465A46084313D0114653EA010019D064
:1007B000C8F140025046FFF777FF05460E46504607
:1007C00059464246FFF761FF084305D0012004E087
:1007D00020463946BDE8F08D0020054346EAE07624
:1007E0002C4337430A986305E40AA0EB0800002273
:1007F000FD0A44EA47540A3002D500200146E9E7E1
:10080000010510196941DDE9084500196941BDE894
:10081000F04DA2E72DE9F04D81EA030404F0004B0E
:1008200021F0004514464FF0000A23F0004150EA41
:10083000050220D054EA01021DD0C5F30A57024632
:10084000C5F31303C1F31300C1F30A5640F4801536
:1008500043F48013A7EB0608101BD64608F2FD38B8
:1008600073EB050002D308F1010801E092185B4127
:10087000B8F1000F03DA00200146BDE8F08D00203A
:100880004FF48011064684460EE0171B73EB0507F4
:1008900005D3121B63EB050306434CEA010C490820
:1008A0004FEA300092185B4150EA0107EDD152EA5D
:1008B000030012D082EA040083EA0501084305D050
:1008C000101BAB4106D20122002306E000224FF0AC
:1008D000004302E06FF0010253101AEB06004CEBEC
:1008E000085110EB0A0041EB0B01BDE8F04DFFF79A
:1008F00034BFC1F30A52C1F3130140F2FF3341F494
:1009000080119A4202DA00200146704740F23343D8
:100910009A42A2F2334202DC5242FFF7C5BEFFF711
:10092000B4BE000030B5041E71F1000404DB4FF0CA
:100930000044404264EB0101141E73F1000405DB26
:100940001C464FF00043524263EB04038B4208BF46
:10095000824230BD30B5041E71F1000404DB4FF05B
:100960000044404264EB0101141E73F1000405DBF6
:100970001C464FF00043524263EB0403994208BF08
:10098000904230BD064C074D06E0E06840F00103A0
:1009900094E8070098471034AC42F6D3FFF7F8FB11
:1009A00010630208306302080EB540F23341029131
:1009B0000021CDE900110A460B46FFF7DDFE03B02A
:1009C00000BD70B58D1810F8014B14F0030201D171
:1009D00010F8012B231106D110F8013B03E010F8A9
:1009E000016B01F8016B521EF9D1ABB110F8012B6C
:1009F00004F00C048A1A0C2C03D0A2EB84129B1C6A
:100A000008E010F8014BA2EB0422F8E712F8014BC2
:100A100001F8014B5B1EF9D5A942D4D3002070BD6B
:100A200080B582B0019042F20030C4F20100009023
:100A30000099486820F44030486001984268009965
:100A400048681043486001980168486820F4807045
:100A50004860019801680269486840EA02204860DD
:100A600001980168486820F040704860019801686A
:100A7000826848681043486001980168886820F4DB
:100A80000060886001980168C268886810438860C7
:100A90000198806A0121C0F60071884219D0FFE7F1
:100AA00001980168886820F070608860019801688A
:100AB000826A88681043886001980168886820F01D
:100AC0004050886001980168C26A88681043886055
:100AD0000CE001980168886820F0706088600198D7
:100AE0000168886820F040508860FFE7019801683D
:100AF000886820F0020088600198027E016888689A
:100B000040EA42008860019890F8200060B3FFE757
:100B10000198406A30B1FFE70198406A082801D87F
:100B2000FFE708E045F21650C0F6020040F2A67159
:100B30001CF0CEFFFFE701980168486840F40060B0
:100B4000486001980168486820F460404860019856
:100B50000168426A4EF20000CFF6FF7000EB4232AD
:100B600048681043486006E001980168486820F42E
:100B700000604860FFE701980168C86A20F47000CF
:100B8000C86201980168C2690020CFF6F07000EBDE
:100B90000252C86A1043C86201980168886820F44C
:100BA00000708860019890F830200168886840EAF9
:100BB0004220886001980168886820F4806088601D
:100BC000019801684269886840EA8220886002B022
:100BD00080BD000080B58AB008900791089820B9C0
:100BE000FFE7FF208DF827009BE0079820B9FFE77B
:100BF000FF208DF8270094E0079890ED000A90ED13
:100C0000013A90ED021A90ED032A20EE030A21EE3C
:100C1000021A30EE010A30EE000A8DED060A07983E
:100C200090ED010A90ED021A20EE000A21EE011A61
:100C300030EE010A30EE001AB7EE000A8DED010A1F
:100C400030EE410A8DED050A9DED060ADDED050A3F
:100C500022F092F89DED011A089880ED010A07989C
:100C600090ED000A90ED013A90ED024A90ED032AD2
:100C700020EE040A22EE032A30EE420A30EE000A89
:100C80008DED040A9DED040AB0EEC00AB4EE410AEF
:100C9000F1EE10FA0ADBFFE7DDED040A9FED230A0F
:100CA0001CF02AFF089880ED020A07E09DED040A77
:100CB00021F060FD089880ED020AFFE7079890EDAB
:100CC000000A90ED011A90ED022A90ED033A20EE11
:100CD000030A21EE021A30EE010A30EE000A8DED11
:100CE000030A079890ED020A90ED031A20EE000A1D
:100CF00021EE011A30EE010A30EE001AB7EE000ABA
:100D000030EE410A8DED020A9DED030ADDED020A87
:100D100022F032F8089880ED000A00208DF82700B4
:100D2000FFE79DF927000AB080BD00BFDB0FC93F78
:100D300080B58CB00A9009918DED080A0A9820B907
:100D4000FFE7FF208DF82F0029E19DED081AB7EE8F
:100D5000000A80EE010A0A9880ED040A0A994FF011
:100D60007E5008600A99002048600A9988600A99B4
:100D7000C8600998002800F00E81FFE70998016813
:100D800000914068FFF73CFC0246009801920A4639
:100D9000019942EC101B8DED020BFFF731FC9DED2C
:100DA000020B41EC110B21F0E7FE8DED040B9DF8D9
:100DB000170080F080008DF8170004980599FFF760
:100DC00032FC0790099890ED000AB5EE400AF1EE6A
:100DD00010FA2BD1FFE7099890ED010AB5EE400A11
:100DE000F1EE10FA22D1FFE7099890ED020AB5EE74
:100DF000400AF1EE10FA19D1FFE70A9940F2C560F6
:100E0000C3F64D7008600A9944F62D20C3F60D40D4
:100E100048600A994AF25640CBF6393088600A9900
:100E200044F2AD70C3F61970C860B3E09DED070AD7
:100E30009FED5D1AB4EE410AF1EE10FA08DBFFE710
:100E40009DED070AB5EE400AF1EE10FA19DDFFE755
:100E50000A9945F66E10C3F67F7008600A9945F24C
:100E60000C30C3F6B01048600A9948F6AB00CBF6D8
:100E7000BB3088600A9949F28550C3F69750C86024
:100E800087E09DED070A9FED491AB4EE410AF1EEA5
:100E900010FA0ADBFFE79DED070A9FED431AB4EE57
:100EA000410AF1EE10FA19DDFFE70A9940F2C56038
:100EB000C3F64D7008600A9944F62D20C3F60D4024
:100EC00048600A994AF25640CBF6393088600A9950
:100ED00044F2AD70C3F61970C86059E09DED070A81
:100EE0009FED331AB4EE410AF1EE10FA0ADBFFE788
:100EF0009DED070A9FED2D1AB4EE410AF1EE10FAAE
:100F000019DDFFE70A9940F2C560C3F64D7008602D
:100F10000A9944F62D20C3F60D4048600A994AF21A
:100F20005640CBF6393088600A9944F2AD70C3F66A
:100F30001970C8602BE09DED070A9FED1D1AB4EEF5
:100F4000410AF1EE10FA08DBFFE79DED070AB5EE66
:100F5000400AF1EE10FA19DDFFE70A9940F2C56088
:100F6000C3F64D7008600A9944F62D20C3F60D4073
:100F700048600A994AF25640CBF6393088600A999F
:100F800044F2AD70C3F61970C860FFE7FFE7FFE7F2
:100F9000FFE7FFE7FFE700208DF82F00FFE79DF94F
:100FA0002F000CB080BD00BFDB0FC93FDB0F4940F5
:100FB0000000B44281B00090009900208860486031
:100FC000086001B07047000080B52DED048BB2B011
:100FD00030902F912E922D93309828B9FFE7FF2063
:100FE0008DF8C70000F0F7BD2F9828B9FFE7FF2064
:100FF0008DF8C70000F0EFBD2E9828B9FFE7FF205D
:101000008DF8C70000F0E7BD40F28411C2F2000184
:101010004EF69E70C3F6275008602D9848B9FFE73A
:1010200030982F992E9A00F0DDFD8DF8C70000F062
:10103000D2BD2D98006809902D98406808902D9891
:10104000806807909DED090AB5EE400AF1EE10FAAE
:1010500019D1FFE79DED080AB5EE400AF1EE10FA4E
:1010600011D1FFE79DED070AB5EE400AF1EE10FA47
:1010700009D1FFE730982F992E9A00F0B3FD8DF833
:10108000C70000F0A8BD2F98006806902F98406810
:1010900005902F98806804902E98006803902E98F1
:1010A000406802902E988068019030989DED033A38
:1010B00090ED010A90ED022A90ED031A20EE430A0A
:1010C0009DED023A22EE032A30EE420A9DED012AFE
:1010D00021EE021A30EE410AB6EE001A20EE010AA5
:1010E0008DED270A30989DED034A90ED000A90EDB2
:1010F000023A90ED032A20EE040A9DED014A23EE08
:10110000043A30EE030A9DED023A22EE032A30EE55
:10111000420A20EE010A8DED260A30989DED024A22
:1011200090ED000A90ED013A90ED032A20EE040ABA
:101130009DED014A23EE043A30EE430A9DED033A59
:1011400022EE032A30EE020A20EE010A8DED250A76
:1011500030989DED014A90ED000A90ED013A90ED36
:10116000022A20EE040A9DED024A23EE043A30EEF4
:10117000030A9DED033A22EE032A30EE420A20EEE6
:10118000010A8DED240A9DED060AB5EE400AF1EE46
:1011900010FA11D1FFE79DED050AB5EE400AF1EE18
:1011A00010FA09D1FFE79DED040AB5EE400AF1EE11
:1011B00010FA00F09984FFE79DED060A20EE000A80
:1011C0009DED051A21EE011A30EE010A9DED041A7B
:1011D00021EE011A30EE010A11F0AEFB8DED2C0A62
:1011E0009DED2C1A9DED060A20EE010A8DED060AF2
:1011F0009DED2C1A9DED050A20EE010A8DED050AE4
:101200009DED2C1A9DED040A20EE010A8DED040AD5
:101210009DED090A20EE000A9DED081A21EE011A43
:1012200030EE010A9DED071A21EE011A30EE010A97
:1012300011F082FB8DED2C0A9DED2C1A9DED090A13
:1012400020EE010A8DED090A9DED2C1A9DED080A8C
:1012500020EE010A8DED080A9DED2C1A9DED070A7E
:1012600020EE010A8DED070A309890ED000A30EE6D
:10127000000A9DED091A20EE010A8DED210A309831
:1012800090ED000A30EE000A9DED081A20EE010AEA
:101290008DED200A309890ED000A30EE000A9DEDA9
:1012A000071A20EE010A8DED1F0A309890ED010A11
:1012B00030EE000A9DED091A20EE010A8DED1E0A9E
:1012C000309890ED000A30EE000A8DED190A309842
:1012D00090ED010A30EE000A8DED180A309890ED7D
:1012E000020A30EE000A8DED170A309890ED030ADD
:1012F00030EE000A8DED160A309890ED000A90ED60
:10130000021A30EE000A20EE010A8DED150A30981F
:1013100090ED020A90ED031A30EE000A20EE010A69
:101320008DED140A309890ED000A20EE000A8DED44
:10133000130A309890ED000A90ED011A20EE010A90
:101340008DED120A309890ED000A90ED021A20EE11
:10135000010A8DED110A309890ED000A90ED031A04
:1013600020EE010A8DED100A309890ED010A20EE72
:10137000000A8DED0F0A309890ED010A90ED021AE7
:1013800020EE010A8DED0E0A309890ED010A90EDE5
:10139000031A20EE010A8DED0D0A309890ED020A35
:1013A00020EE000A8DED0C0A309890ED020A90EDC7
:1013B000031A20EE010A8DED0B0A309890ED030A16
:1013C00020EE000A8DED0A0A9DED091A9DED130A23
:1013D00021EE000A9DED202A309890ED025A90ED02
:1013E000033A22EE032A30EE420A9DED1F2A22EE36
:1013F000052A30EE020A9DED0F2A21EE022A30EE78
:10140000020A9DED182A9DED084A22EE044A24EEB8
:10141000054A30EE040A9DED074A22EE042A22EE28
:10142000032A30EE020A9DED0C2A21EE022A30EE4C
:10143000420A9DED0A2A21EE021A30EE410A8DED94
:10144000230A9DED210A309890ED015A90ED024A51
:1014500090ED033A20EE030A9DED081A9DED132A44
:1014600021EE022A30EE020A9DED1F2A22EE052A05
:1014700030EE420A9DED1E2A22EE042A30EE020AC8
:101480009DED0F2A21EE022A30EE420A9DED0C2A34
:1014900021EE022A30EE020A9DED172A9DED074A41
:1014A00022EE042A22EE032A30EE020A9DED0A2AD9
:1014B00021EE021A30EE410A8DED220A9DED230A3B
:1014C00020EE000A9DED221A21EE011A30EE010AEB
:1014D00011F032FAB7EE006A86EE000A8DED1D0AB1
:1014E0009DED210A309890ED012A90ED021A90EDC1
:1014F000033A20EE011A9DED200A20EE020A30EE9A
:10150000412A9DED071A9DED130A21EE000A30EEE7
:10151000022A9DED1E0A20EE030A30EE020A9DED1E
:101520000F2A21EE022A30EE420A9DED172A9DED88
:10153000084A22EE042A22EE032A30EE020A9DED2A
:101540000C2A21EE022A30EE420A9DED0A2A21EEF3
:10155000021A30EE010A8DED1C0A9DED1D0A30EED7
:10156000000A8DED1B0A9DED1C0A30EE000A8DED80
:101570001A0A9DED170ADDED0D0A30EEA02A9DED49
:10158000151A31EE422A9DED061A31EE021A20EEAE
:10159000010A9DED181ADDED123A33EEA32A9DEDF6
:1015A000143A32EE032A9DED053A32EE432A21EE3B
:1015B000021A70EE014A9DED1C3A309890ED011A26
:1015C00090ED020AD0ED032A63EE001A9DED1D2A6C
:1015D0009DED0C7AB6EE004A8DED004A77EE445A46
:1015E0009DED0A5A35EE255A62EE055A9DED115AC7
:1015F00075EE606A63EE266A75EEA66ADDED095A3D
:1016000075EEA65A61EEA51A71EEA41A62EE222AB0
:1016100023EE011A31EE621ADDED0E2ADDED104ADD
:1016200072EEE42A62EE222ADDED0B4A73EEA43A52
:1016300063EE233A72EEA32ADDED083A72EEE32A56
:1016400021EE221A31EE211A22EE000A35EE205A3E
:1016500022EE052A9DED0F5A34EE455A35EE475AD3
:1016600023EE053A32EE032A9DED073A32EE432A85
:1016700020EE020A30EE010A8DED2B0A9DED160ACE
:10168000DDED0D2A32EEA21A9DED152A31EE421A39
:101690009DED062A31EE421A20EE010A9DED191A3F
:1016A000DDED126A36EEA62A9DED143A32EE032ADB
:1016B0009DED053A32EE432A21EE021A30EE011A70
:1016C0003098D0ED005AD0ED014AD0ED023A90EDBD
:1016D000032AB1EE000A24EE803A9DED0F7A37EE30
:1016E000075A75EE461ADDED0C0A30EEA05A75EE7B
:1016F000211A9DED045A35EE215A23EE053A31EEBA
:10170000031A9DED1C5A65EE027A9DED1D3A74EEAA
:10171000601A9DED0A8A71EEC81A23EE218ADDED6A
:10172000111A32EEE19A25EE099A38EE098A9DEDFA
:10173000099A38EE498A67EE887A31EE271A63EE05
:10174000233A65EE255A73EEA53ADDED0E5ADDED2E
:10175000107A75EEE75A63EE255ADDED0B7A76EED8
:10176000A76A65EE266A75EEA65ADDED086A75EE83
:10177000E65A63EEA53A31EE231A23EE022ADDED96
:101780001A3A63EEA43A32EE632A71EEA21A23EEFD
:10179000213A34EE477A37EE607A25EE075A33EE77
:1017A000053A9DED075A33EE453A22EE032A31EE13
:1017B000021A8DED2A1A9DED191ADDED0D0A30EE93
:1017C000A03A9DED152A32EE433A9DED062A32EEFF
:1017D000032A21EE021A9DED162ADDED124A34EE9F
:1017E000A43A9DED145A33EE053A9DED055A33EEB9
:1017F000453A22EE032A31EE022A309890ED001A83
:10180000D0ED011AD0ED022AD0ED033A22EE800A83
:101810009DED0F5A35EE053A33EE467A9DED0C6A92
:1018200036EE063A33EE077A9DED043A33EE073A88
:1018300020EE030A70EE025A9DED1B0A20EE620AAA
:101840009DED1C3A23EE012A30EE420A9DED1D2A41
:1018500034EE467ADDED0A6A37EE667A62EE076AA2
:101860009DED117A70EEC77A63EE277A76EEA76A5D
:10187000DDED097A76EEE76A20EE260A30EE250ADB
:1018800062EE211A63EE233A71EEA31ADDED0E3AF1
:10189000DDED105A73EEE53A62EE233ADDED0B5AB8
:1018A00074EEA54A63EE244A73EEA43ADDED084ACD
:1018B00073EEE43A61EEA31A30EE210A22EE011A29
:1018C000DDED1A1A61EEA21A31EE611A37EE207AB6
:1018D00022EE072A34EE455A35EE465A23EE053AF3
:1018E00032EE032A9DED073A32EE432A21EE021A28
:1018F00030EE010A8DED290A9DED180A9DED0D7A55
:1019000037EE071A9DED152A31EE421A9DED062A93
:1019100031EE421A20EE010A9DED171ADDED122A72
:1019200032EEA22A9DED143A32EE032A9DED053ADD
:1019300032EE432A21EE021A70EE013A9DED1B1A97
:101940003098D0ED001A90ED010AD0ED020A90ED2A
:10195000032A21EE022A9DED1C3A23EE001A31EEF5
:10196000421A9DED1D2A9DED0C5A34EE456ADDEDBF
:101970000A4A36EE646A62EE064A9DED116A77EE17
:10198000465A63EE255A74EEA54ADDED095A74EE07
:10199000E54A21EE241A31EE231A62EE211A63EE93
:1019A000200A70EEE10ADDED0E1ADDED103A71EE5F
:1019B000E31A62EE211ADDED0B3A72EEA32A63EE12
:1019C000222A71EEA21ADDED082A71EEE21A60EE0B
:1019D000A10A31EE201A22EE000A36EE076A22EE44
:1019E000062A9DED0F6A34EE464A34EE454A23EE50
:1019F000043A32EE032A9DED073A32EE432A20EEF6
:101A0000020A30EE010A8DED280A9DED2B0A20EE28
:101A1000000A9DED2A1A21EE011A30EE010A9DED11
:101A2000291A21EE011A30EE010A9DED281A21EE45
:101A3000011A30EE010A10F07FFF8DED2C0A9DEDAA
:101A40002C1A9DED2B0A20EE010A8DED2B0A9DED3F
:101A50002C1A9DED2A0A20EE010A8DED2A0A9DED31
:101A60002C1A9DED290A20EE010A8DED290A9DED23
:101A70002C1A9DED280A20EE010A8DED280A40F26D
:101A80008410C2F2000090ED000A9DED2B1A20EEAA
:101A9000011A9DED270A30EE410A8DED270A90EDDF
:101AA000000A9DED2A1A20EE011A9DED260A30EE5D
:101AB000410A8DED260A90ED000A9DED291A20EECF
:101AC000011A9DED250A30EE410A8DED250A90EDB3
:101AD000000A9DED281A20EE011A9DED240A30EE31
:101AE000410A8DED240AFFE79DED271A309890ED0D
:101AF000000A90ED042A21EE021A30EE010A80ED70
:101B0000000A9DED261A309890ED010A90ED042A06
:101B100021EE021A30EE010A80ED010A9DED251A30
:101B2000309890ED020A90ED042A21EE021A30EE70
:101B3000010A80ED020A9DED241A309890ED030A07
:101B400090ED042A21EE021A30EE010A80ED030A1C
:101B5000309890ED000A90ED013A90ED022A90ED58
:101B6000031A20EE000A23EE033A30EE030A22EEB7
:101B7000022A30EE020A21EE011A30EE010A10F0BC
:101B8000DBFE8DED2C0A9DED2C1A309890ED000AAD
:101B900020EE010A80ED000A9DED2C1A309890EDA0
:101BA000010A20EE010A80ED010A9DED2C1A309801
:101BB00090ED020A20EE010A80ED020A9DED2C1A3A
:101BC000309890ED030A20EE010A80ED030A002010
:101BD0008DF8C700FFE79DF9C70032B0BDEC048B5C
:101BE00080BD000080B5A0B01E901D911C921E9873
:101BF00020B9FFE7FF208DF87F00D3E21D9820B9C0
:101C0000FFE7FF208DF87F00CCE21C9820B9FFE7AA
:101C1000FF208DF87F00C5E240F28411C2F200017E
:101C200042F60230C3F6075008601D9800681B900A
:101C30001D9840681A901D98806819901C9800683B
:101C400018901C98406817901C98806816901E98F1
:101C50009DED183A90ED010A90ED022A90ED031ADD
:101C600020EE430A9DED173A22EE032A30EE420A97
:101C70009DED162A21EE021A30EE410AB6EE001A48
:101C800020EE010A8DED100A1E989DED184A90ED88
:101C9000000A90ED023A90ED032A20EE040A9DED31
:101CA000164A23EE043A30EE030A9DED173A22EE6F
:101CB000032A30EE420A20EE010A8DED0F0A1E982B
:101CC0009DED174A90ED000A90ED013A90ED032A40
:101CD00020EE040A9DED164A23EE043A30EE430A44
:101CE0009DED183A22EE032A30EE020A20EE010A98
:101CF0008DED0E0A1E989DED164A90ED000A90EDAE
:101D0000013A90ED022A20EE040A9DED174A23EED7
:101D1000043A30EE030A9DED183A22EE032A30EE23
:101D2000420A20EE010A8DED0D0A9DED1B0AB5EE6B
:101D3000400AF1EE10FA11D1FFE79DED1A0AB5EE57
:101D4000400AF1EE10FA09D1FFE79DED190AB5EE50
:101D5000400AF1EE10FA00F0AE81FFE79DED1B0A9C
:101D600020EE000A9DED1A1A21EE011A30EE010A4A
:101D70009DED191A21EE011A30EE010A10F0DCFD7A
:101D80008DED150A9DED151A9DED1B0A20EE010A39
:101D90008DED1B0A9DED151A9DED1A0A20EE010A24
:101DA0008DED1A0A9DED151A9DED190A20EE010A16
:101DB0008DED190A1E9890ED000A30EE000A8DEDA7
:101DC0000C0A1E9890ED010A30EE000A8DED0B0A08
:101DD0001E9890ED020A30EE000A8DED0A0A1E9858
:101DE00090ED030A30EE000A8DED090A1E9890ED81
:101DF000000AB1EE003A20EE030A8DED080A1E98A3
:101E000090ED010A20EE030A8DED070A1E9890ED71
:101E1000020A20EE030A8DED060A1E9890ED010AD3
:101E2000B2EE001A20EE010A8DED050A1E9890ED23
:101E3000020A20EE010A8DED040A1E9890ED000AB8
:101E400020EE000A8DED030A1E9890ED010A20EEA7
:101E5000000A8DED020A1E9890ED020A20EE000A9B
:101E60008DED010A1E9890ED030A20EE000A8DED1B
:101E7000000A9DED081A9DED010A21EE000A9DED74
:101E80000A2A9DED1B4A22EE042A30EE020A9DED3D
:101E9000022A21EE021A30EE010A9DED0B1A9DED89
:101EA0001A2A21EE021A30EE410A8DED140A9DED38
:101EB000071A9DED000A21EE000A9DED092A9DED0D
:101EC0001B4A22EE042A30EE420A9DED032A22EE3E
:101ED000032A1E9890ED014A22EE042A30EE020AEF
:101EE0009DED0C2A9DED1A4A22EE042A30EE420A9C
:101EF00030EE410A9DED052A9DED024A22EE044A8C
:101F000030EE040A9DED014A22EE042A30EE020A68
:101F10009DED192A21EE021A30EE010A8DED130A09
:101F20009DED030A20EE030A1E9890ED021A20EEA2
:101F3000010A9DED0C1A9DED1B2A21EE021A30EECE
:101F4000010A9DED061A9DED002A21EE022A30EECF
:101F5000020A9DED092A9DED1A4A22EE042A30EE6E
:101F6000420A30EE410A9DED042A9DED024A22EE1E
:101F7000044A30EE040A9DED014A22EE042A30EEB6
:101F8000020A9DED192A21EE021A30EE010A8DEDAA
:101F9000120A9DED020A20EE030A1E9890ED032A14
:101FA00020EE020A9DED0B1A9DED1B4A21EE041A4C
:101FB00030EE410A9DED011A21EE031A21EE021ABC
:101FC00030EE010A9DED0A1A9DED1A2A21EE021A41
:101FD00030EE410A8DED110A9DED140A20EE000A43
:101FE0009DED131A21EE011A30EE010A9DED121A31
:101FF00021EE011A30EE010A9DED111A21EE011AAF
:1020000030EE010A10F098FC8DED150A9DED151AC1
:102010009DED140A20EE010A8DED140A9DED151AAE
:102020009DED130A20EE010A8DED130A9DED151AA0
:102030009DED120A20EE010A8DED120A9DED151A92
:102040009DED110A20EE010A8DED110A40F2841077
:10205000C2F2000090ED000A9DED141A20EE011A64
:102060009DED100A30EE410A8DED100A90ED000A48
:102070009DED131A20EE011A9DED0F0A30EE410A74
:102080008DED0F0A90ED000A9DED121A20EE011A57
:102090009DED0E0A30EE410A8DED0E0A90ED000A1C
:1020A0009DED111A20EE011A9DED0D0A30EE410A48
:1020B0008DED0D0AFFE79DED101A1E9890ED000AB8
:1020C00090ED042A21EE021A30EE010A80ED000A9A
:1020D0009DED0F1A1E9890ED010A90ED042A21EE55
:1020E000021A30EE010A80ED010A9DED0E1A1E98CB
:1020F00090ED020A90ED042A21EE021A30EE010A58
:1021000080ED020A9DED0D1A1E9890ED030A90EDE8
:10211000042A21EE021A30EE010A80ED030A1E980D
:1021200090ED000A90ED013A90ED022A90ED031A2D
:1021300020EE000A23EE033A30EE030A22EE022AD2
:1021400030EE020A21EE011A30EE010A10F0F4FB23
:102150008DED150A9DED151A1E9890ED000A20EEE2
:10216000010A80ED000A9DED151A1E9890ED010AF6
:1021700020EE010A80ED010A9DED151A1E9890EDE2
:10218000020A20EE010A80ED020A9DED151A1E9842
:1021900090ED030A20EE010A80ED030A00208DF87D
:1021A0007F00FFE79DF97F0020B080BD84B00290E2
:1021B0000191029820B9FFE7FE208DF80F001FE083
:1021C000019820B9FFE7FE208DF80F0018E0029972
:1021D0000020009081F84F000299C1F81B0088612F
:1021E00048610861C86088604860019988614861F9
:1021F0000861C8608860486008608DF80F00FFE7DC
:102200009DF90F0004B0704780B584B00290FFE7DD
:10221000029840B9FFE745F6B500C0F602002D214F
:102220001BF052FBFFE7FFE742F21050C2F2000042
:102230000078C00720B1FFE7FD208DF80F003BE0DC
:10224000FFE71CF021F943F24011C2F200010860DF
:1022500040B9FFE745F6B500C0F602002F211BF09C
:1022600033FBFFE7FFE742F22572C0F600020220CF
:102270000190032101F042FA019842F20D72C0F67A
:102280000002082101F03AFA02994DF20A70C3F6F1
:102290002330C1F81F00029941F26F20C3F60330CA
:1022A000C1F8230042F21051C2F20001012008706F
:1022B00000208DF80F00FFE79DF90F0004B080BDEE
:1022C00082B00190009101984068009908600198DF
:1022D0008068009948600198007FC0F3C0000099B1
:1022E0000876019800690099C860019840690099D2
:1022F0000861019880690099486102B07047000048
:1023000080B584B00390029101920399C42081F8B2
:102310002E000399DDF808C0DCF80000DCF804208A
:10232000DCF80830DCF80CC0C1F83BC0C1F837302D
:10233000C1F83320C1F82F000399019B18685A682F
:102340009B68C1F84730C1F84320C1F83F000399AA
:10235000002081F84B00039890F84E00012808D126
:10236000FFE7039991F84B0040F0010081F84B0022
:102370001DE0039890F84E00022808D1FFE703996A
:1023800091F84B0040F0020081F84B000EE00398FA
:1023900090F84E00032808D1FFE7039991F84B000D
:1023A00040F0040081F84B00FFE7FFE7FFE70398E8
:1023B0002F301D214FF6FF7202F0E6FA0399A1F8C3
:1023C0004C00002004B080BD80B582B00190009127
:1023D0000199A82081F827000198283004214FF6A0
:1023E000FF7202F0D1FA01998885002002B080BD09
:1023F00080B584B0029042F65850C2F200001B2112
:1024000002F0DEFA08B9FFE71BE00299012081F82B
:102410004F000298043042F65851C2F20001009178
:102420001B22FDF711FF009900200190C1F8170051
:1024300048610861C8608860486008608DF80F00D6
:102440000AE041F2E421C2F20001086801300860AC
:10245000FF208DF80F00FFE79DF90F0004B080BD4D
:1024600080B584B003900291019201984068FEF714
:10247000C7F841EC100B9FED501B53EC112B51ECA6
:10248000100BFEF757F868B9FFE70398D0F8230060
:1024900000EE100A1BF0BCFB039910EE100AC1F805
:1024A00023001FE001984068FEF7AAF841EC100BEA
:1024B0009FED431B53EC112B51EC100BFEF755F81D
:1024C00078B9FFE70398D0F8230000EE100A1BF05C
:1024D0009FFB10EE100A039980F00040C1F8230022
:1024E000FFE7FFE701980068FEF78AF841EC100B60
:1024F0009FED351B53EC112B51EC100BFEF71AF826
:10250000F8B9FFE701980068FEF77AF841EC100B84
:102510009FED2F1B53EC112B51EC100BFEF725F800
:1025200078B9FFE70398D0F81F0000EE100A1BF0FF
:102530006FFB10EE100A039980F00040C1F81F00F5
:102540002DE001980068FEF75BF841EC100B9FED61
:10255000221B53EC112B51EC100BFDF7EBFFE8B9EC
:10256000FFE701980068FEF74BF841EC100B9FED78
:102570001C1B53EC112B51EC100BFDF7F6FF68B947
:10258000FFE70398D0F81F0000EE100A1BF040FB95
:10259000039910EE100AC1F81F00FFE7FFE7039848
:1025A000D0F81F00029908600398D0F82300029920
:1025B000486004B080BD00BF33333333333303404E
:1025C0009A99999999990140666666666666F63F9A
:1025D000333333333333FB3FCDCCCCCCCCCC164070
:1025E000000000000000184080B582B0009002207A
:1025F00001F024F842F65851C2F200011B220FF0FC
:10260000B7FF20B9FFE700208DF8070003E0FF20A7
:102610008DF80700FFE79DF9070002B080BD0000BC
:1026200080B584B002908DF807109DF80700C007B0
:1026300090B1FFE7022001F001F80299273127222B
:1026400010F026F820B9FFE700208DF80F0015E004
:10265000FF208DF80F0011E0022000F0EFFF02993B
:102660002E31202210F014F820B9FFE700208DF859
:102670000F0003E0FF208DF80F00FFE79DF90F002A
:1026800004B080BD80B54FF48040012100221BF0D2
:102690006DFEA0F58040B0FA80F0400980BD0000DA
:1026A00084B08DED030ACDED020A9DED030A9DED88
:1026B000021AB1EE411AB4EE410AF1EE10FA07DA4D
:1026C000FFE79DED020AB1EE400A8DED010A18E028
:1026D0009DED030A9DED021AB4EE410AF1EE10FAE7
:1026E00005DDFFE79DED020A8DED000A04E09DED9A
:1026F000030A8DED000AFFE79DED000A8DED010A4A
:10270000FFE79DED010A04B07047000080B543F279
:102710004010C2F2000000684FF480411BF0D4FD6D
:1027200080BD000080B543F24010C2F20000006896
:102730004FF480411BF0C8FD80BD000080B543F21E
:102740003010C2F20000006802211BF0BDFD80BD08
:1027500080B582B040F61832C2F20002002001902B
:102760001221132300F06EFA019802B080BD000020
:1027700080B5082001214FF0FF321BF0F7FD80BD2E
:1027800081B000909FED010A01B070470000C8437E
:1027900080B543F23010C2F20000006801211BF046
:1027A00093FD80BD82B00190019890ED000A002059
:1027B0009FED141AB4EE410AF1EE10FA00901BDA04
:1027C000FFE7019890ED010A00209FED0E1AB4EE8C
:1027D000410AF1EE10FA00900EDAFFE7019890ED51
:1027E000020A9FED081A0020B4EE410AF1EE10FA39
:1027F000B8BF01200090FFE7009800F0010002B090
:10280000704700BF8FC2F53C80B540F61830C2F269
:102810000000C21D01200221062300F013FA00204F
:1028200080BD000080B5042001214FF0FF321BF075
:102830009DFD80BD80B58CB00A9009910A9820B9A1
:10284000FFE7FE208DF82F00B5E0099820B9FFE7DB
:10285000FE208DF82F00AEE042F20C50C2F20000D4
:102860000078C00720B1FFE7FD208DF82F00A2E01F
:102870001BF00AFE43F23011C2F20001086020B9D9
:10288000FFE7FE208DF82F0095E009980A99C861AE
:10289000002008907E21B622069200F087FA069A60
:1028A0000120142100F082FA1E20079000F01CFB8A
:1028B0000799089800F00CFA0899084600F008FA01
:1028C0001E2804D0FFE7FC208DF82F0073E00120C4
:1028D000002100F0FDF90F2804D0FFE7FC208DF85F
:1028E0002F0068E01020039000F0A6FB2020049049
:1028F00000F0A2FB42F6CD32C0F6000201210291A7
:10290000084600F079FE039842F23D71C0F60001DE
:1029100000F006FC049842F29171C0F6000100F04C
:10292000FFFB002005904021AA2200F03FFA029A06
:102930000598412100F03AFA05985321082200F049
:1029400035FA059858210422019200F02FFA019AD5
:1029500005987D2100F02AFA322000F0C5FA029A8B
:102960000F21104600F022FA02980399032200F08A
:102970001DFA0298059A162100F018FA029A1821F9
:10298000104600F013FA02981521802200F00EFA8A
:102990000A2000F0A9FA0299039842F20C52C2F2FE
:1029A0000002117000F082FB049800F07FFB059894
:1029B0008DF82F00FFE79DF92F000CB080BD0000BF
:1029C00084B00290029820B9FFE7FE208DF80F0036
:1029D0006AE040F61831C2F20001B1F80100ADF82A
:1029E0000600B1F80300ADF80400B1F80500ADF839
:1029F0000200BDF9060000EE100AB8EEC00A029807
:102A000080ED000ABDF9040000EE100AB8EEC00A1D
:102A1000029880ED010ABDF9020000EE100AB8EE3E
:102A2000C00A029880ED020A029890ED000A9FED1C
:102A3000201A80EE010A80ED000A029890ED010A4A
:102A400080EE010A80ED010A029890ED020A80EE04
:102A5000010A80ED020A487C897CC00040EA5110DE
:102A6000ADF80000BDF90000B0F5806F07DBFFE7AF
:102A7000BDF80000A0F50060ADF80000FFE7BDF96B
:102A8000000000EE100AB8EEC00AB4EE001A20EE04
:102A9000010AB3EE071A30EE010A029880ED060A29
:102AA00000208DF80F00FFE79DF90F0004B070477C
:102AB00000A0AA4584B00290029820B9FFE7FE204A
:102AC0008DF80F007AE040F61830C2F20000B0F83E
:102AD0000710ADF80610B0F80910ADF80410B0F802
:102AE0000B00ADF80200BDF9060000EE100AB8EECA
:102AF000C00A029880ED030ABDF9040000EE100A36
:102B0000B8EEC00A029880ED040ABDF9020000EE9A
:102B1000100AB8EEC00A029880ED050A029890EDFE
:102B2000030A9FED281A80EE010A80ED030A02983D
:102B300090ED040A80EE010A80ED040A029890EDFF
:102B4000050A80EE010A80ED050A029890ED030A5D
:102B50009FED1D1A20EE010A80ED030A029890ED08
:102B6000040A20EE010A80ED040A029890ED050A9D
:102B700020EE010A80ED050A0298C16991ED001A64
:102B800090ED030A30EE410A80ED030A0298C16914
:102B900091ED011A90ED040A30EE410A80ED040A2D
:102BA0000298C16991ED021A90ED050A30EE410AD2
:102BB00080ED050AFE208DF80F00FFE79DF90F005C
:102BC00004B070476F12034235FA8E3C80B5002086
:102BD000C4F20200102108F077FD80B9FFE7002061
:102BE000C4F202001021012208F098FD43F23010D7
:102BF000C2F20000006808211BF066FBFFE740F20C
:102C00000040C4F20200012108F05EFD88B9FFE730
:102C100040F20040C4F202000122114608F07EFD9D
:102C200043F23010C2F20000006804211BF04CFB9C
:102C3000FFE780BD80B5032001214FF0FF321BF07C
:102C400095FB80BD80B586B08DF817008DF8161005
:102C500004928DF80F30049808B9FFE736E09DF82C
:102C600017000146029120B1FFE70298012808D021
:102C700010E00020C4F202001021002208F04EFDF6
:102C800008E040F20040C4F202000121002208F0F6
:102C900045FDFFE79DF8160040F0800040F62B311F
:102CA000C2F20001009108700120019000F084FC44
:102CB0000099019A14230BF06FFF019800F07CFC3F
:102CC00004999DF80F200BF029FEFFE706B080BDA8
:102CD00080B586B08DF816008DF81510012000F033
:102CE00003F99DF816000146049120B1FFE704980E
:102CF000012808D010E00020C4F2020010210022B8
:102D000008F00CFD08E040F20040C4F2020001218E
:102D1000002208F003FDFFE79DF8150040F0800059
:102D200040F62B31C2F200010191087001200090A1
:102D300000F042FC009A0199142302930BF02CFF3F
:102D4000009800F039FC0199029B02220BF0CEFCA6
:102D50009DF816000146039120B1FFE70398012872
:102D60000FD01EE00020C4F202001021012208F062
:102D7000D5FC40F62B30C2F2000040788DF81700E9
:102D80000FE040F20040C4F202000122114608F0B8
:102D9000C5FC40F62B30C2F2000000788DF8170019
:102DA000FFE79DF8170006B080BD000080B584B035
:102DB0008DF80F008DF80E108DF80D209DF80E0087
:102DC00000F07F0040F62B31C2F2000108709DF840
:102DD0000D004870012000F087F89DF80F000146B3
:102DE000029120B1FFE70298012808D010E00020EE
:102DF000C4F202001021002208F090FC08E040F22A
:102E00000040C4F202000121002208F087FCFFE725
:102E1000012000F0D1FB40F62B31C2F2000102226A
:102E200014230BF0B9FE9DF80F000146019120B16B
:102E3000FFE70198012808D010E00020C4F202004A
:102E40001021012208F06AFC08E040F20040C4F2C0
:102E500002000122114608F061FCFFE704B080BDCA
:102E600083B08DF807009DF807000146009150B12E
:102E7000FFE7009801280CD1FFE741F69800C2F265
:102E80000000029008E041F67000C2F200000290DB
:102E900002E000200290FFE7029803B070470000B4
:102EA00082B08DF806008DF805100092009820B9C8
:102EB000FFE7FE208DF8070011E000989DF806104E
:102EC00040F25043C2F20003342211FB02319DF85C
:102ED000052041F8220000208DF80700FFE79DF94A
:102EE000070002B07047000080B586B004901AF069
:102EF00073FF01464FF47A70B0FBF1F00390049831
:102F00000399B0FBF1F002901AF028FF0146481C2B
:102F1000019198B1FFE70198022820D3FFE70198BB
:102F200002280FD0FFE701980338022806D3FFE7F5
:102F300001986FF00041884215D1FFE7FF208DF81E
:102F4000170014E0029818B1FFE70298009002E021
:102F500001200090FFE700981AF0BAFE03E0049801
:102F600007F046FEFFE700208DF81700FFE79DF908
:102F7000170006B080BD000080B588B007900798A4
:102F8000E0B1FFE707980B2818D8FFE707980490EF
:102F900000200290022006900120059007F088FF93
:102FA000FFE7322004F0D0FA08B1FFE7F9E702A802
:102FB00001A907F03FFE07F0EDFEFFE708B080BD76
:102FC00080B584B003900291019202980399019A0E
:102FD000FDF73AF904B080BD80B584B0039002914A
:102FE000019207F065FFFFE70198C0B1FFE7FFE737
:102FF000322004F0A9FA08B1FFE7F9E70399029833
:1030000002780023184607F0CFFE039801300390A2
:10301000029801300290019801380190E4E707F02E
:10302000B9FE04B080BD000080B582B00190019867
:103030001DF010F802B080BD80B582B0ADF804007C
:10304000BDF804000138014600911F2822D80099DC
:10305000DFE801F0182020202020201C2020202044
:103060002020201020202020202020202020202070
:10307000202020140A2008F079FF0FE0172008F024
:1030800075FF0BE0062008F071FF07E0092008F04B
:103090006DFF03E0FF208DF8070003E000208DF8AE
:1030A0000700FFE79DF9070002B080BD80B582B040
:1030B000ADF80400BDF804000138014600911F2856
:1030C00022D80099DFE801F0182020202020201CC1
:1030D0002020202020202010202020202020202000
:1030E00020202020202020140A2008F057FF0FE085
:1030F000172008F053FF0BE0062008F04FFF07E011
:10310000092008F04BFF03E0FF208DF8070003E0E3
:1031100000208DF80700FFE79DF9070002B080BD91
:1031200083B0ADF808000191019820B9FFE7FE20B7
:103130008DF80B0025E000208DF80300FFE79DF8D7
:1031400003000F2819DCFFE7BDF808009DF8031005
:10315000C840C00750B1FFE701989DF8032040F236
:10316000D441C2F2000141F8220006E0FFE79DF8D9
:10317000030001308DF80300E1E700208DF80B001B
:10318000FFE79DF90B0003B07047000080B588B0E1
:10319000082004900120059000200690079041F639
:1031A0002800C2F2000004A904F0D6FE18B1FFE71F
:1031B00003F01AFFFFE741F62800C2F20000019079
:1031C00005F004FB0198052105F06AFA019805F065
:1031D00023F803909DED030AB8EE400A40F2444004
:1031E000C2F2000090ED001A20EE010A9FED041AD1
:1031F00020EE010A8DED020A9DED020A08B080BDA5
:103200005D74214180B588B01020049001200590A4
:1032100000200690079041F2E070C2F2000004A97D
:1032200004F09AFE18B1FFE703F0DEFEFFE741F27B
:10323000E070C2F20000019005F0C8FA0198052183
:1032400005F02EFA019804F0E7FF03909DED030AC4
:10325000B8EE400A40F24440C2F2000090ED001A7D
:1032600020EE010A8DED020A9DED020A9FED061A7D
:1032700030EE010A9FED051A20EE010AB3EE091A9D
:1032800030EE010A08B080BD5C8F42BF0000C84329
:1032900080B588B006AA0392024603988DF81E20D6
:1032A0008DF81D1080ED000A90ED000AB7EE001AAF
:1032B000B4EE410AF1EE10FA04DDFFE7FF208DF8CD
:1032C0001F0097E0039890ED000A9FED4C1A20EE46
:1032D000010ABDEEC00A10EE100AADF812009DF80A
:1032E0001E0001460291F0B1FFE70298012804D0C8
:1032F000FFE7029802280BD020E0BDF8120042F24E
:103300002C31C2F200010968C8630820059015E05D
:10331000BDF8120042F22C31C2F200010968886344
:10332000042005900AE0BDF8120042F22C31C2F2EE
:1033300000010968486300200590FFE79DF81D0023
:103340000146019140B1FFE70198012814D0FFE741
:103350000198022820D049E0059942F22C30C2F2AF
:1033600000000EF049F8059A42F22451C2F2000121
:1033700008681043086039E0059942F22C30C2F227
:1033800000000EF01BFA059A42F22451C2F200012D
:1033900008689043086029E042F22450C2F200001D
:1033A00000680599084210D0FFE7059942F22C30D9
:1033B000C2F200000EF002FA059A42F22451C2F263
:1033C00000010868904308600FE0059942F22C3034
:1033D000C2F200000EF010F8059A42F22451C2F237
:1033E0000001086810430860FFE7FFE700208DF840
:1033F0001F00FFE79DF91F0008B080BD00FF7F4759
:1034000080B582B0019001981CF000FB02B080BD35
:1034100080B586B004A90291014602988DF8161075
:1034200080ED000A90ED000AB7EE001AB4EE410AF2
:10343000F1EE10FA04DDFFE7FF208DF817006AE0D7
:10344000029890ED000AB5EE400AF1EE10FA03DAA8
:10345000FFE700200490FFE79DF816000146019168
:1034600020B1FFE70198012815D029E0029890EDDE
:10347000000A42F25420C2F20000006890ED0B1ADC
:10348000B8EE411A20EE010ABDEEC00A10EE100A95
:10349000ADF80E0014E0029890ED000A42F20C2004
:1034A000C2F20000006890ED0B1AB8EE411A20EE4F
:1034B000010ABDEEC00A10EE100AADF80E00FFE7DB
:1034C000BDF80E0001281DDBFFE79DF81600014640
:1034D000009120B1FFE70098012809D011E0BDF864
:1034E0000E0042F25421C2F200010968486308E06C
:1034F000BDF80E0042F20C21C2F2000109684863D7
:10350000FFE704E09DF8160000F02CF8FFE700202C
:103510008DF81700FFE79DF9170006B080BD000089
:1035200080B582B08DF807009DF807000146009134
:1035300020B1FFE70098012808D00FE042F25420A4
:10354000C2F2000000210DF057FF07E042F20C200C
:10355000C2F2000000210DF04FFFFFE7002002B093
:1035600080BD000080B584B08DF80F009DF80F007D
:103570000146029120B1FFE70298012808D00FE030
:1035800042F25420C2F2000000210EF017F907E0C9
:1035900042F20C20C2F2000000210EF00FF9FFE70A
:1035A00041F20040C4F2020040210022019208F0E2
:1035B000B5F8019804B080BD83B08DF807009DF880
:1035C00007000146009120B1FFE70098012806D0CE
:1035D0000BE042F2B410C2F20000029008E042F2A6
:1035E0005C10C2F20000029002E000200290FFE7AF
:1035F000029803B07047000082B08DF806008DF885
:1036000005100092009820B9FFE7FE208DF8070012
:1036100010E000989DF8062040F29851C2F2000197
:1036200001EB42119DF8052041F8220000208DF8A1
:103630000700FFE79DF9070002B0704783B08DF8DF
:1036400007009DF807000146009140B1FFE7009890
:1036500001280AD0FFE7009802280CD011E042F2BE
:103660004840C2F2000002900EE042F20440C2F272
:103670000000029008E042F28C40C2F2000002908A
:1036800002E000200290FFE7029803B070470000BC
:1036900080B582B00190019800680068C0060028DB
:1036A0002AD5FFE7FFE70020009001980068006836
:1036B000009001980068406800900098FFE701982A
:1036C00016F0EEF800EBC00140F21860C2F2000004
:1036D00000EB8100006A70B1FFE7019816F0E0F896
:1036E00000EBC00140F21860C2F2000000EB810064
:1036F000006A8047FFE7FFE702B080BD82B08DF827
:1037000006008DF805100092009820B9FFE7FE2012
:103710008DF8070012E000989DF8061001EBC10239
:1037200040F21861C2F2000101EB82019DF8052010
:1037300041F8220000208DF80700FFE79DF90700FF
:1037400002B0704783B080B585B0099308920791A5
:1037500003900020ADF8060007A80290039A029B90
:1037600049F29830C2F2000040F2FF311EF0BCFF77
:10377000ADF80600BDF8060001280CDBFFE7BDF838
:10378000061049F29830C2F2000000F02FF8002035
:103790008DF8130003E0FE208DF81300FFE79DF97C
:1037A000130005B0BDE8804003B0704749F21830FF
:1037B000C2F200000078704780B582B00090009897
:1037C00020B9FFE7FE208DF807000BE0009841F2DA
:1037D0003C31C2F20001086000F068FC00208DF866
:1037E0000700FFE79DF9070002B080BD80B582B0F9
:1037F0000190ADF8021000208DF80100FFE701985C
:10380000BDF8021000F078FC48B1FFE79DF8010018
:1038100001308DF801000A20FFF766FB00E005E0AB
:10382000FFE79DF801000328E9DBFFE7002002B075
:1038300080BD0000FFE7FEE780B541F67000C2F2F0
:10384000000005F0E7FC80BD80B541F67000C2F2D3
:10385000000005F0DFFC80BD80B541F69800C2F2A3
:10386000000005F0D7FC80BD80B541F69800C2F29B
:10387000000005F0CFFC80BD80B582B00020019033
:10388000FFF7EEFA019942F6C822C2F20002009256
:1038900002F11C0305F0B4FB0099019B41F240309A
:1038A000C2F200000068D0F8C8001A461AF02AFCDC
:1038B00002B080BD80B582B001200090FFF7D0FA41
:1038C000009942F6EC22C2F20002019202F11C03BE
:1038D00005F096FB019941F24030C2F20000006809
:1038E000D0F8C80000231A461AF00CFC02B080BDC4
:1038F00083B0029001918DED000A029900200871B9
:1039000000980199086003B07047000080B588B046
:10391000079006910798006805909DED050A9FEDB8
:10392000181A20EE010ABDEEC00A10EE100AADF81A
:10393000120042F61031C2F2000101914FF40470FE
:103940000860002003908860C860082008619DF826
:103950001320084600F8182F0290BDF81200487690
:103960000698D0F8B400C078FFF77AFA0199029A65
:10397000069BC43305F082F8039808B080BD00BFF1
:103980000000C84282B0019000910098008800EECB
:10399000100AB8EEC00A9FED151A80EE010A0198D0
:1039A00080ED000A0098408800EE100AB8EEC00AC8
:1039B00080EE010A019880ED010A0098808800EEEF
:1039C000100AB8EEC00A80EE010A019880ED020AE2
:1039D0000098C08800EE100AB8EEC00A80EE010A16
:1039E000019880ED030A02B0704700BF0000C84292
:1039F00083B001900091019820B9FFE700208DF875
:103A00000B000AE00198006800990840401AB0FADB
:103A100080F040098DF80B00FFE79DF80B0003B024
:103A20007047000083B001900091019820B9FFE732
:103A3000FE208DF80B0008E0009A01990868904379
:103A4000086000208DF80B00FFE79DF90B0003B024
:103A50007047000082B000900098006846F60001B0
:103A6000C4F20001884204D1FFE701208DF807006D
:103A700010E00098006846F20041C4F2000188425C
:103A800004D1FFE700208DF8070003E003208DF844
:103A90000700FFE79DF8070002B0704780B592B0BD
:103AA00010900F91109820B9FFE7FE208DF8470085
:103AB0007DE042F20D50C2F200000078C00720B154
:103AC000FFE7FD208DF8470071E01AF0DDFC43F2BE
:103AD0003411C2F20001086020B9FFE7FE208DF822
:103AE000470064E020202421002204921AF08AFA80
:103AF0001099C1F8C8000F981099C1F8B40005A832
:103B000002902821FCF7B9FB04980A9005900690D2
:103B10000B90012103910C91079008900D910E21BB
:103B200001910E910990FFF79BF9029905F0CAF8EF
:103B30000498FFF795F906F077F9049843F67902AF
:103B4000C0F600020621FFF7ABF90498FFF788F9E9
:103B5000022104F057FF019903980A910990FFF799
:103B60007FF9029905F0AEF80398FFF779F906F0AE
:103B70005BF9039843F6B502C0F600020821FFF78F
:103B80008FF90398FFF76CF9102104F03BFF0399BC
:103B90000498109A41F24033C2F200031A6042F2D4
:103BA0000D52C2F2000211708DF84700FFE79DF937
:103BB000470012B080BD000080B590B08DF83E0087
:103BC0000E910D920E9820B9FFE7FE208DF83F0070
:103BD00013E19DF83E000146079158B1FFE70798B1
:103BE0000138022869D3FFE7079803380228C0F09C
:103BF000A980FDE00E9890ED000A9FED821A20EE5C
:103C0000010ABDEEC00A10EE100AADF832000E989F
:103C100090ED010A20EE010ABDEEC00A10EE100A76
:103C2000ADF830000E9890ED020A20EE010ABDEECC
:103C3000C00A10EE100AADF82E000E9890ED030A9F
:103C400020EE010ABDEEC00A10EE100AADF82C00FD
:103C500042F61031C2F2000105914FF40070086085
:103C600000208860C860082008619DF8332008465D
:103C700000F8182F0690BDF8320048769DF8310004
:103C80008876BDF83000C8769DF82F000877BDF81B
:103C90002E0048779DF82D008877BDF82C00C87756
:103CA0000D98D0F8B4000078FFF7DAF80599069A75
:103CB0000D9BB83304F0E2FE9BE00E9890ED040AF1
:103CC0009FED521A20EE010ABDEEC00A10EE100A56
:103CD000ADF82A000E9890ED050A20EE010ABDEE1F
:103CE000C00A10EE100AADF8280042F61031C2F2F8
:103CF0000001039140F2FF20086000208860C86046
:103D000008220A619DF82B300A4602F8183F0492F7
:103D1000BDF82A204A769DF829208A76BDF8282009
:103D2000CA76087748778877C8770D98D0F8B400B6
:103D30004078FFF795F80399049A0D9BBC3304F083
:103D40009DFE56E00E9890ED070A9FED2E1A20EE8C
:103D5000010ABDEEC00A10EE100AADF826000E985A
:103D600090ED080A20EE010ABDEEC00A10EE100A1E
:103D7000ADF824000E9890ED090A9FED231A20EE6D
:103D8000010ABDEEC00A10EE100AADF8220042F69C
:103D90001031C2F20001019140F2FF1008600020D2
:103DA0008860C86008220A619DF827300A4602F838
:103DB000183F0292BDF826204A769DF825208A7683
:103DC000BDF82420CA769DF823200A77BDF822206A
:103DD0004A778877C8770D98D0F8B4008078FFF7D5
:103DE0003FF80199029A0D9BC03304F047FE00E0B2
:103DF000FFE700208DF83F00FFE79DF93F0010B07E
:103E000080BD00BF0000804600401C460060EA46BE
:103E100083B00290019101980178407840EA012036
:103E2000ADF8020001980179407940EA0120ADF82F
:103E30000000BDF8020000EE100AB8EEC00A9FEDC7
:103E4000191A80EE010A9FED181A20EE010A029855
:103E500080ED000A01988178C07840EA012000B224
:103E600000EE100AB8EEC00A029880ED010ABDF912
:103E7000000000EB8000800000EE100AB8EEC00ADF
:103E80009FED0A1A80EE010A029880ED020A01985D
:103E9000807900EE100AB8EE400A029880ED030A1D
:103EA00003B0704700000046DB0FC94000008046A9
:103EB00080B586B004900391049820B9FFE7FE20F6
:103EC0008DF8170089E0039820B9FFE7FE208DF8F0
:103ED000170082E0039800680190A0F201200428F6
:103EE00017D3FFE70198A0F20520032828D3FFE7A6
:103EF0000198A0F2092002283AD3FFE7019840F286
:103F0000112188424CD0FFE70198B0F5207F53D0B3
:103F10005EE003980068A0F20120029004980299E4
:103F200000EB0110043003991C31FFF771FF029977
:103F3000012000FA01F2049908681043086048E083
:103F400003980068A0F2052002900298811D0120CC
:103F500000FA01F204990868104308600498029975
:103F600000EB0110643003991C31FFF751FF30E082
:103F700003980068A0F2092002900298011D012018
:103F800000FA01F204990868104308600498029945
:103F900000EB0110443003991C31FFF739FF18E0A2
:103FA0000499086840F40070086004989C300399F4
:103FB0001C31FFF7E7FC0CE00499086840F48060CE
:103FC00008600498AC3003991C3100F00BF800E055
:103FD000FFE700208DF81700FFE79DF9170006B0F6
:103FE00080BD000082B00190009100980178427875
:103FF0008078000440EA0220084400EE100AB8EE7F
:10400000C00A9FED0A1A80EE010A019880ED000AAD
:104010000098C0780199087100990879497940EAB7
:1040200001200199C88002B0704700BF00007A44A7
:1040300084B08DF80F000291ADF806209DF80F00B6
:104040000146009123281DD80099DFE801F01213E2
:104050001415161B1B1B1B1B1B1B1B1B1B1B1B1BC2
:104060001B1B1B1B1B1B1B1B1B1B1B1B1B1B1718A7
:10407000191A08E007E006E005E004E003E002E0CA
:1040800001E000E0FFE7002004B070470020704727
:1040900080B541F21050C2F2000049F21831C2F26C
:1040A000000116F02BFD002080BD000080B541F21C
:1040B0001050C2F2000016F0DBFC002080BD0000B2
:1040C00080B582B00190009141F23C30C2F2000014
:1040D000006801211AF0F8F8002002B080BD00004D
:1040E00083B0029001918DF8032000208DF802002A
:1040F0009DF9020003B0704780B586B00490ADF81A
:104100000E1000208DF80D0041F21050C2F2000098
:10411000D0F8BC0202900298D0F8140220B1FFE758
:1041200001208DF8170013E00499BDF80E2041F22C
:104130001050C2F20000019016F0FAFC019816F03F
:10414000E5FD8DF80D009DF80D008DF81700FFE7D7
:104150009DF8170006B080BD80B588B00690059127
:104160008DF8132005989DF8131000F08DF88DF848
:10417000120005989DF8131000F078F88DF81100E2
:104180009DF8120010280DD1FFE70698007F00F07F
:1041900001008DF810000598007B00F001008DF8FB
:1041A0000F0025E09DF8120011280DD1FFE70698B9
:1041B000407F00F001008DF810000598407B00F072
:1041C00001008DF80F0012E00698C08B9DF81210C8
:1041D000C84000F001008DF81000059880889DF817
:1041E0001210C84000F001008DF80F00FFE7FFE754
:1041F0009DF811000146029140B1FFE702980128A5
:1042000017D0FFE70298022824D02AE09DF810106A
:104210000020C907019031B1FFE79DF80F0080F041
:1042200001000190FFE7019800F001008DF81F00E8
:1042300017E09DF810100020C907009021B9FFE792
:104240009DF80F000090FFE7009800F001008DF846
:104250001F0006E09DF8100000F001008DF81F001F
:10426000FFE79DF81F0008B080BD000082B00190FC
:104270008DF80310019800699DF8031000EB4100D0
:10428000007A02B07047000082B001908DF80310F0
:10429000019800699DF8031000EB4100407A02B0DC
:1042A0007047000081B000900098407800F0010055
:1042B00001B0704783B001900091019820B9FFE7E9
:1042C000FF208DF80B000FE0009820B9FFE7FF20DA
:1042D0008DF80B0008E00199002008700099019A00
:1042E00011618DF80B00FFE79DF90B0003B07047DB
:1042F00083B001908DF803109DF80300102807D1BA
:10430000FFE70198007F00F001008DF80B0015E039
:104310009DF80300112807D1FFE70198407F00F0C6
:1043200001008DF80B0009E00198C08B9DF8031087
:10433000C84000F001008DF80B00FFE79DF80B006E
:1043400003B0704784B0029001918DED000A02988D
:1043500020B9FFE7FF208DF80F002BE0019820B96E
:10436000FFE7FF208DF80F0024E002980068019914
:104370008862029840680199C86201988078C007F5
:10438000A0B1FFE70298007EC00748B1FFE701999E
:10439000022081F834000199012081F8360004E000
:1043A0000199022081F83400FFE7FFE700208DF833
:1043B0000F00FFE79DF90F0004B0704780B584B08F
:1043C000029001918DED000A029820B9FFE7FF20CD
:1043D0008DF80F0056E0019820B9FFE7FF208DF817
:1043E0000F004FE002980421FFF782FF80B1FFE742
:1043F00002980521FFF77CFF50B1FFE702980621E4
:10440000FFF776FF20B1FFE7019901200870FFE771
:1044100002980421FFF76CFF80B1FFE702980521A5
:10442000FFF766FF50B1FFE702980721FFF760FF33
:1044300020B1FFE7019900200870FFE70298407D56
:1044400020B1FFE70298007D20B9FFE7019800F056
:104450004BFA13E001980078C00738B1FFE70298E3
:1044600001999DED000A00F011F806E0029801990B
:104470009DED000A00F08EF9FFE7FFE700208DF8C0
:104480000F00FFE79DF90F0004B080BD80B584B038
:10449000039002918DED010A0299012081F8240018
:1044A0000398B0F9160000EE100AB8EEC00A9DEDB0
:1044B000011A20EE010A0298016991ED001A20EE1E
:1044C000010A80ED0A0A0398B0F91800404200EE94
:1044D000100AB8EEC00A9DED011A20EE010A0298FA
:1044E000016991ED001A20EE010A80ED0B0A029895
:1044F0000022C26102988261029880F838200398F5
:104500000299FFF729FE58B1FFE70298016991ED82
:10451000091A90ED070A30EE010A80ED070AFFE75D
:10452000039802990122FFF717FE58B1FFE702989E
:10453000016991ED091A90ED070A30EE410A80ED0C
:10454000070AFFE7039802990222FFF705FE58B118
:10455000FFE70298016991ED091A90ED060A30EE25
:10456000410A80ED060AFFE7039802990322FFF74C
:10457000F3FD58B1FFE70298016991ED091A90ED3A
:10458000060A30EE010A80ED060AFFE70398029959
:104590000422FFF7E1FDA8B1FFE70298016991ED60
:1045A0000A1A90ED060A20EE010A80ED060A02982A
:1045B000016991ED0A1A90ED070A20EE010A80EDDB
:1045C000070AFFE7039802990522FFF7C5FDA8B186
:1045D000FFE70298016991ED0B1A90ED060A20EEB3
:1045E000010A80ED060A0298016991ED0B1A90ED1F
:1045F000070A20EE010A80ED070AFFE703980299F7
:104600000622FFF7A9FD48B1FFE70299022081F8D1
:1046100034000299012081F8360008E00299022056
:1046200081F834000299002081F83600FFE70398F2
:1046300002990722FFF790FDB0B1FFE7029991F8C8
:104640003500013081F83500029991F835004AF6BD
:10465000AB22CAF6AA22A0FB0232520802EB4202A7
:10466000801A81F83500FFE7039802990B22FFF7C3
:1046700073FD38B1FFE70299042008750299022002
:104680004875FFE7039802990A22FFF765FD40B1DC
:10469000FFE7029991F837200120904381F8370015
:1046A000FFE7039802990822FFF756FD20B3FFE7C2
:1046B0000298807B02280BD1FFE702983930042151
:1046C00000F020F90299002048700299887312E0E6
:1046D0000298807B012801D1FFE70BE00298393076
:1046E000032100F00FF9029902208873029901203A
:1046F0004870FFE7FFE7FFE7039802990922FFF7F9
:104700002BFDD8B1FFE70298807B01280BD1FFE792
:10471000029900204870029988730298393002216A
:1047200000F0F0F809E002980121817302984170CD
:104730000298393000F0E6F8FFE703E00299002024
:104740004870FFE7039802990C22FFF705FD28B196
:10475000FFE70299012081F83800FFE703980299EA
:104760000D22FFF7F9FC20B1FFE70299022008753E
:10477000FFE70398C08B029988800299039AD2F8C8
:104780001600D2F81A20C1F80A20C1F8060004B0B9
:1047900080BD000085B0049003918DED020A04985D
:1047A000407D0146019103282AD80199DFE801F0F4
:1047B0002002140B039901200875039900208873C7
:1047C000039948701CE003990220087503990120A1
:1047D00088730399487013E00399042008750399BE
:1047E000002048750399012088730399487007E0F9
:1047F0000399002008750399887303994870FFE7AF
:104800000498007D0146009103283AD80099DFE81A
:1048100001F02E021C0D0399012081F82400039958
:1048200081F834000399002088702AE00399012060
:1048300081F82400039A002182F83610039A02219D
:1048400082F83410039988701BE00399012081F8E5
:104850002400039A022182F83410039A002182F87E
:104860003510039981F836000399887009E003999F
:10487000002081F82400039981F83400039988709E
:10488000FFE70398807B28B1FFE703984078C007D3
:1048900038BBFFE704980068039988610498406872
:1048A0000399C861049890ED020A9DED021A20EE6A
:1048B000010A0398016991ED011A20EE010A80EDC9
:1048C0000A0A049890ED030A9DED021A20EE010AEF
:1048D0000398016991ED011A20EE010A80ED0B0A9F
:1048E000FFE705B07047000081B0009000990020FC
:1048F0000875009981F82400009981F8340001B00E
:104900007047000083B001908DF80310019820B922
:10491000FFE7FF208DF80B001BE00198C07802280C
:1049200006DCFFE70198C078B0F1FF3F04DCFFE749
:10493000FF208DF80B000CE09DF803000199CA7868
:1049400088540199C8780130C87000208DF80B0098
:10495000FFE79DF90B0003B07047000081B0ADF890
:1049600002008DF80110BDF802109DF801004840CA
:10497000C2B244F67060C0F6020030F8120080EA5D
:10498000112001B07047000080B584B003900291FF
:10499000ADF80620FFE70298411E029158B1FFE7EB
:1049A000BDF8060003994A1C03920978FFF7D6FF69
:1049B000ADF80600EFE7BDF8060004B080BD0000CA
:1049C00080B584B0029001910198012804D8FFE7D6
:1049D00000208DF80F001BE00298019902394FF674
:1049E000FF72FFF7D1FFADF80200BDF80200029A96
:1049F000019901F001031A4421F00101114431F839
:104A0000021C401AB0FA80F040098DF80F00FFE751
:104A10009DF80F0004B080BD83B0029001918DF825
:104A20000320FFE70198411E019178B1FFE79DF84F
:104A3000030002994A1C02920978414045F2700035
:104A4000C0F60200405C8DF80300EBE79DF8030020
:104A500003B0704780B584B002900191019801289D
:104A600004D8FFE700208DF80F0015E002980199A7
:104A70000139FF22FFF7D0FF8DF803009DF80300F6
:104A8000029A0199114411F8011C401AB0FA80F001
:104A900040098DF80F00FFE79DF80F0004B080BDBE
:104AA00085B002A900910146009880ED010AC0ED91
:104AB000000A8DF8071090ED010AB5EE400AF1EEFC
:104AC00010FA03D1FFE7002004906DE09DF8070085
:104AD000C007A0B3FFE7009890ED010AB2EE0E1AEE
:104AE000B4EE410AF1EE10FA06D1FFE74FF20000F2
:104AF000C4F29150049057E0009890ED010AB3EE93
:104B0000021AB4EE410AF1EE10FA06D1FFE748F2BC
:104B10000000C4F2A250049046E0009890ED010A13
:104B2000B3EE0E1AB4EE410AF1EE10FA06D1FFE729
:104B30004BF20000C4F2E550049035E022E000980A
:104B400090ED010AB2EE041AB4EE410AF1EE10FA49
:104B500006D1FFE741F20000C4F28B50049023E03D
:104B6000009890ED010AB3EE001AB4EE410AF1EE9E
:104B700010FA06D1FFE744F20000C4F2B5500490E9
:104B800012E0FFE7009890ED010A9FED0A1A20EE6F
:104B9000010A90ED001A9FED082A21EE021A80EE1C
:104BA000010A80ED020AFFE7009890ED020A05B0C5
:104BB000704700BF00007042DB0FC94080B584B071
:104BC00003900291019202980078012805D0FFE736
:104BD00002988068019908600CE0029890ED010A43
:104BE000D0ED020A90ED031A0FF08CFD019880EDD4
:104BF000000AFFE70399012008710398D0ED020A2B
:104C000090ED030AB2EE081A00F0BAF8039880EDAE
:104C1000000A04B080BD000082B0019000910198AC
:104C2000006800990860019800790099087102B045
:104C30007047000084B08DED030A9DED030A20EE5D
:104C4000000A8DED010A9DED010A9DED031A20EE8B
:104C5000010A8DED000A9DED030A9FED3E1AB4EEA8
:104C6000410AF1EE10FA03DAFFE70020029053E068
:104C70009DED030A9FED381AB4EE410AF1EE10FAE9
:104C80001DDAFFE79DED000A9FED391A20EE010ABB
:104C90009DED011A9FED372A21EE021A30EE010A2E
:104CA0009DED031A9FED342A21EE021A30EE010A1F
:104CB0009FED321A30EE010A8DED020A2BE09DEDD8
:104CC000030A9FED261AB4EE410AF1EE10FA1DDA3E
:104CD000FFE79DED000A9FED221A20EE010A9DEDEF
:104CE000011A9FED202A21EE021A30EE010A9DEDF5
:104CF000031A9FED1D2A21EE021A30EE010A9FEDE4
:104D00001B1A30EE010A8DED020A03E04FF07E50CF
:104D10000290FFE7FFE7FFE79DED020AB5EE400ACC
:104D2000F1EE10FA03DAFFE7002002900EE09DEDAD
:104D3000020AB7EE001AB4EE410AF1EE10FA04DDF1
:104D4000FFE74FF07E500290FFE7FFE79DED020A7C
:104D500004B0704700009C413333AF410000CC41A8
:104D600061E0B93C46B6D3BF295C21423333A4C3CA
:104D70001399B93BFB5CADBEE17AD84014AE34C2A6
:104D800084B08DED030ACDED020A8DED011A9DED83
:104D9000030A9DED012A30EE420A9DED021A31EE22
:104DA000421A80EE010A8DED000A9DED000AB5EE73
:104DB000400AF1EE10FA03DAFFE7002000900EE05F
:104DC0009DED000AB7EE001AB4EE410AF1EE10FABA
:104DD00004DDFFE74FF07E500090FFE7FFE79DED19
:104DE000000A04B07047000080B588B08DED070A56
:104DF000CDED060A05909DED050AB8EE400A10EECD
:104E0000100AFBF7FDFB41EC100B9FED2B1B53EC45
:104E1000112B51EC100BFBF71BFB41EC100B51EC71
:104E2000100BFBF700FC00EE100A1EF0A5FA9FED38
:104E3000261A20EE010A10EE100AFBF7E1FB41EC06
:104E4000100B51EC100B9FED1E0B52EC103BD20FD0
:104E500062F3DF7141EC100B8DED020B0798FBF74D
:104E6000CFFB9DED021B41EC100B51EC110B53ECF1
:104E7000102BFBF746FA41EC100B51EC100BFBF733
:104E8000D2FB04909DED040A9FED101AB4EE410A86
:104E9000F1EE10FA05DDFFE79DED060A8DED010A42
:104EA00004E09DED040A8DED010AFFE79DED010A86
:104EB00008B080BD00BF00BFFCA9F1D24D62503FD9
:104EC0000000000000000000CDCC4C3ECDCC4C3F9B
:104ED00080B58EB007AB05930C900B910A920C989D
:104EE00020B9FFE7FE208DF8370067E10B9820B965
:104EF000FFE7FE208DF8370060E10A990C98026800
:104F0000891A00EE101AB8EE400A9FEDAE1A80EE34
:104F1000010A80ED010A0A980C9908600C980B9917
:104F200009780A9A00F02EFB0C98007C0146049147
:104F300000B3FFE7049801280DD0FFE7049802387A
:104F4000032817D3FFE7049805280AD0FFE7049841
:104F500006280FD04CE00C99002048610C9988611C
:104F600046E00B9840680C9948610B9840680C9992
:104F700088613DE005980C9991ED080AC96891EDAA
:104F8000001A30EE410A80ED020A90ED020A1EF08E
:104F9000AFF8059880ED010A90ED020A1EF0ECF9D9
:104FA000059880ED000A90ED010A0B9991ED011A28
:104FB00091ED022A20EE010A90ED001A21EE021A6C
:104FC00030EE410A0C9981ED050A90ED000A0B992B
:104FD00091ED011A91ED022A20EE010A90ED011ADD
:104FE00021EE021A30EE010A0C9880ED060AFFE766
:104FF0000C98007C01460391062848D80399DFE805
:1050000001F00404081A300408000C990020C8615B
:105010003DE00C9901F13800CA6892ED000AD1ED2B
:10502000011AD1ED080A9FED6B1A0FF0D1F80C9818
:1050300080ED070A2BE00C9901F13800CA6892ED67
:10504000000A9FED631A30EE010AD1ED011AD1ED8D
:10505000080A9FED601A0FF0BBF80C9880ED070A64
:1050600015E00C9890ED0B0A8DED020A0A989FED61
:10507000560ADFED560AFFF7B7FEB0EE401A9DED77
:10508000020A20EE010A0C9880ED070AFFE70C9B4C
:1050900003F1120003F114011A6B93F911309FED23
:1050A0004E0A0EF019FD00208DF81B00FFE79DF859
:1050B0001B000C9991F9111088427BDAFFE70C98DC
:1050C000416A406F9DF81B2000EB421001EB82010A
:1050D00091ED000A0DF06CFC0C98406A9DF81B10D5
:1050E00000EB810080ED000A0C98007C01460191E4
:1050F000E0B3FFE701980138052804D3FFE70198E2
:10510000062821D03AE00C99486B9DF81B30C3EB80
:10511000031200EB82000A6B02EB830292ED000A9D
:105120004A6A02EB8302D2ED000AD1ED011A9FED2B
:10513000291A0FF04DF80C98C06F9DF81B1000EB6A
:10514000810080ED000A19E00C989DF81B10026B9D
:10515000C06F02EB810292ED000A9FED201A80EEF3
:10516000010A00EB810080ED000A07E00C98C16F96
:105170009DF81B20002041F82200FFE70C999DF8C4
:105180001B20886FC96F00EB421001EB820191ED8B
:10519000000A0DF00DFC0C98C06F9DF81B1000EB81
:1051A000810080ED000AFFE79DF81B0001308DF8BB
:1051B0001B007CE700208DF83700FFE79DF93700E2
:1051C0000EB080BD00007A449A99193FCDCC4C3F77
:1051D000AB611C3F0000000000C0DA4500A00C4697
:1051E00083B00290019100208DF80300FFE79DF845
:1051F0000300029991F91110884210DAFFE7029832
:10520000C06F9DF8032050F82200019941F8220058
:10521000FFE79DF8030001308DF80300E7E703B0D6
:105220007047000082B0019000910198007C0099C5
:105230000870019890ED080AC06890ED001A30EEF1
:10524000410A009880ED010A02B0704780B58AB02B
:1052500005AB03930346039808930791069280EDEC
:10526000000A089820B9FFE7FE208DF827001CE10E
:10527000079808998860089900200874069808998A
:10528000C860079890F84C00C00728B1FFE708985D
:10529000C06800F0DBFAFFE70898806800780146F4
:1052A0000291062832D80299DFE801F0040B1218A7
:1052B0001F2C250008990420487400208DF8130045
:1052C00024E008990420487401208DF813001DE0A3
:1052D0000899022048748DF8130017E008990420FB
:1052E000487403208DF8130010E0089904204874D6
:1052F0008DF813000AE008990120487405208DF804
:10530000130003E0FC208DF82700CEE0089890F908
:1053100011008000FEF774F8089948620898406A06
:1053200008B9FFE7A5E0089890F911008000FEF7A2
:1053300067F8089988620898806A08B9FFE798E0DA
:10534000089890F911008000FEF75AF80899086350
:105350000898006B08B9FFE78BE0089890F91100F6
:10536000C0EB00108000FEF74BF8089948630898DE
:10537000406B08B9FFE77CE0089890F911008000C5
:10538000FEF73EF80899C8670898C06F08B9FFE7AC
:105390006FE0089890F911004001FEF731F8089984
:1053A00048670898406F08B9FFE762E0089890F9ED
:1053B00011004001FEF724F8089988670898806F6B
:1053C00008B9FFE755E000208DF81200FFE79DF8CF
:1053D0001200089991F91110884233DAFFE7039A15
:1053E00008988168406B9DF81230C3EB031300EB03
:1053F000830092ED000A0A1D00210FF061F8039A64
:1054000008988168406F9DF8123000EB431092EDD0
:10541000000AD1ED110A0DF027FB039A0898816864
:10542000806F9DF8123000EB431092ED000AD1ED31
:10543000120A0DF019FBFFE79DF8120001308DF8FC
:105440001200C4E7039A089901F1380092ED000AAE
:10545000896801F12402002101910FF031F80898C8
:1054600012309DF813100EF089FC01988DF827007A
:105470001BE00898406AFDF7D7FD0898006BFDF720
:10548000D3FD0898406BFDF7CFFD0898C06FFDF77E
:10549000CBFD0898406FFDF7C7FD0898806FFDF7BA
:1054A000C3FDFE208DF82700FFE79DF927000AB015
:1054B00080BD000080B584B003900291019200206D
:1054C000009001980078012805D0FFE70020C4F281
:1054D000FA40009042E002980079012833D1FFE7BA
:1054E000029890ED000A9FED231AB4EE410AF1EE06
:1054F00010FA28DDFFE7029890ED000AB7EE001AD7
:10550000B4EE410AF1EE10FA05DDFFE70020CBF61C
:105510008070009016E0019890ED010A029890EDDD
:10552000001A9FED152A31EE021A9FED142A81EE22
:10553000021A9FED132A21EE021A30EE010A8DEDB8
:10554000000AFFE709E0019890ED010AD0ED020A98
:105550000FF088F98DED000AFFE7FFE79DED000AE7
:10556000039A516AD06F92F911200FF007F90020C9
:1055700004B080BD9A99993E9A9999BE3333333FCE
:105580000000C84280B586B004908DF80F100292DA
:10559000049820B9FFE7FE208DF8170066E09DF81B
:1055A0000F000499097C884204D1FFE700208DF8A0
:1055B00017005BE09DF80F0004281CD1FFE704985A
:1055C000007C042817D0FFE70298FAF735FEFAF7B7
:1055D00029FE00EBD07121F00101411A01200029C0
:1055E00018BF4FF0FF3000EE100AB8EEC00A049862
:1055F00080ED0B0AFFE700208DF80700FFE79DF81C
:105600000700049991F91110884227DAFFE70498FE
:10561000406B9DF80710C1EB011100EB81000FF00A
:105620001BF80498406F9DF8071000EB41109FEDA8
:10563000110A8DED000A0DF0B5FA9DED000A0498EF
:10564000806F9DF8071000EB41100DF0ABFAFFE7FB
:105650009DF8070001308DF80700D0E79DF80F0096
:105660000499087400208DF81700FFE79DF91700D2
:1056700006B080BD0000000084B002900191029845
:1056800020B9FFE7FE208DF80F0048E0019820B90F
:10569000FFE7FE208DF80F0041E00298806890F847
:1056A0004C00C00758B1FFE7019890ED111A9FED2B
:1056B0001E0A30EE410A029880ED080A04E00198C3
:1056C000406C02990862FFE700208DF80300FFE7B5
:1056D0009DF80300029991F9111088421BDAFFE747
:1056E00001989DF8032000EB021080680299496A36
:1056F00041F8220001989DF8032000EB0210C068D9
:105700000299896A41F82200FFE79DF80300013001
:105710008DF80300DCE700208DF80F00FFE79DF90E
:105720000F0004B0704700BFDB0FC94084B0039086
:105730008DED020ACDED010A039890ED000A9DED72
:10574000021A30EE010A8DED000A9DED010AB5EE58
:10575000400AF1EE10FA26DDFFE79DED000A9DED0F
:10576000011AB4EE410AF1EE10FA09DBFFE79DEDF4
:10577000011A9DED000A30EE410A8DED000A11E09C
:105780009DED000AB5EE400AF1EE10FA09DAFFE7E6
:105790009DED011A9DED000A30EE010A8DED000A23
:1057A000FFE7FFE7FFE700980399086004B0704740
:1057B00085B08DED040ACDED030A8DED021A9DED45
:1057C000040A9DED031A30EE410A8DED010A9DEDAC
:1057D000020AB5EE400AF1EE10FA32DDFFE79DED68
:1057E000020AB0EE001A80EE010A8DED000A9DED6E
:1057F000010A9DED001AB4EE410AF1EE10FA09DD3E
:10580000FFE79DED021A9DED010A30EE410A8DED94
:10581000010A15E09DED010A9DED001AB1EE411A55
:10582000B4EE410AF1EE10FA09DAFFE79DED021A33
:105830009DED010A30EE010A8DED010AFFE7FFE759
:10584000FFE79DED010A05B07047000081B00090B0
:10585000009890ED001A9FED040A30EE410A80EDA9
:10586000000A01B0704700BFDB0FC94083B002904F
:105870008DED010ACDED000A029890ED000A9DED34
:10588000001AB4EE410AF1EE10FA04DDFFE70098C9
:1058900002990860FFE7029890ED000A9DED011A59
:1058A000B4EE410AF1EE10FA04DAFFE7019802992A
:1058B0000860FFE703B0704780B5B4B03290319113
:1058C0003092329818B9FFE700203390FDE131980B
:1058D000013831900020ADF84E0040F2B840C2F2DD
:1058E0000000007801461291072800F2C881129941
:1058F000DFE811F008001A002C0097003601610162
:10590000A301B4013298319945F6EC72C0F6020257
:105910001CF0BCFE40F2B841C2F200010878013030
:10592000087001203390D0E13298319945F61A720F
:10593000C0F602021CF0AAFE40F2B841C2F2000119
:1059400008780130087001203390BEE142F674708F
:10595000C2F200001190C06818F086FE1198806BAA
:1059600014A90022052318F0EDFAC0B1FFE7329820
:10597000319945F6EC62C0F602021CF087FE40F257
:10598000B841C2F200010720087042F67470C2F2FA
:105990000000C06818F048FE0120339095E142F6FF
:1059A0007470C2F20000C06818F03EFE14A8FCF744
:1059B000F9FE90B1FFE73298319945F6C272C0F610
:1059C00002021CF063FE40F2B841C2F20001087806
:1059D000013008700120339077E140F2B940C2F203
:1059E0000000017801310170007802280FDCFFE728
:1059F0003298319945F63872C0F602021CF046FE24
:105A000040F2B841C2F200010120087006E040F205
:105A1000B841C2F2000107200870FFE7012033906F
:105A200053E13298319946F20D02C0F602021CF0A1
:105A30002DFE17A8109000F01BFF1098002129914F
:105A40002A912B9100F0D2FFFFE7BDF84E00B0F590
:105A50007A7F4BDAFFE742F67470C2F20000806B87
:105A600014A90F910022052318F06CFA01460F9833
:105A7000B1FA81F149098DF84D10FCF793FE8DF8CC
:105A80004C009DF84D00C00778B3FFE79DF84C002F
:105A9000C00750B3FFE79DED141A40F2BC40C2F2BC
:105AA000000090ED000A30EE010A80ED000A9DED45
:105AB000151A40F2C040C2F2000090ED000A30EE2C
:105AC000010A80ED000A9DED161A40F2C440C2F2B0
:105AD000000090ED000A30EE010A80ED000ABDF8EA
:105AE0004E000130ADF84E00FFE7AEE7BDF84E00C6
:105AF00000EE100AB8EE401A40F2BC40C2F20000BC
:105B000090ED000A80EE010A80ED000ABDF84E001B
:105B100000EE100AB8EE401A40F2C040C2F2000097
:105B200090ED000A80EE010A80ED000ABDF84E00FB
:105B300000EE100AB8EE401A40F2C440C2F2000073
:105B400090ED000A80EE010A80ED000A40F2B841B3
:105B5000C2F2000108780130087001203390B4E0EF
:105B60003298319945F69472C0F602021CF08EFD0F
:105B700017A80E9000F07CFE0E9840F2BC41C2F2D5
:105B800000010968299140F2C041C2F20001096890
:105B90002A9140F2C441C2F2000109682B9100F041
:105BA00025FF40F2B841C2F20001087801300870C8
:105BB0000120339089E032980C9031980D9040F29A
:105BC000BC40C2F200000068FAF71AFD41EC100B6D
:105BD0008DED0A0B40F2C040C2F200000068FAF7F7
:105BE0000FFD41EC100B8DED080B40F2C440C2F2EA
:105BF00000000068FAF704FD9DED081B9DED0A0BFF
:105C000002460C980B460D9943EC122B6A4682ED26
:105C1000042B82ED021B82ED000B46F25002C0F60F
:105C200002021CF033FD40F2B841C2F200010878D4
:105C3000013008700120339047E03298319945F6E1
:105C40008172C0F602021CF021FD40F2B841C2F29E
:105C50000001082008700120339036E03298319915
:105C600045F60572C0F602021CF010FD40F2B84184
:105C7000C2F20001082008700120339025E040F2B4
:105C8000BC41C2F2000100200790086040F2C04110
:105C9000C2F20001086040F2C441C2F20001086093
:105CA00040F2B941C2F2000108703298319946F2CF
:105CB0002012C0F602021CF0E9FC079840F2B8413D
:105CC000C2F2000108703390FFE7339834B080BD12
:105CD00080B5B0B02E902D912C922E9818B9FFE778
:105CE00000202F9060E22D9801382D902C980121F2
:105CF0002BAA01F081FC28902C9802212AAA01F0FD
:105D00007BFC27902C98032129AA01F075FC269092
:105D100028982B9A45F62301C0F60201FAF7E2FA19
:105D2000A0B9FFE72E982D9946F26C22C0F6020228
:105D300045F6F323C0F602031CF0A8FC40F2C8416C
:105D4000C2F20001002008702F902DE228982B9AB3
:105D500046F28A21C0F60201FAF7C4FA00285BD1A4
:105D6000FFE7279818B9FFE7269808B1FFE70BE28D
:105D700040F2C840C2F20000007801460A9120B10A
:105D8000FFE70A98012810D045E02E982D9946F299
:105D90009F12C0F602021CF079FC40F2C841C2F228
:105DA0000001012008702F90FEE10DA809906421E8
:105DB000FAF763FA45F6D300C0F60200089000F047
:105DC0009DFD189045F6E200C0F60200069000F036
:105DD000D7FD069A014609981791142107911CF0E6
:105DE00055FC0799089A099814301CF04FFC099843
:105DF00000F0FCFD2E982D9946F25B12C0F60202CF
:105E00001CF044FC40F2C841C2F2000102200870BC
:105E100001202F90C8E19DE128982B9A46F29B2102
:105E2000C0F60201FAF75EFA002840F0CF80FFE7E3
:105E3000279818B1FFE7269808B1FFE7A4E1279853
:105E40002A9A46F29521C0F60201FAF74BFA002889
:105E500057D1FFE700F088FD0C9040F2C840C2F235
:105E6000000000780146059120B1FFE70598012860
:105E700010D045E02E982D9946F20A22C0F6020273
:105E80001CF004FC40F2C841C2F20001012008707D
:105E90002F9089E10C9840F2C941C2F200010978C3
:105EA00050F83100E0B1FFE72E982D990C9A40F29E
:105EB000C943C2F2000304931B7852F8333046F210
:105EC0006822C0F602021CF0E1FB04990878013058
:105ED000087040F2C841C2F20001012008700CE0D5
:105EE00040F2C941C2F200010020087040F2C841EE
:105EF000C2F2000102200870FFE701202F9053E159
:105F000063E027982A9A46F28F21C0F60201FAF739
:105F1000E9F9002857D1FFE700F02CFD0B9040F283
:105F2000C840C2F2000000780146039120B1FFE7AB
:105F30000398012810D045E02E982D9946F2212291
:105F4000C0F602021CF0A2FB40F2C841C2F20001FE
:105F5000012008702F9027E10B9840F2C941C2F24E
:105F60000001097850F83100E0B1FFE72E982D9933
:105F70000B9A40F2C943C2F2000302931B7852F815
:105F8000333046F26822C0F602021CF07FFB029911
:105F900008780130087040F2C841C2F200010120C7
:105FA00008700CE040F2C941C2F200010020087004
:105FB00040F2C841C2F2000102200870FFE7012050
:105FC0002F90F1E000E0DFE0FFE7C2E028982B9A95
:105FD00046F27521C0F60201FAF784F9002840F074
:105FE000B780FFE7279818B1FFE7269808B9FFE7C1
:105FF000CAE027982A9A46F28F21C0F60201FAF7E2
:1060000071F900283ED1FFE740F2C840C2F200001B
:106010000078B0BBFFE70DA800F02AFC269800F03E
:10602000AFFC88B9FFE72E982D9946F26312C0F6AF
:1060300002021CF02BFB40F2C841C2F20001022018
:10604000087001202F90AFE02E982D9946F2231270
:10605000C0F602021CF01AFB269B46F26C22C0F628
:1060600002020DA8019014211CF010FB019800F011
:10607000BDFC40F2C841C2F20001012008702F901F
:1060800092E04BE027982A9A46F29521C0F6020149
:10609000FAF728F900283FD1FFE740F2C840C2F2E2
:1060A00000000078B8BBFFE70DA800F0E1FB2698E0
:1060B00000F024FC88B9FFE72E982D9946F2F212E1
:1060C000C0F602021CF0E2FA40F2C841C2F200013E
:1060D0000220087001202F9066E02E982D9946F23C
:1060E0002312C0F602021CF0D1FA0DA80090143061
:1060F000269B46F26C22C0F6020214211CF0C6FA5E
:10610000009800F073FC40F2C841C2F20001012087
:1061100008702F9048E000E036E0FFE740F2C8400A
:10612000C2F200000078012811D1FFE72E982D99C6
:1061300046F2C512C0F602021CF0A8FA40F2C841AD
:10614000C2F200010220087001202F902CE0FFE72E
:10615000FFE7FFE7FFE740F2C840C2F20000007827
:10616000022810D1FFE72E982D9945F61E02C0F6A1
:1061700002021CF08BFA40F2C841C2F2000100207A
:1061800008702F9010E0FFE72E982D9945F68D624C
:10619000C0F602021CF07AFA40F2C841C2F20001D5
:1061A000002008702F90FFE72F9830B080BD0000CE
:1061B00080B588B0069005910492069818B9FFE75B
:1061C000002007908DE005980138059042F21120DB
:1061D000ADF80E00BDF80E00ADF80C009DF80E00F5
:1061E0009DF80F1040EA0120ADF80A0040F2CA40C5
:1061F000C2F20000007801460191032861D801999C
:10620000DFE801F00214283C0698059946F20D12C9
:10621000C0F602021CF03AFA40F2CA41C2F2000192
:10622000087801300870012007905AE00698059917
:10623000BDF80C3046F2E002C0F602021CF026FA6D
:1062400040F2CA41C2F20001087801300870012012
:10625000079046E006980599BDF80A3046F2B30269
:10626000C0F602021CF012FA40F2CA41C2F200016A
:106270000878013008700120079032E0BDF80C006A
:10628000BDF80A10884209D1FFE70698059946F241
:106290009B02C0F602021CF0F9F908E00698059985
:1062A00046F28E02C0F602021CF0F0F9FFE740F25F
:1062B000CA41C2F20001087801300870012007903D
:1062C0000FE00698059946F22012C0F602021CF073
:1062D000DDF940F2CA41C2F20001002008700790C7
:1062E000FFE7079808B080BD80B5DAB058905791A5
:1062F0005692589818B9FFE700205990C9E057986E
:106300000138579040F2CB40C2F2000000780146BD
:106310000991042800F2AD800999DFE801F0032417
:10632000778899000AA800F0A3FA58980790579820
:1063300008902298FAF764F9024607980B460899E4
:1063400043EC102B6A4682ED000B46F27E02C0F64B
:1063500002021CF09BF940F2CB41C2F20001012085
:106360000870599095E042F67470C2F200000690F1
:10637000C06818F079F90698406F23A900220A2313
:1063800017F0E0FD80B1FFE742F67470C2F2000042
:10639000C06818F049F940F2CB41C2F20001032075
:1063A00008700120599074E00AA8039000F060FA88
:1063B00042F67470C2F20000C06818F035F9039814
:1063C0003899229100F012FB039800F051FA589886
:1063D0000490579805902298FAF712F9024604980B
:1063E0000B46059943EC102B6A4682ED000B46F2F2
:1063F0004E12C0F602021CF049F940F2CB41C2F243
:106400000001022008700120599042E058985799E5
:1064100046F2C512C0F602021CF038F940F2CB4138
:10642000C2F20001052008700120599031E058980F
:10643000579945F6BD62C0F602021CF027F940F2FA
:10644000CB41C2F20001052008700120599020E0E4
:106450005898579946F27B12C0F602021CF016F9C2
:1064600040F2CB41C2F20001052008700120599092
:106470000FE05898579946F22012C0F602021CF01D
:1064800005F940F2CB41C2F200010020087059909A
:10649000FFE759985AB080BD80B5E2B060905F9137
:1064A0005E92609818B9FFE700206190C2E05F98A3
:1064B00001385F9040F2CC40C2F200000078014603
:1064C000119148B1FFE71198012817D0FFE7119803
:1064D000022800F08E809DE060985F9946F22702C6
:1064E000C0F602021CF0D2F840F2CC41C2F2000128
:1064F000087801300870012061909BE012A800F03C
:10650000B7F942F67470C2F200001090C06818F03B
:10651000ABF81098406F2BA90022052317F012FD4D
:10652000C0B1FFE760985F9945F6D162C0F60202FC
:106530001CF0ACF840F2CC41C2F20001022008701D
:1065400042F67470C2F20000C06818F06DF80120C5
:1065500061906FE042F67470C2F20000C06818F0FB
:1065600063F83C9827904098289012A800F03EFAD3
:1065700060980E905F980F90279828990691299916
:106580000891FAF73DF80246069807920A460799DD
:1065900042EC101B8DED0C0BFAF732F8024608980E
:1065A00009920A46099942EC101B8DED0A0BFAF785
:1065B00027F89DED0A1B9DED0C0B02460E980B462D
:1065C0000F9943EC122B6A4682ED042B82ED021BDD
:1065D00082ED000B46F22E12C0F602021CF056F8B5
:1065E00040F2CC41C2F2000103200870012061900A
:1065F00020E060985F9945F60572C0F602021CF033
:1066000045F840F2CC41C2F200010320087001209D
:1066100061900FE060985F9946F22012C0F6020286
:106620001CF034F840F2CC41C2F2000100200870A6
:106630006190FFE7619862B080BD000080B596B0C0
:10664000149013911292149818B9FFE70020159036
:106650000AE113980138139040F2CD40C2F20000D5
:10666000007801460A91092800F2EE800A99DFE8D5
:1066700001F00517243643557385BCCE1498139A40
:1066800045F6F031C0F60201F9F702FE40F2CD41C5
:10669000C2F2000108780130087001201590E3E093
:1066A00014981AF0B5F840F2CD41C2F20001087812
:1066B0000130087001201590D6E01498139A45F621
:1066C0007F51C0F60201F9F7E3FD40F2CD41C2F27D
:1066D000000108780130087001201590C4E014987A
:1066E0001AF004F840F2CD41C2F2000108780130FE
:1066F000087001201590B7E01498139A45F67F4171
:10670000C0F60201F9F7C4FD40F2CD41C2F200012A
:1067100008780130087001201590A5E00BA819F049
:1067200001FD149813990B9AC2F5C04C6B46C3F83F
:1067300004C01A6046F26A02C0F602024FF4C04377
:106740001BF0A4FF40F2CD41C2F2000108780130F5
:1067500008700120159087E01498139A45F60051AF
:10676000C0F60201F9F794FD40F2CD41C2F20001FA
:106770000878013008700120159075E01498089091
:106780001398099042F67470C2F20000D0F8B0106D
:106790000491D0F8B800F9F733FF02460498059247
:1067A0000A46059942EC101B8DED060BF9F728FF00
:1067B0009DED060B024608980B46099943EC112BF8
:1067C0006A4682ED021B82ED000B46F27602C0F6AD
:1067D00002021BF05BFF40F2CD41C2F200010878DB
:1067E00001300870012015903EE01498139A45F688
:1067F0000C61C0F60201F9F74BFD40F2CD41C2F247
:106800000001087801300870012015902CE01498E0
:10681000139942F67472C2F2000202F1D003EC4600
:10682000CCF8003002F1BC0346F2AA02C0F6020224
:106830001BF02CFF40F2CD41C2F20001087801307C
:106840000870012015900FE01498139946F2201259
:10685000C0F602021BF01AFF40F2CD41C2F2000165
:10686000002008701590FFE7159816B080BD000055
:1068700080B582B0019001990020C0F60E0064221C
:10688000FCF79EFB0198143000F038F80199C862BB
:10689000019800F075F8019988620198806A38B90A
:1068A000FFE7019940F28810C2F200008862FFE71A
:1068B0000198C06A38B9FFE7019944F6A850C0F6BC
:1068C0000200C862FFE70198806A013038B9FFE72B
:1068D000019940F28810C2F200008862FFE7019837
:1068E000C06A013038B9FFE7019944F6A850C0F6F4
:1068F0000200C862FFE702B080BD000080B584B02E
:106900000290029818B9FFE70020039029E00020C8
:106910000190FFE7019945F20C30C0F6020050F8F3
:106920003100D8B1FFE7019945F20C30C0F6020002
:1069300050F831000299F9F7BEFC50B9FFE7019910
:1069400045F20C30C0F6020000EBC1004068039035
:1069500007E0FFE7019801300190DBE7002003909A
:10696000FFE7039804B080BD45F20C30C0F602008A
:106970007047000045F22430C0F602007047000066
:1069800080B584B00290029818B9FFE70020039008
:1069900029E000200190FFE7019945F22430C0F67C
:1069A000020050F83100D8B1FFE7019945F22430D8
:1069B000C0F6020050F831000299F9F77CFC50B99A
:1069C000FFE7019945F22430C0F6020000EBC10058
:1069D0004068039007E0FFE7019801300190DBE792
:1069E00000200390FFE7039804B080BD80B582B01B
:1069F000019017F019FA0B20FCF7BEFA019900205C
:106A0000C0F60E006422FCF7E7FA17F063FA02B052
:106A100080BD000080B541F60830C2F2000003F0EE
:106A200049FC80BD80B541F62810C2F2000003F099
:106A300041FC80BD80B541F6C800C2F2000003F001
:106A400039FC80BD80B541F66830C2F2000003F029
:106A500031FC80BD80B541F68810C2F2000003F021
:106A600029FC80BD80B541F6E810C2F2000003F0B9
:106A700021FC80BD80B541F64820C2F2000003F041
:106A800019FC80BD80B541F6C830C2F2000003F0A9
:106A900011FC80BD80B541F6A820C2F2000003F0D1
:106AA00009FC80BD82B001900198007810384AF648
:106AB000AB21CAF6AA21A0FB0110000900900099A1
:106AC00044F6A830C0F60200405C0199C865009801
:106AD000042807D3FFE701990868042262F309003C
:106AE000886506E00199086840F2FF3290438865A6
:106AF000FFE70198806D02B07047000086B00590F6
:106B000000208DF813000598806A0390059880692D
:106B100010BBFFE70398029003281BD80299DFE817
:106B200001F0020D0218059890F82F00C00720B15F
:106B3000FFE701208DF81300FFE70CE00598C06A1D
:106B4000B0F1C07F04D1FFE701208DF81300FFE70B
:106B500001E000E0FFE745E005988069B0F5005FDF
:106B600025D1FFE70398019003281ED80199DFE89B
:106B700001F00206021101208DF8130016E00598BD
:106B800090F82F00C00720B1FFE701208DF8130017
:106B9000FFE70BE00598C06AB0F1C07F04D1FFE7C2
:106BA00001208DF81300FFE700E0FFE719E00398EC
:106BB0000090032804D3FFE70098032804D00EE0D8
:106BC00001208DF813000BE0059890F82F00C00706
:106BD00020B1FFE701208DF81300FFE700E0FFE799
:106BE000FFE7FFE79DF8130006B0704784B00390FD
:106BF00002910192009303980168086820F48020B4
:106C000008600098039909684860039880684028E4
:106C100009D1FFE7019803990968886002980399F0
:106C20000968C86008E002980399096888600198BB
:106C300003990968C860FFE704B0704782B000900C
:106C4000009820B9FFE701208DF8070074E0009854
:106C500000886FF3DF20B0F5B67F09D3FFE7009817
:106C600000886FF3DF2040F29561884204D3FFE78C
:106C700001208DF807005FE000980068C0F3CA208B
:106C8000B0F5B67F09D3FFE700980068C0F3CA20CB
:106C900040F29561884204D3FFE701208DF8070098
:106CA0004AE0009881880068800D40EA81206FF3F7
:106CB000DF20B0F5B67F0DD3FFE70098818800682C
:106CC000800D40EA81206FF3DF2040F29561884219
:106CD00004D3FFE701208DF807002DE0009880889D
:106CE000C0F34A00B0F5B67F09D3FFE7009880886B
:106CF000C0F34A0040F29561884204D3FFE70120C7
:106D00008DF8070018E0009881880020B0EB913FD3
:106D100004D1FFE701208DF807000DE0009880887E
:106D2000000B800720B9FFE701208DF8070003E082
:106D300000208DF80700FFE79DF8070002B07047BC
:106D400080B584B002900191029820B9FFE7FE203F
:106D50008DF80F000EE0019820B9FFE7FE208DF8B6
:106D60000F0007E001982421F9F787FA00208DF839
:106D70000F00FFE79DF90F0004B080BD80B584B01F
:106D80000290029820B9FFE7FE208DF80F002BE05B
:106D900042F20E50C2F200000078C00720B1FFE7B7
:106DA000FD208DF80F001FE017F06EFB43F2381145
:106DB000C2F20001086020B9FFE7FE208DF80F0045
:106DC00012E046F65572C0F6000200200190032141
:106DD000FCF794FC019842F20E52C2F2000201212B
:106DE00011708DF80F00FFE79DF90F0004B080BD12
:106DF00080B584B002900191029820B9FFE7FE208F
:106E00008DF80F009FE00298FFF718FF20B1FFE711
:106E1000FF208DF80F0096E001982421F9F72DFA54
:106E2000FFE70020C4F2A5400090029800886FF3AD
:106E3000DF2000EE100AB8EE400A9FED451A30EE52
:106E4000410A30EE000A9DED002A80EE020A019808
:106E500080ED020A02980068C0F3CA2000EE100A12
:106E6000B8EE400A30EE410A30EE000A9DED002AED
:106E700080EE020A019880ED030A0298818800687A
:106E8000800D40EA81206FF3DF2000EE100AB8EE9B
:106E9000400A30EE410A30EE000A9DED002A80EEF5
:106EA000020A019880ED000A02988088C0F34A0027
:106EB00000EE100AB8EE400A30EE410A30EE000A49
:106EC0009DED002A80EE020A019880ED010A0298E9
:106ED0008088800B0199487502988088C0F3013042
:106EE000019908750298C0880199C88202980089A2
:106EF0000199088302984089019948830298007B90
:106F0000002818BF0120019908770298407B0028CB
:106F100018BF0120019948770298C0890199C88358
:106F20000298008A00EE100AB8EE400A30EE410ADC
:106F30009DED001A80EE010A019880ED040A002000
:106F40008DF80F00FFE79DF90F0004B080BD00BF72
:106F50000000804480B543F23810C2F2000000689F
:106F6000802117F0B1F980BD80B582B0009000207B
:106F7000FCF764FB009912220BF0FAFA20B9FFE744
:106F800000208DF8070003E0FF208DF80700FFE7E1
:106F90009DF9070002B080BD80B582B00190019AD2
:106FA0008020012117F0E2F98038B0FA80F0400922
:106FB00002B080BD7047000080B5012003F0D8FF0B
:106FC00080BD000080B5082003F0D2FF80BD000026
:106FD00080B5102003F0CCFF80BD000080B52020DC
:106FE00003F0C6FF80BD0000FFE700BFFDE7000023
:106FF00080B584B003908DF80B10002001900398A9
:1070000060B3FFE70398012828D0FFE70398022820
:1070100024D0FFE70398032820D0FFE70398042833
:107020001CD0FFE70398052818D0FFE7039806282F
:1070300014D0FFE70398072810D0FFE7039808282B
:107040000CD0FFE70398092808D0FFE703980A2827
:1070500004D0FFE703980B2801D1FFE708E045F2D1
:107060002D40C0F6020040F2DB3116F031FDFFE7A3
:107070009DF80B0078B1FFE79DF80B0001280AD0BE
:10708000FFE79DF80B00022805D0FFE79DF80B00F5
:10709000032801D1FFE708E045F22D40C0F60200C9
:1070A0004FF4777116F014FDFFE79DF80B0018B947
:1070B000FFE70020019017E09DF80B00012804D1A4
:1070C000FFE74FF4807001900DE09DF80B0002285F
:1070D00004D1FFE74FF40070019003E04FF44070DB
:1070E0000190FFE7FFE7FFE743F61041C4F202011A
:1070F000086820F440700860019A0868104308602E
:10710000086820F0F8000860039A086840EAC200A6
:1071100040F002000860086840F48030086004B065
:1071200080BD000043F60040C4F202000068800504
:1071300000281FD5FFE743F60041C4F202010868AA
:1071400020F400700860FFE743F60041C4F202013A
:10715000086840F400600860086820F40060086077
:10716000FFE743F60041C4F20201086840F40070F2
:107170000860FFE743F60040C4F2020000684005E3
:1071800000281FD5FFE743F60041C4F2020108685A
:1071900020F480600860FFE743F60041C4F202017A
:1071A000086840F480500860086820F48050086047
:1071B000FFE743F60041C4F20201086840F4806032
:1071C0000860FFE77047000080B582B08DF80700C7
:1071D00000919DF8070078B1FFE79DF807000128AE
:1071E0000AD0FFE79DF80700022805D0FFE79DF8C9
:1071F0000700032801D1FFE708E045F22D40C0F663
:1072000002004FF46F7116F063FCFFE7009801284D
:1072100001D1FFE708E045F22D40C0F6020040F240
:10722000BD3116F055FCFFE743F61041C4F20201F0
:10723000086820F440700860086840F004000860A6
:107240009DF80720086840EA022040F4803008607A
:1072500002B080BD80B582B001908DF80310019816
:10726000B0F1006F05D3FFE70198B0F1016F10D3C3
:10727000FFE7019847F60001C1F6FF71884209D384
:10728000FFE7019847F60F21C1F6FF71884201D848
:10729000FFE708E045F2F330C0F6020040F2BB2100
:1072A00016F016FCFFE743F61041C4F2020108682D
:1072B00020F44070086008680860086840F0010029
:1072C00008609DF803000199087002B080BD0000BD
:1072D00080B584B00390019300920398B0F1006FE1
:1072E00005D3FFE70398B0F1016F10D3FFE70398D0
:1072F00047F60001C1F6FF71884209D3FFE7039802
:1073000047F60F21C1F6FF71884201D8FFE708E078
:1073100045F2F330C0F6020040F2672116F0D8FBC8
:10732000FFE743F61041C4F20201086820F4407000
:107330000860086840F440700860086840F0010088
:107340000860009803990860BFF36F8F0198039954
:10735000486004B080BD000080B582B00190ADF8F7
:1073600002100198B0F1006F05D3FFE70198B0F16A
:10737000016F10D3FFE7019847F60001C1F6FF71D6
:10738000884209D3FFE7019847F60F21C1F6FF7144
:10739000884201D8FFE708E045F2F330C0F602006A
:1073A00040F2A22116F094FBFFE743F61041C4F22D
:1073B0000201086820F440700860086840F480709A
:1073C0000860086840F001000860BDF802000199FB
:1073D000088002B080BD000080B582B001900091AD
:1073E0000198B0F1006F05D3FFE70198B0F1016F8C
:1073F00010D3FFE7019847F60001C1F6FF718842FC
:1074000009D3FFE7019847F60F21C1F6FF718842C3
:1074100001D8FFE708E045F2F330C0F6020040F281
:10742000892116F055FBFFE743F61041C4F2020133
:10743000086820F440700860086840F40070086034
:10744000086840F00100086000980199086002B0E7
:1074500080BD000043F60C40C4F202000068C00684
:1074600000280FD5FFE742F22851C2F20001C86997
:1074700040F01000C86143F60C41C4F20201102034
:107480000860FFE743F60C40C4F202000068800683
:1074900000280FD5FFE742F22851C2F20001C86967
:1074A00040F00800C86143F60C41C4F202012020FC
:1074B0000860FFE743F60C40C4F202000068400693
:1074C00000280FD5FFE742F22851C2F20001C86937
:1074D00040F00400C86143F60C41C4F202014020B0
:1074E0000860FFE743F60C40C4F2020000680006A3
:1074F00000280FD5FFE742F22851C2F20001C86907
:1075000040F00200C86143F60C41C4F20201802041
:107510000860FFE743F60C40C4F2020000688007F1
:1075200000280FD5FFE742F22851C2F20001C869D6
:1075300040F02000C86143F60C41C4F20201022071
:107540000860FFE77047000080B584B0029000201B
:10755000019042F22851C2F20001C86104F01AF908
:107560000190FFE743F60C40C4F202000068C0033C
:10757000002815D5FFE70298013080B1FFE7029897
:1075800040B1FFE704F006F90199401A02998842D8
:1075900004D9FFE703208DF80F0023E0FFE7E1E7C0
:1075A00043F60C40C4F202000068C00738B1FFE7A0
:1075B00043F60C41C4F2020101200860FFE743F6E4
:1075C0000C40C4F20200006810F0F20F06D0FFE792
:1075D000FFF740FF01208DF80F0003E000208DF839
:1075E0000F00FFE79DF80F0004B080BD40F62D307E
:1075F000C2F200007047000088B007900691059223
:1076000000200490039005990860FFE7049806990C
:10761000884260D2FFE7FFE70798017800200290D8
:1076200039B1FFE707980078203818BF0120029091
:10763000FFE70298C00720B1FFE7079801300790E5
:10764000EAE7FFE7079801780020019041B1FFE7E2
:10765000079800782038B0FA80F040090190FFE7E1
:107660000198C00720B1FFE7079801300790E9E7CC
:107670000798007868B3FFE70498013004900498F5
:107680000699884224D1FFE707980390FFE70798FF
:1076900001780020009039B1FFE707980078203882
:1076A00018BF01200090FFE70098C00740B1FFE736
:1076B0000599086801300860079801300790E6E7EF
:1076C0000598006818B9FFE700200390FFE702E083
:1076D00000E000E09AE7039808B0704780B586B0F4
:1076E0000590049103920120029040F2D040C2F232
:1076F00000000068002859D1FFE740F2D041C2F2F3
:10770000000140F24840C2F200000860FFE740F28A
:10771000D040C2F200000068002846D0FFE740F2E7
:10772000D040C2F200000068006800680190019833
:10773000F8F7BAFD009005980099405C202805D024
:10774000FFE705980099405C30BBFFE70598019979
:10775000009AF8F7C7FDF0B9FFE740F2D040C2F257
:1077600000000068006890F90C00002812D4FFE7C0
:10777000059817F0E1FA40F2D041C2F20001096821
:10778000096891F90C10884203D0FFE700200290AD
:10779000FFE7FFE709E0FFE7FFE740F2D041C2F271
:1077A0000001086840680860B1E7FFE740F2D04098
:1077B000C2F20000006890B1FFE7029878B9FFE7D5
:1077C0000498039A45F24B71C0F60201F8F760FD88
:1077D00040F2D041C2F200010020086029E040F2EE
:1077E000D040C2F200000068B8B1FFE740F2D040DC
:1077F000C2F2000000680068836804980399059A43
:1078000098470290029838B9FFE740F2D041C2F29F
:10781000000100200860FFE70AE00498039A45F29F
:10782000A371C0F60201F8F733FD00200290FFE7D4
:10783000FFE7029806B080BD80B586B003900020B7
:107840000190039858B9FFE74FF0500080F311887A
:10785000BFF36F8FBFF34F8F0490FFE7FEE7082061
:1078600018F0D4F80290029858B9FFE74FF0500092
:1078700080F31188BFF36F8FBFF34F8F0590FFE741
:10788000FEE70298B0B1FFE718F092FB0398029967
:107890000860029900204860029840F22401C2F278
:1078A00000010A6850600298086018F0ADFB0120E2
:1078B0000190FFE7019806B080BD000080B584B05C
:1078C00047F61020C1F6FF700068039047F61420B9
:1078D000C1F6FF700068029047F61820C1F6FF70ED
:1078E000006801900199039808440390039888B1B7
:1078F000FFE7039840F26811C2F2000100910231E3
:1079000008220AF0DDFF00990298123104220AF0E1
:10791000D7FFFFE704B080BD80B58EB006AB0493FF
:107920000C900B910A920C9820B9FFE7FF208DF87C
:10793000370089E10B9820B9FFE7FF208DF8370069
:1079400082E10A990C980268891A00EE101AB8EEC2
:10795000400A9FEDBF1A80EE010A80ED010A0A98E5
:107960000C9908600C980B99097800F037FA0B987D
:1079700090ED020AB1EE400A80ED020A0B9890EDFC
:10798000010AB1EE400A80ED010A0C9810300B9903
:1079900091ED010ADFEDAF0ACDED030AFDF7C6FE5A
:1079A0009DED031A0C9890ED052A90ED430A90ED99
:1079B0005E3A33EE022A72EE430AFDF7F9FE9DEDC0
:1079C000031A049880ED030A0C9890ED052A90EDB7
:1079D000440A90ED5E3A33EE022A72EE430AFDF756
:1079E000E7FE049981ED020A0B98083091ED020A36
:1079F000D1ED030AFDF73AFF0B9890ED021A0C98AF
:107A000090ED050A30EE010A80ED050A0C9890ED24
:107A1000040A9FED911AB4EE410AF1EE10FA12DD5C
:107A2000FFE70C9890ED040AB1EE081AB4EE410A93
:107A3000F1EE10FA07DAFFE70C994CF6CD40C4F2EC
:107A4000BC0008611BE00C9890ED040A9FED831ABE
:107A5000B4EE410AF1EE10FA10DDFFE70C9890ED5C
:107A6000040AB7EE081AB4EE410AF1EE10FA05DA8C
:107A7000FFE70C994FF07F500861FFE7FFE70B9895
:107A80000430F9F797FA0C98007B0146029140B157
:107A9000FFE7029801281DD0FFE7029802285CD07A
:107AA00074E000208DF81700FFE79DF8170001280B
:107AB0000FDCFFE70C989DF8171000EB8101002008
:107AC000C1F85401FFE79DF8170001308DF8170049
:107AD000EBE75BE00C9901F15800D1ED011A91ED53
:107AE000040AD1ED5D0A9FED5E1A8DED011A0CF0CE
:107AF0006FFB049A9DED011A82ED010A0C9901F1C8
:107B00001C0092ED010AD1ED011AF0EE410A0CF0D1
:107B10005FFB9DED011A0C9880ED550A0C9901F15F
:107B2000D000D1ED011A91ED050AD1ED5E0A0CF0FD
:107B30004FFB049A9DED011A82ED000A0C9901F1A8
:107B4000940092ED000AD1ED011AF0EE410A0CF01A
:107B50003FFB0C9880ED560A18E000208DF81600C7
:107B6000FFE79DF8160001280FDCFFE70C989DF851
:107B7000161000EB81010020C1F85401FFE79DF8C9
:107B8000160001308DF81600EBE7FFE700208DF8B6
:107B90001500FFE79DF8150001281BDCFFE70C9995
:107BA0009DF8152001EB421000F58A7001EB82016F
:107BB00091ED550A0AF0FCFE0C989DF8151000EBAB
:107BC000810080ED550AFFE79DF8150001308DF822
:107BD0001500DFE70C98806890F88C00C00740B172
:107BE000FFE70C9890ED550AB1EE400A80ED550A7A
:107BF000FFE70C98806890F88D00C00740B1FFE760
:107C00000C9890ED560AB1EE400A80ED560AFFE757
:107C10000C9890ED550AB5EE400AF1EE10FA02DA32
:107C2000FFE700BFFFE70C9890ED560AB6EE001A8A
:107C3000B4EE410AF1EE10FA02DDFFE700BFFFE704
:107C400000208DF83700FFE79DF937000EB080BDAA
:107C500000007A44DB0FC940CDCCBC403333B33F86
:107C60000000000082B0019000910198D0F854010A
:107C7000009908600198D0F858010099486002B056
:107C80007047000082B0019000910198007B00993C
:107C9000087002B07047000080B58AB005AA039250
:107CA000024603980892079180ED010AC0ED000A90
:107CB000089820B9FFE7FF208DF8270076E00798A5
:107CC000089988600899002008730898806890F8DF
:107CD0008D00C00720B1FFE706A8FDF7B7FDFFE75D
:107CE000039890ED010A089880ED430A089880ED0A
:107CF000440A089901F58870896891ED220AB1EE6D
:107D0000400ADFED2C0AFDF711FD039A089901F1F5
:107D1000580092ED000A896801F1200200210291C9
:107D20000CF0CEFB039A089901F11C0092ED000AB9
:107D30008A68012101910CF0C3FB039B0299089A08
:107D400002F1D00093ED000A926860320CF0B8FBAB
:107D5000039B0199089A02F1940093ED000A92683E
:107D600040320CF0ADFB02988DF81300FFE79DF850
:107D70001300012816DCFFE7039A08999DF8130009
:107D800001EB401000F58A7092ED000A8968D1ED90
:107D9000200A0AF069FEFFE79DF8130001308DF814
:107DA0001300E4E700208DF82700FFE79DF9270086
:107DB0000AB080BDDB0FC94082B0019000910099EC
:107DC000019BD3F87401D3F87821D3F87C318B6010
:107DD0004A600860002002B07047000080B584B09F
:107DE00002908DF80710029820B9FFE7FF208DF868
:107DF0000F006DE09DF807000299097B884204D1CD
:107E0000FFE700208DF80F0062E000208DF80600EB
:107E1000FFE79DF80600032811DCFFE702989DF8B4
:107E20000610C1EB011100EB81001C300CF014FCBA
:107E3000FFE79DF8060001308DF80600E9E7002015
:107E40008DF80500FFE79DF80500012812DCFFE72B
:107E500002989DF8051000EB411000F58A709FED27
:107E60001E0A0AF09FFEFFE79DF8050001308DF81D
:107E70000500E8E702981030F9F79CF80298007BBB
:107E8000F0B9FFE79DF8070001280DD1FFE702993F
:107E90004CF6CD40C4F26C00086102994CF6CD401E
:107EA000C4F20C0048610AE09DF80700022805D1E1
:107EB000FFE70299D1F874010861FFE7FFE7FFE7E8
:107EC0009DF807000299087300208DF80F00FFE766
:107ED0009DF90F0004B080BD0000000080B584B0A3
:107EE00002900191029820B9FFE7FF208DF80F0062
:107EF0002EE0019820B9FFE7FF208DF80F0027E062
:107F00000198406C0299C1F874010198406D029982
:107F1000C1F878010298806890F88C00C00730B1F1
:107F2000FFE7029800F5BA70FDF790FCFFE70298B2
:107F3000806890F88D00C00730B1FFE7029800F527
:107F4000BC70FDF783FCFFE700208DF80F00FFE712
:107F50009DF90F0004B080BD80B586B004900391F8
:107F60000020029003980068122801D8FFE708E07B
:107F700045F21650C0F6020040F2896115F0A8FDE6
:107F8000FFE70398406830B1FFE703984068102886
:107F900001D8FFE708E045F21650C0F6020040F2B3
:107FA0008A6115F095FDFFE70398806818B3FFE735
:107FB0000398806801281ED0FFE703988068022894
:107FC00019D0FFE703988068032814D0FFE70398CF
:107FD000806804280FD0FFE70398806805280AD03E
:107FE000FFE703988068062805D0FFE703988068BC
:107FF000072801D1FFE708E045F21650C0F602005D
:1080000040F28B6115F064FDFFE7FFE7049890F8FC
:108010003C00012804D1FFE702208DF81700F7E0AB
:108020000499012081F83C00FFE7FFE7039800680E
:108030000A281CD3FFE70398008800EB4000A0F15A
:108040001E01072000FA01F204980168C8689043F5
:10805000C86003998868098801EB41011E3900FA5C
:1080600001F204980168C8681043C86018E00398DA
:10807000008800EB4001072000FA01F20498016833
:1080800008699043086103998868098801EB4101F8
:1080900000FA01F204980168086910430861FFE7DB
:1080A0000398406806281BD8FFE70398406800EB58
:1080B0008000411F1F2000FA01F204980168486BFC
:1080C0009043486303990888496801EB81010539A9
:1080D00000FA01F204980168486B104348633DE0E0
:1080E000039840680C281CD8FFE70398406800EB11
:1080F0008000A0F123011F2000FA01F2049801681A
:10810000086B9043086303990888496801EB810173
:10811000233900FA01F204980168086B10430863E0
:108120001BE00398406800EB8000A0F141011F2094
:1081300000FA01F204980168C86A9043C862039982
:108140000888496801EB8101413900FA01F204987D
:108150000168C86A1043C862FFE7FFE742F20030D7
:10816000C4F2010001900498006842F20001C4F2D8
:10817000010188420BD1FFE703980068122806D15D
:10818000FFE70199486840F480004860FFE70498E1
:10819000006842F20001C4F2010188422ED1FFE7DB
:1081A00003980068102805D0FFE70398006811289D
:1081B00024D1FFE70199486840F400004860039823
:1081C0000068102819D1FFE740F22800C2F2000031
:1081D00000684DF68361C4F21B31A0FB0110800CD6
:1081E00000EB800040000290FFE7029820B1FFE71B
:1081F000029801380290F8E7FFE7FFE7FFE70499EC
:10820000002081F83C00FFE700208DF81700FFE711
:108210009DF8170006B080BD81B0009000980068FE
:10822000C06C01B07047000080B584B0029000209F
:108230008DF80700029820B9FFE701208DF80F00A4
:10824000C7E10298006842F20001C4F201018842CD
:1082500012D0FFE70298006842F20011C4F2010157
:10826000884209D0FFE70298006842F20021C4F278
:108270000101884201D1FFE708E045F21650C0F63F
:10828000020040F2431115F023FCFFE7029840681A
:1082900090B1FFE702984068B0F5803F0CD0FFE74F
:1082A00002984068B0F5003F06D0FFE702984068AA
:1082B000B0F5403F01D1FFE708E045F21650C0F6A7
:1082C00002004FF4A27115F003FCFFE702988068EA
:1082D00090B1FFE702988068B0F1807F0CD0FFE793
:1082E00002988068B0F1007F06D0FFE702988068AE
:1082F000B0F1407F01D1FFE708E045F21650C0F62B
:10830000020040F2451115F0E3FBFFE70298006917
:1083100028B1FFE702980069012801D1FFE708E0D2
:1083200045F21650C0F602004FF4A37115F0D0FBD1
:10833000FFE70298007E28B1FFE70298007E01283F
:1083400001D1FFE708E045F21650C0F6020040F206
:10835000471115F0BDFBFFE70298806A002862D044
:10836000FFE70298806AB0F1807F5CD0FFE7029857
:10837000806AB0F1007F56D0FFE70298806AB0F1C2
:10838000407F50D0FFE70298806AB0F1806F4AD0FA
:10839000FFE70298806AB0F1A06F44D0FFE702982F
:1083A000806AB0F1C06F3ED0FFE70298806AB0F1FA
:1083B000E06F38D0FFE70298806AB0F1006F32D0EA
:1083C000FFE70298806AB0F1106F2CD0FFE70298A7
:1083D000806AB0F1206F26D0FFE70298806AB0F182
:1083E000306F20D0FFE70298806AB0F1406F1AD05A
:1083F000FFE70298806AB0F1506F14D0FFE702984F
:10840000806AB0F1606F0ED0FFE70298806AB0F129
:10841000706F08D0FFE70298806A0121C0F60071F2
:10842000884201D1FFE708E045F21650C0F602008D
:108430004FF4A47115F04CFBFFE70298C06830B10F
:10844000FFE70298C068B0F5006F01D1FFE708E0D0
:1084500045F21650C0F6020040F2491115F038FB03
:10846000FFE70298C06930B1FFE70298C0691028A1
:1084700001D8FFE708E045F21650C0F602004FF4BD
:10848000A57115F025FBFFE7029890F8300030B198
:10849000FFE7029890F83000012801D1FFE708E0DB
:1084A00045F21650C0F6020040F24B1115F010FBD9
:1084B000FFE702984069012809D0FFE70298406968
:1084C00028B1FFE702984069022801D1FFE708E0E0
:1084D00045F21650C0F602004FF4A67115F0F8FAF6
:1084E000FFE7029890F8200030B1FFE7029890F87B
:1084F0002000012801D1FFE708E045F21650C0F640
:10850000020040F24D1115F0E3FAFFE70298806A8D
:108510000121C0F60071884221D0FFE70298C06AAD
:1085200090B1FFE70298C06AB0F1805F0CD0FFE71E
:108530000298C06AB0F1005F06D0FFE70298C06AF7
:10854000B0F1405F01D1FFE708E045F21650C0F6F8
:10855000020040F2511115F0BBFAFFE7FFE7029865
:10856000006C50B9FFE7029800F038F8029900203B
:108570004864029981F83C00FFE70298006CC0064D
:10858000002817D4FFE70298006C40F0020020F4A6
:108590008850029908640298F8F742FA029900207C
:1085A00048640298006C40F0010020F0020002993B
:1085B000086403E001208DF80700FFE7FFE7029958
:1085C000002081F83C00FFE79DF807008DF80F00C0
:1085D000FFE79DF80F0004B080BD000080B58AB0B1
:1085E0000990002008900790069005900490099843
:1085F000006842F20001C4F20101884212D1FFE793
:10860000FFE70020039043F64400C4F20200016833
:1086100041F480710160006800F480700390039859
:10862000FFE73AE00998006842F20021C4F2010134
:10863000884231D1FFE7FFE70020029043F6440073
:10864000C4F20200016841F480610160006800F436
:10865000806002900298FFE7FFE70020019043F658
:108660003000C4F20200016841F02001016000689E
:1086700000F0200001900198FFE74FF48060049023
:10868000032005900020069041F20040C4F2020051
:1086900004A902F089FCFFE7FFE70AB080BD0000F3
:1086A00080B584B00290019100200090029800688B
:1086B00080684005002816D5FFE7029800688068AA
:1086C000C00500280FD5FFE70299086C40F0200094
:1086D0000864FFE70299002081F83C00FFE70120D1
:1086E0008DF80F006DE003F055F80090FFE7029859
:1086F0000068006800F00200022829D0FFE7019816
:10870000013020B3FFE7019840B1FFE703F042F8E2
:108710000099401A0199884218D9FFE70298006829
:10872000006800F0020002280FD0FFE70299086CF1
:1087300040F004000864FFE70299002081F83C0043
:10874000FFE703208DF80F003BE0FFE7FFE7CEE7F0
:10875000029801686FF0120008600299086C40F4FA
:108760000070086402980068806810F0405F24D1AF
:10877000FFE70298007E00BBFFE702980068C06A2E
:1087800010F4700F07D0FFE702980068806840057A
:10879000002812D4FFE70299086C20F48070086466
:1087A0000298006CC004002806D4FFE70299086C08
:1087B00040F001000864FFE7FFE700208DF80F009C
:1087C000FFE79DF80F0004B080BD000080B584B0C5
:1087D0000290002001900298007E28B1FFE70298E5
:1087E000007E012801D1FFE708E045F21650C0F6EF
:1087F000020040F2D32115F06BF9FFE70298C06A3E
:1088000090B1FFE70298C06AB0F1805F0CD0FFE73B
:108810000298C06AB0F1005F06D0FFE70298C06A14
:10882000B0F1405F01D1FFE708E045F21650C0F615
:1088300002004FF4357115F04BF9FFE7FFE702989E
:1088400090F83C00012804D1FFE702208DF80F00CA
:10885000D4E00299012081F83C00FFE7FFE702988D
:1088600000688068C007F0B9FFE70298016888686F
:1088700040F00100886040F22800C2F20000006869
:108880004DF68361C4F21B31A0FB0110800C00EB9C
:1088900040000190FFE7019820B1FFE701980138FF
:1088A0000190F8E7FFE7029800688068C007002899
:1088B00000F09580FFE70298006C40F4807040F271
:1088C0000161884302990864029800684068400585
:1088D000002809D5FFE70298006C40F4805020F48E
:1088E000005002990864FFE70298006CC004002859
:1088F00006D5FFE70299486C20F00600486403E0C3
:10890000029900204864FFE7FFE70299002081F800
:108910003C00FFE742F20030C4F2010000900298F0
:1089200001686FF02200086000984068C006E8BB4C
:10893000FFE70298006842F20001C4F20101884298
:1089400024D0FFE70298006842F20011C4F201014E
:10895000884208D1FFE742F20430C4F20100006807
:10896000C00698B1FFE70298006842F20021C4F205
:108970000101884219D1FFE742F20430C4F201003C
:10898000006800F01F000F280FD8FFE7029800686A
:10899000806810F0405F07D1FFE70298016888689F
:1089A00040F080408860FFE7FFE717E0029800682A
:1089B00042F20001C4F2010188420ED1FFE70298A1
:1089C0000068806810F0405F07D1FFE702980168F7
:1089D000886840F080408860FFE7FFE70AE002997E
:1089E000086C40F0100008640299486C40F00100E7
:1089F0004864FFE700208DF80F00FFE79DF80F00A7
:108A000004B080BD80B584B002900191029890F8C6
:108A100020008DF80300019848F67F71C0F2030131
:108A2000884201D8FFE708E045F24E50C0F6020048
:108A30004FF4D06115F04CF8FFE79DF803000128D2
:108A400005D0FFE79DF8030002280AD1FFE7019A4D
:108A50000298016848691043486100208DF80F00B2
:108A600008E00299486A40F48020486201208DF8AD
:108A70000F00FFE79DF80F0004B080BD80B588B0FF
:108A80000690059104920393069890F820008DF8C3
:108A9000070006980068806800900598806828B1F3
:108AA000FFE705988068042801D1FFE708E045F258
:108AB0004E50C0F6020040F2E94115F009F8FFE718
:108AC0000598C06828B1FFE70598C068022801D161
:108AD000FFE708E045F24E50C0F6020040F2EA41DE
:108AE00014F0F6FFFFE705980069082801D8FFE7B2
:108AF00008E045F24E50C0F6020040F2EB4114F09F
:108B0000E7FFFFE70598806890B9FFE705980168DF
:108B10000020B0EBD12F01D1FFE708E045F24E5025
:108B2000C0F6020040F2EE4114F0D2FFFFE711E080
:108B3000059841680020B0EB517F01D1FFE708E0C4
:108B400045F24E50C0F6020040F2F24114F0C0FF70
:108B5000FFE7FFE70598007D28B1FFE70598007D56
:108B6000012801D1FFE708E045F24E50C0F60200AF
:108B700040F2F44114F0ACFFFFE79DF80700012834
:108B800006D0FFE79DF80700022840F08D80FFE740
:108B90009DF80300400700280CD4FFE79DF8030070
:108BA0000007002806D4FFE79DF80300C006002850
:108BB00071D5FFE70098C0F3016002900298032886
:108BC00009D3FFE70699486A40F400004862012093
:108BD0008DF81F0071E00299012088400399086018
:108BE0000598806868B9FFE705980168C06840EAA1
:108BF000415006990968029A01EB0211C1F88001FF
:108C00000EE005994A688868C96840EAC2000843CE
:108C100006990968029A01EB0211C1F88001FFE789
:108C20000598006906990968029A01EB0211C1F8DA
:108C300084010598007D01280CD1FFE706980068A3
:108C4000029900EB0111D1F8840140F48070C1F861
:108C50008401FFE70498406806990968029A01EBCD
:108C60000211C1F88C010498006806990968029AFB
:108C700001EB0211C1F8880106980068029900EB27
:108C80000111D1F8800140F00100C1F880010020FD
:108C90008DF81F0011E00699486A40F40010486200
:108CA00001208DF81F0008E00699486A40F48020F2
:108CB000486201208DF81F00FFE79DF81F0008B0F3
:108CC00080BD000080B586B00490039104980068D0
:108CD0000190049890F820008DF803009DF803009F
:108CE000012806D0FFE79DF80300022840F05281DA
:108CF000FFE70398408808B9FFE708E045F24E50C7
:108D0000C0F602004FF4547114F0E2FEFFE703983E
:108D1000C08808B9FFE708E045F24E50C0F60200EF
:108D200040F2513114F0D4FEFFE70398408908B9AE
:108D3000FFE708E045F24E50C0F6020040F2523123
:108D400014F0C6FEFFE70398C08908B9FFE708E002
:108D500045F24E50C0F6020040F2533114F0B8FE16
:108D6000FFE70398806928B1FFE70398806901282D
:108D700001D1FFE708E045F24E50C0F602004FF483
:108D8000557114F0A5FEFFE70398C06928B1FFE70D
:108D90000398C069012801D1FFE708E045F24E5071
:108DA000C0F6020040F2553114F092FEFFE703983E
:108DB000006928B1FFE703980069012801D1FFE7A6
:108DC00008E045F24E50C0F6020040F2563114F071
:108DD0007FFEFFE70398006A28B1FFE70398006A67
:108DE000012801D1FFE708E045F24E50C0F602002D
:108DF00040F2573114F06CFEFFE746F20040C4F237
:108E000000000190039840691B2801D8FFE708E0A3
:108E100045F24E50C0F6020040F2723114F058FE96
:108E2000FFE70398406A1B2801D8FFE708E045F2F6
:108E30004E50C0F6020040F2733114F049FEFFE7D5
:108E40000199D1F8000240F00100C1F80002019937
:108E5000D1F8000220F47C50C1F800020398426A65
:108E60000199D1F8000240EA0220C1F800020398FB
:108E7000406900F01F01012088400290029A019988
:108E8000D1F81C029043C1F81C020398C069F0B9E4
:108E9000FFE7029A0199D1F80C029043C1F80C0245
:108EA000039A9088D168526940EA0140019901EB28
:108EB000C201C1F84002039A10889168526940EAE1
:108EC0000140019901EBC201C1F84402FFE7039898
:108ED000C06901281ED1FFE7029A0199D1F80C025E
:108EE0001043C1F80C02039A90881168526940EA55
:108EF0000140019901EBC201C1F84002039A908937
:108F00009168526940EA0140019901EBC201C1F840
:108F10004402FFE70398806940B9FFE7029A01998C
:108F2000D1F804029043C1F8040207E0029A0199C3
:108F3000D1F804021043C1F80402FFE70398006966
:108F400040B9FFE7029A0199D1F814029043C1F8A1
:108F5000140207E0029A0199D1F814021043C1F8F3
:108F60001402FFE70398006A012808D1FFE7029A7C
:108F70000199D1F81C021043C1F81C02FFE70199C6
:108F8000D1F8000220F00100C1F8000200208DF8A5
:108F9000170008E00499486A40F4802048620120E4
:108FA0008DF81700FFE79DF8170006B080BD0000A0
:108FB00080B582B001900198FAF74CFD8DF803005E
:108FC0009DF80300032819D0FFE79DF8030040F245
:108FD0005042C2F20002342110FB0120006B60B14C
:108FE000FFE79DF8030040F25042C2F20002342134
:108FF00010FB0120006B8047FFE7FFE702B080BD58
:1090000080B586B00490039102920193049890F881
:1090100020008DF80300039820B1FFE70398012892
:1090200001D1FFE708E045F24E50C0F602004FF4D0
:10903000BE6114F04DFDFFE79DF80300012806D046
:10904000FFE79DF80300022840F0D780FFE7039870
:1090500080B9FFE704980068C068800748B9FFE757
:109060000499486A40F40010486201208DF8170006
:10907000CCE00FE0049800680069800748B9FFE77A
:109080000499486A40F40010486201208DF81700E6
:10909000BCE0FFE704980068039900EB0110D0F8EA
:1090A000B00100F00400029988600298806858B905
:1090B000FFE704980068039900EB0110D0F8B001B5
:1090C000400D029908600AE004980068039900EBDB
:1090D0000110D0F8B001C00802994860FFE7049879
:1090E0000068039900EB0110D0F8B00100F0020015
:1090F0000299C86004980068039900EB0110D0F849
:10910000B40100F00F000299086104980068039907
:1091100000EB0110D0F8B40180B2000A0299886116
:1091200004980068039900EB0110D0F8B401000C1A
:109130000299486104980068039900EB0110D0F887
:10914000B8010199087004980068039900EB0110B8
:10915000D0F8B801000A0199487004980068039992
:1091600000EB0110D0F8B801000C01998870049848
:109170000068039900EB0110D0F8B801000E0199C6
:10918000C87004980068039900EB0110D0F8BC0186
:109190000199087104980068039900EB0110D0F858
:1091A000BC01000A0199487104980068039900EB1A
:1091B0000110D0F8BC01000C019988710498006876
:1091C000039900EB0110D0F8BC01000E0199C871A1
:1091D000039838B9FFE704980168C86840F0200098
:1091E000C86006E004980168086940F02000086142
:1091F000FFE700208DF8170008E00499486A40F462
:109200008020486201208DF81700FFE79DF81700C5
:1092100006B080BD80B58AB00990002008900998FA
:1092200000684069079009980068406806900998AE
:1092300000688068059009980068C06804900998E3
:1092400000680069039009980068806902909DF8A1
:109250001C00C007002800F09480FFE79DF8140070
:10926000C00758B3FFE709980168012088609DF89E
:1092700014008007002804D5FFE7099800F042FE9B
:109280001BE09DF814004007002805D5FFE708986B
:1092900040F4006008900FE09DF8140000070028DB
:1092A00005D5FFE7089840F48050089003E009983E
:1092B00000F000FEFFE7FFE7FFE7FFE79DF815007E
:1092C000C00760B3FFE7099801684FF480708860B9
:1092D0009DF815008007002804D5FFE7099800F0E5
:1092E0005FFE1BE09DF815004007002805D5FFE74D
:1092F000089840F4005008900FE09DF81500000712
:10930000002805D5FFE7089840F48040089003E066
:10931000099800F01DFEFFE7FFE7FFE7FFE79DF874
:109320001600C00760B3FFE7099801684FF480306A
:1093300088609DF816008007002804D5FFE709988B
:1093400000F07EFE1BE09DF816004007002805D5C2
:10935000FFE7089840F4004008900FE09DF81600E1
:109360000007002805D5FFE7089840F480300890F2
:1093700003E0099800F03CFEFFE7FFE7FFE7FFE7A7
:10938000FFE79DF81C000007002810D5FFE79DF8B7
:109390001000C006002809D5FFE7089840F40070C7
:1093A0000890099801681020C860FFE7FFE79DF862
:1093B0001C00400700280FD5FFE79DF810000007AC
:1093C000002808D5FFE7099801680820C8600998B7
:1093D00000F062FCFFE7FFE79DF81C008007002813
:1093E0000BD5FFE709980068C068800720B1FFE748
:1093F000099800F079FCFFE7FFE79DF81C004006A4
:10940000002810D5FFE79DF80C00C006002809D5FC
:10941000FFE7089840F480600890099801681020E0
:109420000861FFE7FFE79DF81C00800600280FD5C4
:10943000FFE79DF80C000007002808D5FFE7099812
:10944000016808200861099800F076FCFFE7FFE753
:109450009DF81C00C00600280BD5FFE7099800689E
:109460000069800720B1FFE7099800F08DFCFFE755
:10947000FFE79DF81E00800700280FD5FFE79DF845
:109480001800C006002808D5FFE7099801681020D9
:109490004860099800F0A0FCFFE7FFE79DF81E0078
:1094A000C00778B1FFE79DF818000007002808D52D
:1094B000FFE70998016808204860099800F0E8FD76
:1094C000FFE7FFE79DF81D000006002840F18D80B2
:1094D000FFE79DF818004007002840F18180FFE772
:1094E0009DF81D00C00750B1FFE79DF80800C007B8
:1094F00028B1FFE7089840F001000890FFE79DF8C9
:109500001D00800700280BD5FFE79DF808008007A5
:10951000002805D5FFE7089840F002000890FFE713
:109520009DF81D00400700280BD5FFE79DF80800B7
:109530004007002805D5FFE7089840F00400089090
:10954000FFE79DF81D000007002848D5FFE79DF8BC
:10955000080010F0700F42D0FFE7029800F0700092
:1095600001460191102814D0FFE70198202815D05A
:10957000FFE70198302816D0FFE70198402817D060
:10958000FFE70198502818D0FFE70198602819D00C
:109590001DE0089840F00800089019E0089840F095
:1095A0001000089014E0089840F0200008900FE0A8
:1095B000089840F0400008900AE0089840F08000C9
:1095C000089005E0089840F48070089000E0FFE7FC
:1095D00009980168886920F070008861FFE7FFE75B
:1095E0000998016804204860FFE7089848B1FFE740
:1095F000089A0999486A104348620998FFF7D8FC0D
:10960000FFE70AB080BD000080B584B002900298E8
:1096100020B9FFE701208DF80F0063E2029800688F
:1096200046F20041C4F20001884209D0FFE70298E7
:10963000006846F60001C4F20001884201D1FFE74C
:1096400008E045F24E50C0F6020040F21D1114F041
:109650003FFAFFE70298007E28B1FFE70298007EFC
:10966000012801D1FFE708E045F24E50C0F60200A4
:109670004FF48F7114F02CFAFFE70298407E28B166
:10968000FFE70298407E012801D1FFE708E045F29C
:109690004E50C0F6020040F21F1114F019FAFFE715
:1096A0000298807E28B1FFE70298807E012801D1D0
:1096B000FFE708E045F24E50C0F602004FF490710B
:1096C00014F006FAFFE70298C07E28B1FFE702987F
:1096D000C07E012801D1FFE708E045F24E50C0F6F8
:1096E000020040F2211114F0F3F9FFE70298007F25
:1096F00028B1FFE70298007F012801D1FFE708E0C9
:1097000045F24E50C0F602004FF4917114F0E0F9AA
:10971000FFE70298407F28B1FFE70298407F0128C9
:1097200001D1FFE708E045F24E50C0F6020040F2DA
:10973000231114F0CDF9FFE70298806890B1FFE79C
:1097400002988068B0F1804F0CD0FFE702988068E3
:10975000B0F1004F06D0FFE702988068B0F1404FAB
:1097600001D1FFE708E045F24E50C0F602004FF489
:10977000927114F0ADF9FFE70298C06890B1FFE76D
:109780000298C068B0F1807F0CD0FFE70298C068F3
:10979000B0F1007F06D0FFE70298C068B0F1407FCB
:1097A00001D1FFE708E045F24E50C0F6020040F25A
:1097B000251114F08DF9FFE70298006900285AD0AE
:1097C000FFE702980069B0F5803F54D0FFE70298A8
:1097D0000069B0F5003F4ED0FFE702980069B0F590
:1097E000403F48D0FFE702980069B0F5802F42D093
:1097F000FFE702980069B0F5A02F3CD0FFE7029880
:109800000069B0F5C02F36D0FFE702980069B0F5C7
:10981000E02F30D0FFE702980069B0F5002F2AD082
:10982000FFE702980069B0F5102F24D0FFE70298F7
:109830000069B0F5202F1ED0FFE702980069B0F54F
:10984000302F18D0FFE702980069B0F5402F12D0F2
:10985000FFE702980069B0F5502F0CD0FFE702989F
:109860000069B0F5602F06D0FFE702980069B0F5F7
:10987000702F01D1FFE708E045F24E50C0F602001C
:109880004FF4937114F024F9FFE70298406950B344
:10989000FFE702984069B0F5801F24D0FFE70298E7
:1098A0004069B0F5001F1ED0FFE702984069B0F58F
:1098B000401F18D0FFE702984069B0F5800F12D022
:1098C000FFE702984069B0F5A00F0CD0FFE70298BF
:1098D0004069B0F5C00F06D0FFE702984069B0F5C7
:1098E000E00F01D1FFE708E045F24E50C0F602005C
:1098F00040F2271114F0ECF8FFE70298406838B105
:10990000FFE702984068B0F5806F01D8FFE708E0F4
:1099100045F24E50C0F602004FF4947114F0D8F89E
:10992000FFE7029890F8200020B9FFE7029800F0C6
:10993000DDF8FFE702980168086820F0020008607F
:1099400001F028FF0190FFE7029800684068800757
:10995000002815D5FFE701F01DFF0199401A0B28DB
:109960000DD3FFE70299486A40F40030486202993B
:10997000052081F8200001208DF80F00B2E0E3E718
:1099800002980168086840F00100086001F002FFD9
:109990000190FFE7029800684068C007A8B9FFE798
:1099A00001F0F8FE0199401A0B280DD3FFE7029948
:1099B000486A40F4003048620299052081F820008E
:1099C00001208DF80F008DE0E4E70298007E012869
:1099D00007D1FFE702980168086840F0800008603E
:1099E00006E002980168086820F080000860FFE740
:1099F0000298407E012807D1FFE7029801680868B5
:109A000040F04000086006E002980168086820F015
:109A100040000860FFE70298807E012807D1FFE739
:109A200002980168086840F02000086006E002988B
:109A30000168086820F020000860FFE70298C07EF7
:109A4000012807D1FFE702980168086820F010009C
:109A5000086006E002980168086840F0100008609D
:109A6000FFE70298007F012807D1FFE7029801680D
:109A7000086840F00800086006E00298016808687D
:109A800020F008000860FFE70298407F012807D116
:109A9000FFE702980168086840F00400086006E0EB
:109AA00002980168086820F004000860FFE7029B44
:109AB00019685A689868D3F80CC040EA0C00D3F8CB
:109AC00010C040EA0C005B691843013A1043C861BA
:109AD000029900204862029A012182F820108DF834
:109AE0000F00FFE79DF80F0004B080BD80B594B073
:109AF000139000201290119010900F900E901398D8
:109B0000006846F20041C4F20001884253D1FFE7E9
:109B100040F21450C2F20000016801310160006897
:109B2000012812D1FFE7FFE700200D9043F6400027
:109B3000C4F20200016841F000710160006800F0A9
:109B400000700D900D98FFE7FFE7FFE700200C90F5
:109B500043F63000C4F20200016841F008010160E0
:109B6000006800F008000C900C98FFE703200E90AE
:109B700002210F910021079110911190092012905C
:109B800040F60040C4F202000EA901F00DFA079A57
:109B9000142005900521069102F018FA059802F0AC
:109BA000FDF90699079A1520089002F00FFA089817
:109BB00002F0F4F96EE01398006846F60001C4F272
:109BC0000001884265D1FFE7FFE700200B9043F6D4
:109BD0004000C4F20200016841F080610160006849
:109BE00000F080600B900B98FFE740F21450C2F237
:109BF00000000168013101600068012812D1FFE70F
:109C0000FFE700200A9043F64000C4F2020001681A
:109C100041F000710160006800F000700A900A983D
:109C2000FFE7FFE7FFE70020099043F63000C4F2AA
:109C30000200016841F002010160006800F00200CA
:109C400009900998FFE760200E9002200F900020F5
:109C500003901090032011900920129040F20040D0
:109C6000C4F202000EA901F09FF9039A402001906E
:109C70000521029102F0AAF9019802F08FF90299E8
:109C8000039A4120049002F0A1F9049802F086F9A9
:109C9000FFE7FFE714B080BD80B582B00190019866
:109CA000F9F7D8FE8DF803009DF80300032819D0BA
:109CB000FFE79DF8030040F25042C2F20002342157
:109CC00010FB0120C06960B1FFE79DF8030040F27E
:109CD0005042C2F20002342110FB0120C0698047CB
:109CE000FFE7FFE702B080BD80B582B00190019828
:109CF000F9F7B0FE8DF803009DF80300032819D092
:109D0000FFE79DF8030040F25042C2F20002342106
:109D100010FB0120806960B1FFE79DF8030040F26D
:109D20005042C2F20002342110FB012080698047BA
:109D3000FFE7FFE702B080BD80B582B001900198D7
:109D4000F9F788FE8DF803009DF80300032819D069
:109D5000FFE79DF8030040F25042C2F200023421B6
:109D600010FB0120406A60B1FFE79DF8030040F25C
:109D70005042C2F20002342110FB0120406A8047A9
:109D8000FFE7FFE702B080BD80B582B00190019887
:109D9000F9F760FE8DF803009DF80300032819D041
:109DA000FFE79DF8030040F25042C2F20002342166
:109DB00010FB0120006A60B1FFE79DF8030040F24C
:109DC0005042C2F20002342110FB0120006A804799
:109DD000FFE7FFE702B080BD80B582B00190019837
:109DE000F9F738FE8DF803009DF80300032819D019
:109DF000FFE79DF8030040F25042C2F20002342116
:109E000010FB0120806A60B1FFE79DF8030040F27B
:109E10005042C2F20002342110FB0120806A8047C8
:109E2000FFE7FFE702B080BD80B584B002900298E2
:109E300090F8200001282FD1FFE70299022081F835
:109E4000200002980168086820F00100086001F015
:109E5000A1FC0190FFE7029800684068C007A8B124
:109E6000FFE701F097FC0199401A0B280DD3FFE79B
:109E70000299486A40F4003048620299052081F84E
:109E8000200001208DF80F000FE0E4E70299002088
:109E900048628DF80F0008E00299486A40F40020FB
:109EA000486201208DF80F00FFE79DF80F0004B015
:109EB00080BD000080B582B001900198F9F7CAFD1D
:109EC0008DF803009DF80300032819D0FFE79DF8E3
:109ED000030040F25042C2F20002342110FB012084
:109EE000C06860B1FFE79DF8030040F25042C2F243
:109EF0000002342110FB0120C0688047FFE7FFE724
:109F000002B080BD80B582B001900198F9F7A2FD42
:109F10008DF803009DF80300032817D0FFE79DF894
:109F200003003421414340F25040C2F20000405847
:109F300058B1FFE79DF803003421414340F25040FF
:109F4000C2F2000040588047FFE7FFE702B080BD43
:109F500080B582B001900198F9F77CFD8DF803007F
:109F60009DF80300032819D0FFE79DF8030040F295
:109F70005042C2F20002342110FB0120006960B19E
:109F8000FFE79DF8030040F25042C2F20002342184
:109F900010FB012000698047FFE7FFE702B080BDAA
:109FA00080B582B001900198F9F754FD8DF8030057
:109FB0009DF80300032819D0FFE79DF8030040F245
:109FC0005042C2F20002342110FB0120406860B10F
:109FD000FFE79DF8030040F25042C2F20002342134
:109FE00010FB012040688047FFE7FFE702B080BD1B
:109FF00080B582B001900198F9F72CFD8DF803002F
:10A000009DF80300032819D0FFE79DF8030040F2F4
:10A010005042C2F20002342110FB0120406960B1BD
:10A02000FFE79DF8030040F25042C2F200023421E3
:10A0300010FB012040698047FFE7FFE702B080BDC9
:10A0400080B582B001900198F9F704FD8DF8030006
:10A050009DF80300032819D0FFE79DF8030040F2A4
:10A060005042C2F20002342110FB0120806860B12E
:10A07000FFE79DF8030040F25042C2F20002342193
:10A0800010FB012080688047FFE7FFE702B080BD3A
:10A0900080B582B001900198F9F7DCFC8DF80300DF
:10A0A0009DF80300032819D0FFE79DF8030040F254
:10A0B0005042C2F20002342110FB0120C06A60B19C
:10A0C000FFE79DF8030040F25042C2F20002342143
:10A0D00010FB0120C06A8047FFE7FFE702B080BDA8
:10A0E00080B582B00090009820B9FFE701208DF87C
:10A0F000070023E00098006843F20001C4F2020167
:10A10000884201D1FFE707E045F28650C0F6020021
:10A11000682113F0DDFCFFE70098407938B9FFE7CC
:10A12000009900200871009800F00CF8FFE70099F2
:10A130000120487100208DF80700FFE79DF8070017
:10A1400002B080BD82B001900198006843F2000126
:10A15000C4F20201884212D1FFE7FFE7002000901D
:10A1600043F63000C4F20200016841F480510160FE
:10A17000006800F4805000900098FFE7FFE702B00D
:10A180007047000080B584B002900298806D019005
:10A1900001F000FB0090029890F8350002280DD0E5
:10A1A000FFE7029980204865FFE70299002081F8C7
:10A1B0003400FFE701208DF80F0054E00298016899
:10A1C000086820F01600086002980168486920F0CD
:10A1D000800048610298006C20B9FFE70298806C0B
:10A1E00038B1FFE702980168086820F008000860AD
:10A1F000FFE702980168086820F001000860FFE7A7
:10A20000029800680068C007C0B1FFE701F0C2FA19
:10A210000099401A062810D3FFE7029920204865CC
:10A22000FFE70299002081F83400FFE7029903203C
:10A2300081F835008DF80F0015E0E1E70298C16D57
:10A240003F20884001998860FFE70299002081F84B
:10A250003400FFE70299012081F83500FFE7002074
:10A260008DF80F00FFE79DF80F0004B080BD0000DF
:10A2700082B00090009890F83500022807D0FFE7E0
:10A2800000998020486501208DF807000EE00099B4
:10A29000052081F8350000980168086820F0010069
:10A2A0000860FFE700208DF80700FFE79DF8070032
:10A2B00002B0704780B586B005900020039040F250
:10A2C0002800C2F20000006848F2B511C1F64E3114
:10A2D000A0FB0110800A02900598806D0190019802
:10A2E0000068049004980599C96DC84000070028CB
:10A2F0001AD5FFE70598006800684007002812D5C6
:10A30000FFE705980168086820F0040008600598D8
:10A31000C16D08208840019988600599486D40F01A
:10A3200001004865FFE7FFE704980599C96DC8403B
:10A33000C007A0B1FFE70598006840690006002843
:10A340000CD5FFE70598C16D012088400199886010
:10A350000599486D40F002004865FFE7FFE7049863
:10A360000599C96DC8404007002814D5FFE7059836
:10A3700000680068800700280CD5FFE70598C16DCC
:10A3800004208840019988600599486D40F00400D8
:10A390004865FFE7FFE704980599C96DC840C00606
:10A3A000002847D5FFE705980068006800070028E7
:10A3B0003FD5FFE70598C16D10208840019988605E
:10A3C000059800680068400300281AD5FFE7059843
:10A3D000006800680003002809D4FFE70598006CB6
:10A3E00020B1FFE70598016C8847FFE708E0059872
:10A3F000806C20B1FFE70598816C8847FFE7FFE795
:10A4000016E0059800680068C005002807D4FFE73B
:10A4100005980168086820F008000860FFE70598C3
:10A42000006C20B1FFE70598016C8847FFE7FFE764
:10A43000FFE7FFE704980599C96DC840800600282A
:10A4400040F18D80FFE7059800680068C00600288D
:10A4500040F18480FFE70598C16D20208840019974
:10A460008860059890F83500052834D1FFE70598F5
:10A470000168086820F016000860059801684869BE
:10A4800020F0800048610598006C20B9FFE705982E
:10A49000806C38B1FFE705980168086820F0080073
:10A4A0000860FFE70598C16D3F20884001998860EA
:10A4B000FFE70599002081F83400FFE705990120A6
:10A4C00081F835000598006D20B1FFE70598016D12
:10A4D0008847FFE77BE00598006800684003002894
:10A4E0001AD5FFE70598006800680003002809D422
:10A4F000FFE70598406C20B1FFE70598416C88475D
:10A50000FFE708E00598C06B20B1FFE70598C16B35
:10A510008847FFE7FFE720E0059800680068C0056E
:10A52000002811D4FFE705980168086820F01000A2
:10A530000860FFE70599002081F83400FFE70599DE
:10A54000012081F83500FFE70598C06B20B1FFE7D7
:10A550000598C16B8847FFE7FFE7FFE7FFE705982E
:10A56000406DA0B3FFE70598406DC00730B3FFE72B
:10A570000599052081F8350005980168086820F0E4
:10A5800001000860FFE703980130039002998842B8
:10A5900001D9FFE707E0FFE7059800680068C007FA
:10A5A0000028F0D1FFE7FFE70599002081F834008B
:10A5B000FFE70599012081F83500FFE70598C06C99
:10A5C00020B1FFE70598C16C8847FFE7FFE706B0B9
:10A5D00080BD000080B586B004900020039001F09B
:10A5E000D9F80290049820B9FFE701208DF81700F0
:10A5F00087E20498006846F21001C4F20201884222
:10A6000000F08880FFE70498006846F22801C4F251
:10A61000020188427ED0FFE70498006846F24001BC
:10A62000C4F20201884275D0FFE70498006846F240
:10A630005801C4F2020188426CD0FFE70498006818
:10A6400046F27001C4F20201884263D0FFE7049829
:10A65000006846F28801C4F2020188425AD0FFE73E
:10A660000498006846F2A001C4F20201884251D069
:10A67000FFE70498006846F2B801C4F2020188427C
:10A6800048D0FFE70498006846F21041C4F2020186
:10A6900088423FD0FFE70498006846F22841C4F2A0
:10A6A0000201884236D0FFE70498006846F2404134
:10A6B000C4F2020188422DD0FFE70498006846F2F8
:10A6C0005841C4F20201884224D0FFE70498006890
:10A6D00046F27041C4F2020188421BD0FFE70498A1
:10A6E000006846F28841C4F20201884212D0FFE7B6
:10A6F0000498006846F2A041C4F20201884209D0E1
:10A70000FFE70498006846F2B841C4F202018842AB
:10A7100001D1FFE707E045F2A340C0F60200B821EF
:10A7200013F0D6F9FFE70498406850B3FFE70498A8
:10A730004068B0F1007F24D0FFE704984068B0F192
:10A74000806F1ED0FFE704984068B0F1C06F18D04A
:10A75000FFE704984068B0F1006F12D0FFE704985B
:10A760004068B0F1206F0CD0FFE704984068B0F16A
:10A77000406F06D0FFE704984068B0F1606F01D1E8
:10A78000FFE707E045F2A340C0F60200B92113F04D
:10A790009FF9FFE70498806850B1FFE7049880684C
:10A7A000402805D0FFE704988068802801D1FFE7A2
:10A7B00007E045F2A340C0F60200BA2113F088F981
:10A7C000FFE70498C068B0F5007F04D0FFE7049865
:10A7D000C06808B9FFE707E045F2A340C0F60200F1
:10A7E000BB2113F075F9FFE704980069B0F5806F9D
:10A7F00004D0FFE70498006908B9FFE707E045F2D5
:10A80000A340C0F60200BC2113F062F9FFE70498F0
:10A81000406960B1FFE704984069B0F5006F06D069
:10A82000FFE704984069B0F5805F01D1FFE707E0DA
:10A8300045F2A340C0F60200BD2113F049F9FFE73D
:10A840000498806960B1FFE704988069B0F5005F03
:10A8500006D0FFE704988069B0F5804F01D1FFE78B
:10A8600007E045F2A340C0F60200BE2113F030F924
:10A87000FFE70498C06958B1FFE70498C069B0F5D4
:10A88000807F05D0FFE70498C069202801D1FFE749
:10A8900007E045F2A340C0F60200BF2113F018F90B
:10A8A000FFE70498006A90B1FFE70498006AB0F5EA
:10A8B000803F0CD0FFE70498006AB0F5003F06D057
:10A8C000FFE70498006AB0F5403F01D1FFE707E0D9
:10A8D00045F2A340C0F60200C02113F0F9F8FFE7EB
:10A8E0000498406A28B1FFE70498406A042801D11F
:10A8F000FFE707E045F2A340C0F60200C12113F0D4
:10A90000E7F8FFE70498406A00285BD0FFE7049867
:10A91000806A78B1FFE70498806A01280AD0FFE7CF
:10A920000498806A022805D0FFE70498806A03280B
:10A9300001D1FFE707E045F2A340C0F60200C621BF
:10A9400013F0C6F8FFE70498C06A90B1FFE70498D7
:10A95000C06AB0F5000F0CD0FFE70498C06AB0F1F0
:10A96000807F06D0FFE70498C06AB0F1C07F01D1B4
:10A97000FFE707E045F2A340C0F60200C72113F04D
:10A98000A7F8FFE70498006B90B1FFE70498006B0D
:10A99000B0F5001F0CD0FFE70498006BB0F5800FF6
:10A9A00006D0FFE70498006BB0F5C00F01D1FFE7B8
:10A9B00007E045F2A340C0F60200C82113F088F872
:10A9C000FFE7FFE7FFE70499002081F83400FFE785
:10A9D0000499022081F8350004980168086820F085
:10A9E00001000860FFE7049800680068C00790B1A4
:10A9F000FFE700F0CFFE0299401A06280AD3FFE7CE
:10AA00000499202048650499032081F835008DF8C9
:10AA1000170076E0E7E70498006800680390039861
:10AA200048F23F01CFF210010840039004990091D1
:10AA30004868D1F808C0CB680A6940EA0C0018439E
:10AA400010434A6910438A691043CA691043096A6E
:10AA500001430398084303900498406A042808D1EE
:10AA6000FFE70499C86A096B014303980843039000
:10AA7000FFE7039804990968086004980068406932
:10AA80000390039820F0070003900498416A03980C
:10AA9000084303900498406A04281AD1FFE70498F9
:10AAA000816A0398084303900498C06A80B1FFE765
:10AAB0000498FCF723F850B1FFE70499402048655B
:10AAC0000499012081F835008DF8170019E0FFE79F
:10AAD000FFE703980499096848610498FBF7E2FFCF
:10AAE00001900498C16D3F208840019988600499C5
:10AAF00000204865049A012182F835108DF817006E
:10AB0000FFE79DF8170006B080BD000080B588B053
:10AB1000069005910492039300208DF80B0006988F
:10AB2000806D0190039828B1FFE7BDF80E0008B9C9
:10AB3000FFE708E045F2A340C0F602004FF4E671DB
:10AB400012F0C6FFFFE7FFE7069890F834000128EF
:10AB500004D1FFE702208DF81F0045E0069901208F
:10AB600081F83400FFE7FFE7069890F835000128E8
:10AB70002BD1FFE70699022081F8350006990020C5
:10AB8000486506980599049A039BFCF72FF80698E8
:10AB9000C16D3F2088400199886006980168086867
:10ABA00040F0160008600698006C38B1FFE7069880
:10ABB0000168086840F008000860FFE7069801682F
:10ABC000086840F00100086009E0FFE706990020EE
:10ABD00081F83400FFE702208DF80B00FFE79DF8B5
:10ABE0000B008DF81F00FFE79DF81F0008B080BD27
:10ABF00080B584B0039000F0CDFD029003980190E1
:10AC00000198013048B1FFE740F23840C2F200003D
:10AC10000178019808440190FFE7FFE700F0BAFDD2
:10AC20000299401A0199884201D2FFE7F6E704B081
:10AC300080BD000080B586B00490039101208DF89E
:10AC40000B0000200190FFE742F22850C2F2000002
:10AC5000007E012804D1FFE702208DF8170094E060
:10AC600042F22851C2F2000101200876FFE7FFE717
:10AC70000498006828B1FFE704980068012801D112
:10AC8000FFE707E045F22D40C0F60200AB2112F0CD
:10AC90001FFFFFE74CF25030FCF756FC8DF80B001D
:10ACA0009DF80B00002863D1FFE703994FF0FF30B8
:10ACB000086004980068012814D1FFE70499087C13
:10ACC0004968FCF781FA4CF25030FCF73DFC8DF8F6
:10ACD0000B0043F61041C4F20201086820F00400A2
:10ACE000086042E004988168C068084440B1FFE70A
:10ACF00004988168C06808440C2801D8FFE707E081
:10AD000045F22D40C0F60200C32112F0E1FEFFE73C
:10AD1000049880680190FFE7019804998A68C968DF
:10AD20001144884220D2FFE701980499097CFCF77E
:10AD30005FF94CF25030FCF707FC8DF80B0043F63E
:10AD40001041C4F20201086820F0FA0008609DF882
:10AD50000B0020B1FFE701980399086004E0FFE7CA
:10AD6000019801300190D7E7FFE7FCF7DBF9FFE737
:10AD7000FFE742F22851C2F2000100200876FFE707
:10AD80009DF80B008DF81700FFE79DF8170006B03F
:10AD900080BD000043F61041C4F20201086840F093
:10ADA000004008600020704780B588B0069005918B
:10ADB0000393029201208DF80700FFE742F228502A
:10ADC000C2F20000007E012804D1FFE702208DF8C6
:10ADD0001F0069E042F22851C2F20001012008760A
:10ADE000FFE7FFE7069860B1FFE70698012808D063
:10ADF000FFE70698022804D0FFE70698032801D150
:10AE0000FFE707E045F2F330C0F60200A42112F09C
:10AE10005FFEFFE74CF25030FCF796FB8DF8070021
:10AE20009DF8070098BBFFE7069830B9FFE7059843
:10AE30009DF80810FCF70EFA1AE00698012806D1D2
:10AE4000FFE70598BDF80810FCF786FA0FE00698B2
:10AE5000022805D1FFE705980299FCF7BDFA05E045
:10AE60000598029A039BFCF733FAFFE7FFE7FFE739
:10AE70004CF25030FCF768FB8DF8070043F61041A8
:10AE8000C4F20201086820F001000860FFE7FFE754
:10AE900042F22851C2F2000100200876FFE79DF837
:10AEA00007008DF81F00FFE79DF81F0008B080BD68
:10AEB00081B000208DF8030043F61040C4F2020078
:10AEC0000068C00FD8B1FFE743F60441C4F20201A5
:10AED00040F22310C4F26750086048F6AB10CCF67D
:10AEE000EF50086043F61040C4F202000068C00F43
:10AEF00020B1FFE701208DF80300FFE7FFE79DF891
:10AF0000030001B07047000080B582B0ADF80600C4
:10AF100000208DF80500FFE79DF805000F2824DCD0
:10AF2000FFE7BDF806009DF80510C840C007A8B1AE
:10AF3000FFE79DF8051040F2D440C2F2000050F83F
:10AF4000210050B1FFE79DF8051040F2D440C2F255
:10AF5000000050F821008047FFE7FFE7FFE79DF87A
:10AF6000050001308DF80500D6E702B080BD000075
:10AF700080B582B0ADF8060043F61440C4F201007B
:10AF80000068BDF8061008420CD0FFE7BDF80600C7
:10AF900043F61441C4F201010860BDF80600FFF752
:10AFA000B3FFFFE702B080BD80B58EB00D900C916D
:10AFB00000200A90099008900D980021C4F2020127
:10AFC000884240D0FFE70D9840F20041C4F20201F0
:10AFD000884238D0FFE70D9840F60001C4F2020124
:10AFE000884230D0FFE70D9840F60041C4F20201DC
:10AFF000884228D0FFE70D9841F20001C4F2020117
:10B00000884220D0FFE70D9841F20041C4F20201CE
:10B01000884218D0FFE70D9841F60001C4F2020102
:10B02000884210D0FFE70D9841F60041C4F20201BA
:10B03000884208D0FFE70D9842F20001C4F20201F5
:10B04000884201D1FFE707E045F26A40C0F60200FE
:10B05000AC2112F03DFDFFE70C98008828B1FFE716
:10B060000C98408808B9FFE707E045F26A40C0F64F
:10B070000200AD2112F02CFDFFE70C98406800287B
:10B0800049D0FFE70C984068012844D0FFE70C98AE
:10B09000406811283FD0FFE70C98406802283AD05A
:10B0A000FFE70C984068122835D0FFE70C984068FD
:10B0B0000021C1F2110188422DD0FFE70C984068B1
:10B0C0000021C1F22101884225D0FFE70C98406899
:10B0D0000021C1F2310188421DD0FFE70C98406881
:10B0E0000021C1F21201884215D0FFE70C98406898
:10B0F0000021C1F2220188420DD0FFE70C98406880
:10B100000021C1F23201884205D0FFE70C98406867
:10B11000032801D1FFE707E045F26A40C0F60200CC
:10B12000AE2112F0D5FCFFE70C98806850B1FFE724
:10B130000C988068012805D0FFE70C9880680228E9
:10B1400001D1FFE707E045F26A40C0F60200AF21F7
:10B1500012F0BEFCFFE700200B90FFE70B980F28D2
:10B1600000F2B082FFE70B99012088400A900C980A
:10B1700000680A990840099009980A99884240F0A5
:10B180009C82FFE70C98406800F00300012807D07C
:10B19000FFE70C98406800F0030002284BD1FFE75E
:10B1A0000C98C06878B1FFE70C98C06801280AD0F5
:10B1B000FFE70C98C068022805D0FFE70C98C0682C
:10B1C000032801D1FFE707E045F26A40C0F602001C
:10B1D000C12112F07DFCFFE70D98806808900B9864
:10B1E0004100032000FA01F10898884308900C9868
:10B1F000C0680B99490000FA01F1089808430890CB
:10B2000008980D9988600D98406808900B99012066
:10B2100000FA01F10898884308900C984068C0F340
:10B2200000100B9900FA01F108980843089008985B
:10B230000D994860FFE70C98406800F00300032870
:10B2400018D0FFE70D98C06808900B9841000320C4
:10B2500000FA01F10898884308900C9880680B99CF
:10B26000490000FA01F108980843089008980D99E0
:10B27000C860FFE70C98406800F00300022840F027
:10B28000EE80FFE70C980069002800F0B980FFE726
:10B290000C980069092800F0B380FFE70C9800695A
:10B2A000002800F0AD80FFE70C980069002800F04E
:10B2B000A780FFE70C980069002800F0A180FFE755
:10B2C0000C980069002800F09B80FFE70C9800694B
:10B2D000012800F09580FFE70C980069012800F034
:10B2E0008F80FFE70C980069022800F08980FFE753
:10B2F0000C980069022800F08380FFE70C98006931
:10B3000002287DD0FFE70C980069032878D0FFE77A
:10B310000C980069042873D0FFE70C980069042892
:10B320006ED0FFE70C980069042869D0FFE70C98FD
:10B330000069052864D0FFE70C98006905285FD0F4
:10B34000FFE70C98006909285AD0FFE70C980069BC
:10B35000062855D0FFE70C980069092850D0FFE770
:10B360000C98006907284BD0FFE70C980069072864
:10B3700046D0FFE70C980069072841D0FFE70C98FA
:10B38000006908283CD0FFE70C980069082837D0EE
:10B39000FFE70C980069082832D0FFE70C98006995
:10B3A00009282DD0FFE70C980069092828D0FFE76D
:10B3B0000C9800690A2823D0FFE70C9800690A2836
:10B3C0001ED0FFE70C9800690B2819D0FFE70C98F6
:10B3D00000690C2814D0FFE70C9800690C280FD0E6
:10B3E000FFE70C9800690D280AD0FFE70C98006968
:10B3F0000C2805D0FFE70C9800690F2801D1FFE762
:10B4000007E045F26A40C0F60200DC2112F060FB62
:10B41000FFE70D980B996FF0030202EA510108440F
:10B42000006A08900B9800F0070081000F2000FAD6
:10B4300001F10898884308900C9800690B9901F075
:10B440000701890000FA01F108980843089008985C
:10B450000D990B9B02EA530211440862FFE70D9815
:10B46000006808900B984100032000FA01F1089849
:10B47000884308900C98406800F003000B9949003D
:10B4800000FA01F108980843089008980D9908609F
:10B490000C98C079C006002840F10E81FFE7FFE755
:10B4A0000020079043F64400C4F20200016841F412
:10B4B00080410160006800F4804007900798FFE732
:10B4C0000B9820F0030043F60801C4F20101405834
:10B4D00008900B9800F0030081000F2000FA01F1A2
:10B4E0000898884308900D980021C4F20201884210
:10B4F00003D1FFE7002006905EE00D9840F2004186
:10B50000C4F20201884203D1FFE70120059050E018
:10B510000D9840F60001C4F20201884203D1FFE712
:10B520000220049042E00D9840F60041C4F202016E
:10B53000884203D1FFE70320039034E00D9841F2E5
:10B540000001C4F20201884203D1FFE70420029007
:10B5500026E00D9841F20041C4F20201884203D175
:10B56000FFE70520019018E00D9841F60001C4F2B4
:10B570000201884203D1FFE7062000900AE00D99FE
:10B5800041F60042C4F202020820914208BF07209F
:10B590000090FFE700980190FFE701980290FFE715
:10B5A00002980390FFE703980490FFE70498059042
:10B5B000FFE705980690FFE70698C0B20B9901F0E7
:10B5C0000301890000FA01F10898084308900898DF
:10B5D0000B9921F0030143F60802C4F201028850DE
:10B5E00043F60040C4F201000068089009990898E9
:10B5F000884308900C988079C00728B1FFE7099923
:10B60000089808430890FFE7089843F60041C4F201
:10B610000101086043F60440C4F20100006808908C
:10B6200009990898884308900C9880798007002829
:10B6300005D5FFE70999089808430890FFE708989F
:10B6400043F60441C4F20101086043F60840C4F225
:10B6500001000068089009990898884308900C98A0
:10B660008079C006002805D5FFE7099908980843A6
:10B670000890FFE7089843F60841C4F2010108600A
:10B6800043F60C40C4F2010000680890099908983C
:10B69000884308900C9880798006002805D5FFE73C
:10B6A0000999089808430890FFE7089843F60C4169
:10B6B000C4F201010860FFE7FFE7FFE70B980130E4
:10B6C0000B904BE50EB080BD80B582B00190ADF817
:10B6D0000210BDF8020020B1FFE7002008B9FFE723
:10B6E00008E045F26A40C0F602004FF4BD7112F066
:10B6F000EFF9FFE701980069BDF80210084204D095
:10B70000FFE701208DF8010003E000208DF8010023
:10B71000FFE79DF8010002B080BD000080B582B057
:10B720000190ADF802108DF80120BDF8020020B1A3
:10B73000FFE7002008B9FFE708E045F26A40C0F6DD
:10B74000020040F29B1112F0C3F9FFE79DF80100DF
:10B7500028B1FFE79DF80100012801D1FFE708E0CB
:10B7600045F26A40C0F602004FF4CE7112F0B0F913
:10B77000FFE79DF8010028B1FFE7BDF8020001993D
:10B78000886105E0BDF80200000401998861FFE7C7
:10B7900002B080BD49F29870C2F2000000687047A4
:10B7A00080B58EB00C900C9820B9FFE701208DF881
:10B7B000370002E20C98006845F20041C4F2000133
:10B7C000884212D0FFE70C98006845F60001C4F2E9
:10B7D0000001884209D0FFE70C98006845F6004157
:10B7E000C4F20001884201D1FFE708E045F2BE50F3
:10B7F000C0F6020040F2BF1112F06AF9FFE70C98A0
:10B80000406850B1FFE70C98406841F68021C0F2D3
:10B810000601884201D8FFE708E045F2BE50C0F6B5
:10B8200002004FF4E07112F053F9FFE70C988068C2
:10B8300030B1FFE70C988068B0F5804F01D1FFE789
:10B8400008E045F2BE50C0F6020040F2C11112F00D
:10B850003FF9FFE70C98C068800A08B9FFE708E0E5
:10B8600045F2BE50C0F602004FF4E17112F030F91B
:10B87000FFE70C980069B0F5804F06D0FFE70C9801
:10B880000069B0F5404F01D1FFE708E045F2BE5036
:10B89000C0F6020040F2C31112F01AF9FFE70C984B
:10B8A000406928B1FFE70C984069012801D1FFE702
:10B8B00008E045F2BE50C0F602004FF4E27112F00B
:10B8C00007F9FFE70C9880696FF0FE01084201D18B
:10B8D000FFE708E045F2BE50C0F6020040F2C51195
:10B8E00012F0F6F8FFE70C98C06928B1FFE70C9852
:10B8F000C069402801D1FFE708E045F2BE50C0F61C
:10B9000002004FF4E37112F0E3F8FFE70C98006ACD
:10B9100028B1FFE70C98006A802801D1FFE708E012
:10B9200045F2BE50C0F6020040F2C71112F0D0F846
:10B93000FFE70C9890F83D0040B9FFE70C99002014
:10B9400081F83C000C9800F03DF9FFE70C992420A9
:10B9500081F83D000C980168086820F0010008603B
:10B960000C980168086840F4004008600C98016871
:10B97000086820F40040086001F054FE0A900C981A
:10B98000406848F2A061C0F2010188420BD8FFE78D
:10B990000A9948F28042C0F21E020020914238BF4C
:10B9A000012009900AE00A9940F60012C0F23D0217
:10B9B0000020914238BF01200990FFE70998012833
:10B9C00004D1FFE701208DF83700F6E00A984DF624
:10B9D0008361C4F21B31A0FB0110800C0B900C980A
:10B9E0000068406820F03F000B9908430C990968F3
:10B9F00048600C980068006A20F03F0008900C989E
:10BA0000406848F2A061C0F20101884204D8FFE713
:10BA10000B98013007900EE00B984FF49671484355
:10BA200044F6D351C1F26201A0FB0101012000EBF9
:10BA300091100790FFE70898079908430C99096847
:10BA400008620C980068C0694CF6FF718843069044
:10BA50000C98406848F2A061C0F2010188421FD8EA
:10BA6000FFE70A9801380C9949684900B0FBF1F0EA
:10BA700001306FF31F30032803D8FFE7042005903F
:10BA80000BE00A9801380C9949684900B0FBF1F0C5
:10BA900001306FF31F300590FFE7059804904CE0EC
:10BAA0000C98806868B9FFE70A9801380C994968D2
:10BAB00001EB4101B0FBF1F001306FF31F30039057
:10BAC0000DE00A9801380C99496819225143B0FBDE
:10BAD000F1F00130042161F31F300390FFE7039878
:10BAE000000518B9FFE70120029023E00C98806858
:10BAF00068B9FFE70A9801380C99496801EB4101E0
:10BB0000B0FBF1F001306FF31F3001900DE00A98A7
:10BB100001380C99496819225143B0FBF1F001300A
:10BB2000042161F31F300190FFE7019840F40040C9
:10BB30000290FFE702980490FFE7069804990843F3
:10BB40000C990968C8610C980068006820F0C00072
:10BB50000C9B1968DA691B6A1A43104308600C9839
:10BB60000068806848F2FF3188430C9A1168D368F6
:10BB700012691A43104388600C980068C06820F06E
:10BB8000FF000C9B19685A699B691A431043C860EF
:10BB90000C980168086840F0010008600C990020CA
:10BBA00008640C9A202182F83D100C9908630C99C6
:10BBB00081F83E008DF83700FFE79DF837000EB0A2
:10BBC00080BD000080B594B01390002012901190B9
:10BBD00010900F900E901398006845F20041C4F247
:10BBE0000001884235D1FFE7FFE700200D9043F6C2
:10BBF0003000C4F20200016841F0020101600068F7
:10BC000000F002000D900D98FFE74FF440700E9089
:10BC100012200F9001201090032011900420129008
:10BC200040F20040C4F202000EA9FFF7BDF9FFE7A1
:10BC300000200C9043F64000C4F20200016841F479
:10BC400000110160006800F400100C900C98FFE7F0
:10BC5000FBE01398006845F60001C4F20001884239
:10BC60005FD1FFE7FFE700200B9043F63000C4F2FE
:10BC70000200016841F020010160006800F020002E
:10BC80000B900B98FFE703200E9012210F910121DA
:10BC9000109111900420129041F20040C4F2020071
:10BCA0000EA9FFF781F9FFE700200A9043F6400054
:10BCB000C4F20200016841F480010160006800F4F0
:10BCC00080000A900A98FFE741F6C800C2F200001F
:10BCD000069046F2B801C4F2020101604FF06061C3
:10BCE0004160402181600021C1604FF480620261A7
:10BCF00041618161C1614FF4003202624162FEF72D
:10BD000069FC18B1FFE7FBF76FF9FFE7FFE713984E
:10BD100041F6C801C2F20001416313988863FFE74E
:10BD200092E01398006845F60041C4F20001884291
:10BD300040F08980FFE7FFE70020099043F63000DC
:10BD4000C4F20200016841F004010160006800F0E3
:10BD5000040009900998FFE7FFE70020089043F6E8
:10BD60003000C4F20200016841F001010160006886
:10BD700000F0010008900898FFE74FF400700E9063
:10BD8000122001900F900120029010900320039048
:10BD9000119004200490129040F60000C4F20200BA
:10BDA0000EA90591FFF700F9DDF804C0029B039A84
:10BDB000049805994FF4807ECDF838E0CDF83CC06A
:10BDC0001093119212900020C4F20200FFF7ECF8D9
:10BDD000FFE70020079043F64000C4F2020001682C
:10BDE00041F400010160006800F40000079007982A
:10BDF000FFE741F62810C2F20000009046F2400131
:10BE0000C4F2020101604FF0C06141600021816015
:10BE1000C1604FF48062026141618161C161016270
:10BE20004162FEF7D7FB18B1FFE7FBF7DDF8FFE74C
:10BE3000FFE7139841F62811C2F2000181631398BD
:10BE40008863FFE7FFE7FFE7FFE714B080BD00006E
:10BE500040F23840C2F20000027849F29871C2F212
:10BE600000010868104408607047000080B543F680
:10BE70000041C4F20201086840F4007008600868DC
:10BE800040F480600860086840F480700860032017
:10BE900000F0D0F80F2000F005F800F03BF800208B
:10BEA00080BD000080B582B0009040F22800C2F250
:10BEB0000000006840F23841C2F200010A784FF4F5
:10BEC0007A71B1FBF2F1B0FBF1F003F005FB20B1A8
:10BED000FFE701208DF8070018E000980F280DD823
:10BEE000FFE700994FF0FF30002200F06FF8009854
:10BEF00040F23C41C2F20001086003E001208DF8ED
:10BF0000070003E000208DF80700FFE79DF8070019
:10BF100002B080BD80B582B0FFE70020019043F6FB
:10BF20004400C4F20200016841F4804101600068ED
:10BF300000F4804001900198FFE7FFE700200090A7
:10BF400043F64000C4F20200016841F080510160F4
:10BF5000006800F0805000900098FFE76FF001004B
:10BF60000F21002200F032F802B080BD80B582B00F
:10BF70008DF807009DF90700002801D4FFE707E0CE
:10BF800045F2DB40C0F60200CE2111F0A1FDFFE733
:10BF90009DF9070011F0FEFC02B080BD80B582B0B3
:10BFA0008DF807009DF90700002801D4FFE707E09E
:10BFB00045F2DB40C0F60200BE2111F089FDFFE72B
:10BFC0009DF9070011F002FD02B080BD80B586B07A
:10BFD0008DF81700049103920020029003980F2817
:10BFE00001D8FFE707E045F2DB40C0F60200AA21D6
:10BFF00011F06EFDFFE704980F2801D8FFE707E076
:10C0000045F2DB40C0F60200AB2111F061FDFFE715
:10C0100011F0F4FC02909DF9170001900298049928
:10C02000039A07F0C5FE0146019811F0EFFC06B037
:10C0300080BD000080B582B001900198072810D023
:10C04000FFE7019806280CD0FFE70198052808D0E3
:10C05000FFE70198042804D0FFE70198032801D1E5
:10C06000FFE707E045F2DB40C0F60200922111F045
:10C070002FFDFFE7019811F00DFD02B080BD00001B
:10C0800082B001908DF8031002B0704782B0019029
:10C09000ADF80210BDF8020001990968486200205D
:10C0A00002B0704784B003908DF80B10ADF80820F3
:10C0B00003980068406A00909DF80B0048B9FFE7BC
:10C0C000BDF80810009840EA0140039909688862A9
:10C0D00033E003980068816A009800EB11400090FB
:10C0E00000208DF80700FFE79DF807009DF80B1072
:10C0F0000139884213D2FFE7039800689DF80710C2
:10C1000000EB8100D0F80411009800EB1140009082
:10C11000FFE79DF8070001308DF80700E4E7BDF860
:10C120000810009840EA0140039909689DF80B2027
:10C1300001EB8201C1F80001FFE7002004B0704765
:10C1400080B582B001900198D0F804040FF080FB14
:10C1500002B080BD80B582B001908DF80310019AC5
:10C16000D2F804049DF80310C1EBC10302EB830273
:10C17000926C0FF04BFA02B080BD000080B582B027
:10C1800001908DF80310019AD2F804049DF8031071
:10C19000C1EBC10302EB8302D2F808220FF0DCFAF4
:10C1A00002B080BD80B582B001900198D0F804043F
:10C1B0000FF054FB02B080BD80B584B002908DF8C2
:10C1C00007109DF80700000600280FD5FFE702982A
:10C1D0009DF8071001F00F01C1EBC10100EB8100D8
:10C1E0003C3000900099012048700FE002989DF8C3
:10C1F000071001F00F01C1EBC10100EB810000F558
:10C20000FE700090009900204870FFE79DF807003D
:10C2100000F00F0000990870FFE7029890F8BC0347
:10C22000012804D1FFE702208DF80F0014E00299E5
:10C23000012081F8BC03FFE7FFE70298006800993E
:10C2400010F0D0FAFFE70299002081F8BC03FFE765
:10C2500000208DF80F00FFE79DF80F0004B080BDAF
:10C2600080B584B002908DF807109DF8070000F0AB
:10C270000F0002994968884204D9FFE701208DF830
:10C280000F004DE09DF80700000600280FD5FFE7DE
:10C2900002989DF8071001F00F01C1EBC10100EBFE
:10C2A00081003C3000900099012048700FE0029816
:10C2B0009DF8071001F00F01C1EBC10100EB8100F7
:10C2C00000F5FE700090009900204870FFE700998B
:10C2D000002088709DF8070000F00F00009908709A
:10C2E000FFE7029890F8BC03012804D1FFE7022081
:10C2F0008DF80F0014E00299012081F8BC03FFE7DC
:10C30000FFE702980068009910F0F0FDFFE702993E
:10C31000002081F8BC03FFE700208DF80F00FFE745
:10C320009DF80F0004B080BD82B001908DF803101D
:10C3300001989DF8031001F00F01C1EBC10100EB62
:10C340008100D0F8140202B07047000080B586B0BA
:10C3500004908DF80F10ADF80C208DF80B300020F4
:10C360008DF80A009DF80F00000600280FD5FFE7A2
:10C3700004989DF80F1001F00F01C1EBC10100EB13
:10C3800081003C3001900199012048700FE0049831
:10C390009DF80F1001F00F01C1EBC10100EB81000E
:10C3A00000F5FE700190019900204870FFE79DF8AC
:10C3B0000F0000F00F0001990870BDF80C00019902
:10C3C00088609DF80B000199C8700198407820B1F1
:10C3D000FFE701990878C880FFE79DF80B00022865
:10C3E00004D1FFE7019900200871FFE7FFE70498F7
:10C3F00090F8BC03012804D1FFE702208DF8170054
:10C4000015E00499012081F8BC03FFE7FFE70498D9
:10C410000068019910F0A2F8FFE70499002081F864
:10C42000BC03FFE79DF80A008DF81700FFE79DF8B1
:10C43000170006B080BD000080B586B005908DF86D
:10C4400013100392029305989DF8131001F00F0149
:10C45000C1EBC10100EB810000F5FE700190039873
:10C460000199C8600298019948610199002088618A
:10C47000019948709DF8130000F00F0001990870B1
:10C4800005980069012804D1FFE703980199086124
:10C49000FFE79DF81300000738B9FFE7059A106819
:10C4A0000199127C10F0DAFB06E0059A10680199F8
:10C4B000127C10F0BFFDFFE7002006B080BD000039
:10C4C00080B584B002908DF807109DF8070000F049
:10C4D0000F0002994968884204D9FFE701208DF8CE
:10C4E0000F0058E09DF80700000600280FD5FFE771
:10C4F00002989DF8071001F00F01C1EBC10100EB9C
:10C5000081003C3000900099012048700DE00298B5
:10C510009DF80710C1EBC10100EB810000F5FE7032
:10C520000090009900204870FFE700990120887072
:10C530009DF8070000F00F0000990870FFE70298CF
:10C5400090F8BC03012804D1FFE702208DF80F000A
:10C5500021E00299012081F8BC03FFE7FFE7029880
:10C560000068009910F012FD9DF80700000740B91F
:10C57000FFE7029A1068117C02F5717210F066FCF8
:10C58000FFE7FFE70299002081F8BC03FFE70020E6
:10C590008DF80F00FFE79DF80F0004B080BD00008C
:10C5A00080B586B005908DF813100392029305981C
:10C5B0009DF8131001F00F01C1EBC10100EB8100E8
:10C5C0003C30019003980199C86002980199486134
:10C5D0000199002088610199012048709DF813009D
:10C5E00000F00F000199087005980069012804D136
:10C5F000FFE7039801990861FFE79DF81300000722
:10C6000038B9FFE7059A10680199127C10F026FBF3
:10C6100006E0059A10680199127C10F00BFDFFE707
:10C62000002006B080BD000080B58CB00B900B9848
:10C6300000680A900A9809900B98006810F02CFF87
:10C64000002840F01A83FFE70B98006810F090FF75
:10C6500008B9FFE711E30B98006810F089FF800725
:10C66000002807D5FFE70B980168486900F0020031
:10C670004861FFE70B98006810F07AFFC0060028B9
:10C6800062D5FFE70B980168886920F01000886187
:10C690000A98006A03900B98039901F00F01C1EB0F
:10C6A000C10100EB810000F5FE700290039800F4D8
:10C6B000F0110220B0EB514F23D1FFE7BDF80C0081
:10C6C00047F6F07108421BD0FFE70A980299C96843
:10C6D000039AC2F30A1210F059FF039847F6F0715B
:10C6E00000EA0103029AD06800EB1310D0600398AF
:10C6F00000EA01020299886900EB12108861FFE7E5
:10C700001BE0039800F4F0110620B0EB514F12D15A
:10C71000FFE70A980B9901F57171082210F036FFB6
:10C72000039847F6F07100EA01020299886900EB6C
:10C730001210886100E0FFE7FFE70B980168886945
:10C7400040F010008861FFE70B98006810F010FFC0
:10C750000003002870D5FFE7002005900B980068C3
:10C7600010F0B4FE0790FFE70798002863D0FFE7BA
:10C770009DF81C00C007002856D0FFE70B98006802
:10C780009DF8141010F0DCFE06909DF81800C0070C
:10C7900060B1FFE70998059900EB41110120C1F84C
:10C7A000080B0B98059907F087FBFFE79DF8180029
:10C7B000000700280CD5FFE70998059900EB411107
:10C7C0000820C1F8080B0B98059907F02FFBFFE72D
:10C7D0009DF81800C006002808D5FFE709980599BC
:10C7E00000EB41111020C1F8080BFFE79DF818007D
:10C7F0008006002808D5FFE70998059900EB41114C
:10C800002020C1F8080BFFE79DF8190080060028DA
:10C8100009D5FFE70998059900EB41114FF4005045
:10C82000C1F8080BFFE7FFE705980130059007986E
:10C830004008079098E7FFE70B98006810F098FE13
:10C840004003002840F1AC80FFE70B98006810F02F
:10C850002BFE079000200590FFE70798002800F0C6
:10C860009E80FFE79DF81C00C007002800F0908024
:10C87000FFE70B9800689DF8141010F039FE069041
:10C880009DF81800C00700283ED0FFE7059800F08B
:10C890000F01012000FA01F10491049B099AD2F8DA
:10C8A00034189943C2F834180999059A01EB4211DA
:10C8B000C1F808090B98006901281FD1FFE70B9800
:10C8C0000599C1EBC10100EB81014A6C886C1044F1
:10C8D0008864059888B9FFE70B980599C1EBC101F9
:10C8E00000EB8100006D40B9FFE70B99086801F586
:10C8F0007172012110F0AAFAFFE7FFE70B989DF88B
:10C900001410FFF727FCFFE79DF818000007002828
:10C9100008D5FFE70998059900EB41110820C1F8F7
:10C920000809FFE79DF81800C006002808D5FFE7B2
:10C930000998059900EB41111020C1F80809FFE79B
:10C940009DF818004006002808D5FFE709980599CA
:10C9500000EB41114020C1F80809FFE79DF81800DD
:10C960008007002808D5FFE70998059900EB4111D9
:10C970000220C1F80809FFE79DF81800000600280A
:10C9800005D5FFE70B98059907F088FBFFE7FFE760
:10C990000598013005900798400807905DE7FFE78C
:10C9A0000B98006810F0E4FDC00F00B3FFE7099991
:10C9B000D1F8040820F00100C1F804080B9890F8A1
:10C9C000F403012808D1FFE70B98002180F8F41345
:10C9D0000B98FFF755FB03E00B9800F061FBFFE7B6
:10C9E0000B980168486900F000404861FFE70B9828
:10C9F000006810F0BDFD0005002811D5FFE709987B
:10CA0000D0F80808C00720B1FFE70B9800F0D6FB6C
:10CA1000FFE70B980168486900F400604861FFE790
:10CA20000B98006810F0A4FDC004002840F190802D
:10CA3000FFE70999D1F8040820F00100C1F80408C3
:10CA40000B980068102110F0D7FC00200890FFE739
:10CA500008980B99496888423BD2FFE709980899E2
:10CA600000EB41114FF67F30C1F808090999089A87
:10CA700001EB4212D2F8001921F40011C2F800199A
:10CA80000999089A01EB4212D2F8001941F00061AD
:10CA9000C2F800190999089A01EB4211C1F8080B74
:10CAA0000998089900EB4111D1F8000B20F400100F
:10CAB000C1F8000B0998089900EB4111D1F8000B5F
:10CAC00040F00060C1F8000BFFE7089801300890C3
:10CAD000BEE70999D1F81C0840F00110C1F81C0804
:10CAE0000B98006B78B1FFE70999D1F8840840F002
:10CAF0000B00C1F884080999D1F8440840F00B00F4
:10CB0000C1F844080FE00999D1F8140842F22B0249
:10CB10001043C1F814080999D1F8100840F00B002F
:10CB2000C1F81008FFE70999D1F8000820F4FE6069
:10CB3000C1F800080B9A1068117C02F5717210F0B0
:10CB400085F90B980168486900F480504861FFE757
:10CB50000B98006810F00CFD800400281FD5FFE73B
:10CB60000B9800680FF06AFD0B98006810F06EFCDF
:10CB70000B99C8600B980068019000F04DFD0146CC
:10CB800001980B9A127B10F087FD0B9800F05EFA6B
:10CB90000B980168486900F400504861FFE70B9862
:10CBA000006810F0E5FC000700280AD5FFE70B98A5
:10CBB00000F080FA0B980168486900F008004861AD
:10CBC000FFE70B98006810F0D3FCC00200280ED5D8
:10CBD000FFE7002005900B989DF8141000F050F826
:10CBE0000B980168486900F480104861FFE70B98D2
:10CBF000006810F0BDFC800200280ED5FFE7002081
:10CC000005900B989DF8141000F048F80B980168F7
:10CC1000486900F400104861FFE70B98006810F0C5
:10CC2000A7FC400000280AD5FFE70B98FFF788FA19
:10CC30000B980168486900F080404861FFE70B9855
:10CC4000006810F095FC4007002815D5FFE70B9809
:10CC50000068406803909DF80C004007002804D548
:10CC6000FFE70B98FFF79EFAFFE7039A0B9801681E
:10CC7000486810434860FFE7FFE70CB080BD000044
:10CC800080B582B001908DF803100198D0F80404AB
:10CC90009DF803100EF074FE02B080BD80B582B026
:10CCA00001908DF803100198D0F804049DF803104A
:10CCB0000EF092FE02B080BD2DE9F04F97B01590B6
:10CCC000159820B9FFE701208DF85B0060E1159809
:10CCD0000068B0F1A04F08D0FFE715980068002168
:10CCE000C4F20401884201D1FFE707E045F2833036
:10CCF000C0F60200872110F0EBFEFFE715980068F0
:10CD00001490159890F8BD0340B9FFE715990020DD
:10CD100081F8BC03159800F041F9FFE7159903204D
:10CD200081F8BD031498C06BC005002804D4FFE748
:10CD3000159900200861FFE7159800680FF084FF3F
:10CD4000159810900168119141688268C368D0F805
:10CD500010C044698569C669076AD0F82480D0F894
:10CD60002890D0F82CA0D0F830B0D0F834E0684645
:10CD70001290C0F824E01198DDF848E0CEF820B019
:10CD8000CEF81CA0CEF81890CEF81480CEF8107013
:10CD9000CEF80C60CEF80850CEF80440CEF800C0B3
:10CDA0000FF062FC40B1FFE71599022081F8BD0346
:10CDB00001208DF85B00EBE01598006800210F91D1
:10CDC00010F00CFC0F988DF84F00FFE79DF84F0016
:10CDD00015994968884245D2FFE715989DF84F108C
:10CDE000C1EBC10100EB8101012081F83D009DF8FC
:10CDF0004F001599C0EBC00201EB820181F83C00A5
:10CE00009DF84F001599C0EBC00201EB8201A1F81B
:10CE1000420015989DF84F10C1EBC10100EB810154
:10CE2000002081F83F0015999DF84F20C2EBC20207
:10CE300001EB8201486415999DF84F20C2EBC202B4
:10CE400001EB8201886415999DF84F20C2EBC20264
:10CE500001EB82010865FFE79DF84F0001308DF876
:10CE60004F00B3E700208DF84F00FFE79DF84F001B
:10CE70001599496888423ED2FFE715989DF84F10F2
:10CE8000C1EBC10100EB8101002081F8FD019DF89B
:10CE90004F10159AC1EBC10302EB830282F8FC111B
:10CEA00015999DF84F20C2EBC20201EB820181F877
:10CEB000FF0115999DF84F20C2EBC20201EB8201E0
:10CEC000C1F8040215999DF84F20C2EBC20201EB94
:10CED0008201C1F8080215999DF84F20C2EBC202E9
:10CEE00001EB8201C1F81002FFE79DF84F0001300D
:10CEF0008DF84F00BAE715980C9001680D914168C4
:10CF00008268C368D0F810C044698569C669076A39
:10CF1000D0F82480D0F82890D0F82CA0D0F830B0E9
:10CF2000D0F834E068460E90C0F824E00D98DDF8A3
:10CF300038E0CEF820B0CEF81CA0CEF81890CEF88D
:10CF40001480CEF81070CEF80C60CEF80850CEF8F1
:10CF50000440CEF800C00FF015FD40B1FFE7159971
:10CF6000022081F8BD0301208DF85B0010E01599C7
:10CF700000200B9081F838001599012081F8BD033D
:10CF8000159800680FF0E8FC0B988DF85B00FFE740
:10CF90009DF85B0017B0BDE8F08F000080B58AB047
:10CFA0000990002008900790069005900490099839
:10CFB0000068B0F1A04F47D1FFE7FFE700200390E2
:10CFC00043F63000C4F20200016841F00101016043
:10CFD000006800F0010003900398FFE74FF4C05091
:10CFE00004900220059000200690032007900A205C
:10CFF00008900020C4F2020004A9FDF7D5FFFFE766
:10D0000043F63401C4F20201086840F08000086071
:10D01000FFE70020029043F64400C4F202000168DA
:10D0200041F480410160006800F480400290029861
:10D03000FFE7FFE74320019005210022FEF7C6FF2E
:10D040000198FEF7ABFFFFE70AB080BD80B582B064
:10D05000019001208DF803000198C06820B9FFE716
:10D0600000208DF803000CE00198C068022804D16C
:10D07000FFE701208DF8030002E0F9F7B5FFFFE7B5
:10D08000FFE70198D0F804049DF803100EF0A2FD0C
:10D090000198D0F804040EF013FD02B080BD00002A
:10D0A00080B582B001900198D0F804040EF058FDCC
:10D0B00002B080BD80B582B001900198D0F8040420
:10D0C0000EF060FD02B080BD80B584B002908DF896
:10D0D0000710FFE7029890F8BC03012804D1FFE78E
:10D0E00002208DF80F001AE00299012081F8BC039C
:10D0F000FFE7FFE79DF80700029981F838000298E2
:10D1000000689DF8071010F099FAFFE702990020D7
:10D1100081F8BC03FFE700208DF80F00FFE79DF8C2
:10D120000F0004B080BD000080B582B0019001996D
:10D13000D1F8040401F571710EF076FD02B080BDE6
:10D1400080B584B00290029800680190FFE70298D1
:10D1500090F8BC03012804D1FFE702208DF80F00EE
:10D1600027E00299012081F8BC03FFE7FFE702985E
:10D17000806A01280BD1FFE702988069012806D058
:10D18000FFE70199886B40F480308863FFE70298DD
:10D19000006810F001F9029800680FF0C7FBFFE784
:10D1A0000299002081F8BC03FFE700208DF80F00F2
:10D1B000FFE79DF80F0004B080BD000080B582B08D
:10D1C00001900198D0F804040EF0B0FD01980168B8
:10D1D000D1F8000E40F00100C1F8000E0198006A7D
:10D1E00048B1FFE74EF61051CEF20001086840F05A
:10D1F00006000860FFE702B080BD000080B584B083
:10D2000002900191029820B9FFE701208DF80F00EC
:10D21000FDE10298006830B1FFE7029800680F282E
:10D2200001D8FFE708E045F2BB30C0F602004FF43A
:10D23000177110F04DFCFFE70198E0B1FFE701988E
:10D24000012818D0FFE70198022814D0FFE70198C1
:10D25000032810D0FFE7019804280CD0FFE70198BD
:10D26000052808D0FFE70198062804D0FFE70198B9
:10D27000072801D1FFE708E045F2BB30C0F6020005
:10D2800040F25D2110F024FCFFE7019843F60041D5
:10D29000C4F20201096801F00701884212D9FFE7D0
:10D2A000019943F60040C4F202000170006800F0EA
:10D2B00007000199884204D0FFE701208DF80F0094
:10D2C000A5E1FFE7029800788007002860D5FFE716
:10D2D000029800784007002809D5FFE743F60801C7
:10D2E000C4F20201086840F4E0500860FFE70298C9
:10D2F00000780007002809D5FFE743F60801C4F2CB
:10D300000201086840F460400860FFE70298806806
:10D3100040B3FFE702988068802823D0FFE7029897
:10D32000806890281ED0FFE702988068A02819D056
:10D33000FFE702988068B02814D0FFE70298806861
:10D34000C0280FD0FFE702988068D0280AD0FFE7F6
:10D3500002988068E02805D0FFE702988068F028EE
:10D3600001D1FFE708E045F2BB30C0F602004FF400
:10D37000207110F0ADFBFFE743F60801C4F2020193
:10D38000086820F0F000029A926810430860FFE7F6
:10D3900002980078C007002800F08C80FFE7029810
:10D3A000406878B1FFE70298406801280AD0FFE79B
:10D3B00002984068022805D0FFE7029840680328D9
:10D3C00001D1FFE708E045F2BB30C0F6020040F2B1
:10D3D000872110F07DFBFFE702984068012811D1FA
:10D3E000FFE743F60000C4F20200006800F40031D9
:10D3F0000020B0EB514F04D1FFE701208DF80F0062
:10D4000005E12CE002984068022805D0FFE7029869
:10D410004068032811D1FFE743F60000C4F2020080
:10D42000006800F000710020B0EB516F04D1FFE7FD
:10D4300001208DF80F00EAE010E043F60000C4F28E
:10D440000200006800F002010020B0EB510F04D18F
:10D45000FFE701208DF80F00D9E0FFE7FFE743F673
:10D460000801C4F20201086820F00300029A526821
:10D4700010430860FEF78EF90090FFE743F60800BE
:10D48000C4F20200006800F00C0002994968B0EB99
:10D49000810F0ED0FFE7FEF77DF90099401A41F2A7
:10D4A0008931884204D3FFE703208DF80F00AEE0F6
:10D4B000E4E7FFE7019843F60041C4F2020109687E
:10D4C00001F00701884212D2FFE7019943F60040BC
:10D4D000C4F202000170006800F007000199884260
:10D4E00004D0FFE701208DF80F0090E0FFE70298DD
:10D4F00000784007002832D5FFE70298C068C0B125
:10D50000FFE70298C068B0F5805F12D0FFE702988D
:10D51000C068B0F5A05F0CD0FFE70298C068B0F516
:10D52000C05F06D0FFE70298C068B0F5E05F01D1A8
:10D53000FFE708E045F2BB30C0F6020040F2C5212B
:10D5400010F0C6FAFFE743F60801C4F202010868CA
:10D5500020F4E050029AD26810430860FFE7029876
:10D5600000780007002833D5FFE702980069C0B1B2
:10D57000FFE702980069B0F5805F12D0FFE70298DC
:10D580000069B0F5A05F0CD0FFE702980069B0F524
:10D59000C05F06D0FFE702980069B0F5E05F01D1F7
:10D5A000FFE708E045F2BB30C0F602004FF43371EC
:10D5B00010F08EFAFFE743F60801C4F20201086892
:10D5C00020F46040029A126940EAC2000860FFE756
:10D5D00000F04CF843F60801C4F202010968C9B230
:10D5E0000A0944F69031C0F60201895CC84040F255
:10D5F0002801C2F20001086040F23C40C2F2000083
:10D600000068FEF74FFC00208DF80F00FFE79DF843
:10D610000F0004B080BD000040F22800C2F20000FC
:10D620000068704780B5FFF7F7FF43F60801C4F2C2
:10D6300002010968C1F3822244F6A031C0F602015A
:10D64000895CC84080BD000080B5FFF7E5FF43F668
:10D650000801C4F20201096889B24A0B44F6A031FC
:10D66000C0F60201895CC84080BD000080B586B06C
:10D670000020059004900390029043F60800C4F245
:10D680000200006800F00C000146019140B1FFE784
:10D69000019804280AD0FFE7019808280CD04FE031
:10D6A00042F20040C0F2F40002904FE041F6003038
:10D6B000C0F2B700029049E043F60400C4F2020051
:10D6C000016801F03F01059100684002002813D570
:10D6D000FFE743F60400C4F202000068C0F38810BC
:10D6E00041F60031C0F2B701A0FB0101059A002309
:10D6F000F2F766FD049012E043F60400C4F2020063
:10D700000068C0F3881042F20041C0F2F401A0FBAF
:10D710000101059A0023F2F753FD0490FFE743F659
:10D720000400C4F20200006800F44031022000EB63
:10D73000D130039004980399B0FBF1F0029005E01A
:10D7400042F20040C0F2F4000290FFE7029806B0F7
:10D7500080BD000080B586B00490049828B9FFE72A
:10D7600001208DF8170000F048BC049800680F28CD
:10D7700001D8FFE707E045F2BB30C0F60200E82120
:10D7800010F0A6F9FFE704980078C007002800F021
:10D79000BE80FFE70498406860B1FFE704984068E6
:10D7A000B0F5803F06D0FFE704984068B0F5A02FA1
:10D7B00001D1FFE707E045F2BB30C0F60200ED21E2
:10D7C00010F086F9FFE743F60800C4F20200006893
:10D7D00000F00C00042813D0FFE743F60800C4F261
:10D7E0000200006800F00C0008281ED1FFE743F695
:10D7F0000400C4F2020000684002002815D5FFE7CB
:10D8000043F60000C4F20200006800F4003100207A
:10D81000B0EB514F08D0FFE70498406820B9FFE70C
:10D8200001208DF81700E8E370E0FFE704984068F6
:10D83000B0F5803F09D1FFE743F60001C4F20201D1
:10D84000086840F48030086020E004984068B0F533
:10D85000A02F0DD1FFE743F60001C4F202010868D2
:10D8600040F480200860086840F4803008600CE0D4
:10D8700043F60001C4F20201086820F48030086019
:10D88000086820F480200860FFE7FFE7FFE70498BE
:10D890004068E8B1FFE7FDF77DFF0390FFE743F63F
:10D8A0000000C4F20200006800F400310020B0EB78
:10D8B000514F0CD1FFE7FDF76DFF0399401A652822
:10D8C00004D3FFE703208DF8170096E3E7E71CE099
:10D8D000FDF760FF0390FFE743F60000C4F202008B
:10D8E000006800F400310020B0EB514F0CD0FFE78E
:10D8F000FDF750FF0399401A652804D3FFE7032082
:10D900008DF8170079E3E7E7FFE7FFE7FFE7049803
:10D9100000788007002840F1B880FFE70498C068CD
:10D9200028B1FFE70498C068012801D1FFE708E0AB
:10D9300045F2BB30C0F6020040F21F1110F0C8F8EB
:10D94000FFE7049800691F2801D8FFE708E045F2C7
:10D95000BB30C0F602004FF4907110F0B9F8FFE749
:10D9600043F60800C4F20200006810F00C0F13D058
:10D97000FFE743F60800C4F20200006800F00C0064
:10D9800008282CD1FFE743F60400C4F20200006827
:10D990004002002823D4FFE743F60000C4F202004F
:10D9A000006800F002010020B0EB510F09D0FFE742
:10D9B0000498C068012804D0FFE701208DF8170003
:10D9C0001BE343F60001C4F20201086820F0F800EE
:10D9D000049A126940EAC2000860FFE754E0049824
:10D9E000C06870B3FFE70021C4F24721012008603E
:10D9F000FDF7D0FE0390FFE743F60000C4F20200FB
:10DA0000006800F002010020B0EB510F0CD1FFE7DD
:10DA1000FDF7C0FE0399401A032804D3FFE7032053
:10DA20008DF81700E9E2E7E743F60001C4F20201CE
:10DA3000086820F0F800049A126940EAC200086001
:10DA400021E00021C4F2472100200860FDF7A2FE7A
:10DA50000390FFE743F60000C4F20200006800F004
:10DA600002010020B0EB510F0CD0FFE7FDF792FE52
:10DA70000399401A032804D3FFE703208DF8170009
:10DA8000BBE2E7E7FFE7FFE7FFE70498007800075E
:10DA900000285ED5FFE70498406928B1FFE70498A5
:10DAA0004069012801D1FFE708E045F2BB30C0F62C
:10DAB00002004FF4B07110F00BF8FFE704984069D2
:10DAC00018B3FFE740F68061C4F2472101200860E7
:10DAD000FDF760FE0390FFE743F67400C4F2020016
:10DAE000006800F002010020B0EB510F0CD1FFE7FD
:10DAF000FDF750FE0399401A032804D3FFE70320E3
:10DB00008DF8170079E2E7E722E040F68061C4F281
:10DB1000472100200860FDF73DFE0390FFE743F634
:10DB20007400C4F20200006800F002010020B0EBB3
:10DB3000510F0CD0FFE7FDF72DFE0399401A032883
:10DB400004D3FFE703208DF8170056E2E7E7FFE76D
:10DB5000FFE7049800784007002840F1E680FFE7DF
:10DB600000208DF807000498806850B1FFE7049802
:10DB70008068012805D0FFE704988068052801D156
:10DB8000FFE708E045F2BB30C0F602004FF4C67173
:10DB90000FF09EFFFFE743F64000C4F2020000686A
:10DBA000C000002815D4FFE7FFE70020009043F6EF
:10DBB0004000C4F20200016841F080510160006839
:10DBC00000F0805000900098FFE701208DF80700DA
:10DBD000FFE747F20000C4F200000068C00500281B
:10DBE00022D4FFE747F20001C4F20001086840F4C4
:10DBF00080700860FDF7CEFD0390FFE747F200005C
:10DC0000C4F200000068C00500280CD4FFE7FDF74F
:10DC1000C1FD0399401A032804D3FFE703208DF8C0
:10DC20001700EAE1EAE7FFE7FFE7049880680128C8
:10DC300009D1FFE743F67001C4F20201086840F021
:10DC4000010008601FE00498806805280DD1FFE7F7
:10DC500043F67001C4F20201086840F00400086055
:10DC6000086840F0010008600CE043F67001C4F25F
:10DC70000201086820F001000860086820F0040034
:10DC80000860FFE7FFE7FFE704988068F8B1FFE767
:10DC9000FDF780FD0390FFE743F67000C4F2020039
:10DCA000006800F002010020B0EB510F0ED1FFE739
:10DCB000FDF770FD0399401A41F28931884204D37F
:10DCC000FFE703208DF8170097E1E5E71EE0FDF779
:10DCD00061FD0390FFE743F67000C4F202000068A4
:10DCE00000F002010020B0EB510F0ED0FFE7FDF76E
:10DCF00051FD0399401A41F28931884204D3FFE76C
:10DD000003208DF8170078E1E5E7FFE79DF80700AD
:10DD1000012809D1FFE743F64001C4F20201086877
:10DD200020F080500860FFE7FFE70498806950B159
:10DD3000FFE704988069012805D0FFE7049880690F
:10DD4000022801D1FFE708E045F2BB30C0F602002F
:10DD500040F2CF110FF0BCFEFFE704988069002865
:10DD600000F04781FFE743F60800C4F202000068B4
:10DD700000F00C00082800F0F080FFE704988069AC
:10DD8000022840F0C780FFE70498C06930B1FFE780
:10DD90000498C069B0F5800F01D1FFE708E045F2B3
:10DDA000BB30C0F602004FF4EC710FF091FEFFE7BC
:10DDB0000498006A3F2801D8FFE708E045F2BB302D
:10DDC000C0F6020040F2D9110FF082FEFFE704987E
:10DDD000406A322807D3FFE70498406AB0F5D87F3D
:10DDE00001D8FFE708E045F2BB30C0F602004FF46F
:10DDF000ED710FF06DFEFFE70498806A02280FD0E6
:10DE0000FFE70498806A04280AD0FFE70498806A34
:10DE1000062805D0FFE70498806A082801D1FFE7AB
:10DE200008E045F2BB30C0F6020040F2DB110FF013
:10DE30004FFEFFE70498C06A022806D3FFE7049864
:10DE4000C06A0F2801D8FFE708E045F2BB30C0F6F2
:10DE500002004FF4EE710FF03BFEFFE76021C4F2C9
:10DE6000472100200860FDF795FC0390FFE743F68B
:10DE70000000C4F20200006800F000710020B0EB66
:10DE8000516F0CD0FFE7FDF785FC0399401A03287A
:10DE900004D3FFE703208DF81700AEE0E7E704990D
:10DEA000C869D1F820C04B6A8A6A40EA0C0040EA8F
:10DEB0008310D2034FF6FF739A43A2F580321043CA
:10DEC000C96A40EA016043F60401C4F20201086035
:10DED0006021C4F2472101200860FDF75BFC03903C
:10DEE000FFE743F60000C4F20200006800F0007192
:10DEF0000020B0EB516F0CD1FFE7FDF74BFC03990D
:10DF0000401A032804D3FFE703208DF8170074E0BC
:10DF1000E7E721E06021C4F2472100200860FDF717
:10DF200039FC0390FFE743F60000C4F202000068EA
:10DF300000F000710020B0EB516F0CD0FFE7FDF74F
:10DF400029FC0399401A032804D3FFE703208DF826
:10DF5000170052E0E7E7FFE74AE0049880690128EC
:10DF600004D1FFE701208DF8170046E043F60400D6
:10DF7000C4F202000068029004988069012831D040
:10DF8000FFE7029800F480000499C969884229D10A
:10DF9000FFE7029800F03F000499096A884221D106
:10DFA000FFE7029847F6C07108400499496AB0EB50
:10DFB000811F17D1FFE7029800F440300499896A65
:10DFC000C9034FF6FF729143A1F58031884209D110
:10DFD000FFE7029800F070600499C96AB0EB016F26
:10DFE00004D0FFE701208DF8170006E0FFE7FFE708
:10DFF000FFE700208DF81700FFE79DF8170006B037
:10E0000080BD000080B582B00090009820B9FFE785
:10E0100001208DF807002EE00098006840F600010E
:10E02000C5F20601884201D1FFE707E045F2F6504C
:10E03000C0F60200A3210FF04BFDFFE700984079E6
:10E0400038B9FFE7009900200871009800F018F82F
:10E05000FFE700990220487100980168086840F0C5
:10E060000400086000990120487100990020886030
:10E070008DF80700FFE79DF8070002B080BD0000A3
:10E0800082B001900198006840F60001C5F20601D7
:10E09000884212D1FFE7FFE70020009043F63400EA
:10E0A000C4F20200016841F040010160006800F024
:10E0B000400000900098FFE7FFE702B070470000C3
:10E0C00080B582B00190019808F03AFC8DF8030009
:10E0D0009DF8030003281BD0FFE7019808F030FCEF
:10E0E000014640F29850C2F2000000EB41108069F6
:10E0F00068B1FFE7019808F023FC014640F2985010
:10E10000C2F2000000EB411080698047FFE7FFE7A3
:10E1100002B080BD80B584B00290029820B9FFE7BC
:10E1200001208DF80F00D2E10298006843F200014F
:10E13000C4F20101884212D0FFE70298006843F65A
:10E140000001C4F20001884209D0FFE7029800688C
:10E1500043F60041C4F20001884201D1FFE708E024
:10E1600045F22E60C0F602004FF4A1710FF0B0FC32
:10E17000FFE70298406830B1FFE702984068B0F5C9
:10E18000827F01D1FFE708E045F22E60C0F6020071
:10E1900040F243110FF09CFCFFE70298806860B1E9
:10E1A000FFE702988068B0F5806F06D0FFE702981D
:10E1B0008068B0F5004F01D1FFE708E045F22E601E
:10E1C000C0F602004FF4A2710FF082FCFFE7029844
:10E1D000C068B0F5006F04D0FFE70298C06808B9C6
:10E1E000FFE708E045F22E60C0F6020040F245115C
:10E1F0000FF06EFCFFE702988069B0F5007F0AD04F
:10E20000FFE70298806930B1FFE702988069B0F5B6
:10E21000802F01D1FFE708E045F22E60C0F6020032
:10E220004FF4A3710FF054FCFFE70298C06918B3D4
:10E23000FFE70298C06908281ED0FFE70298C0696E
:10E24000102819D0FFE70298C069182814D0FFE7FA
:10E250000298C06920280FD0FFE70298C0692828DB
:10E260000AD0FFE70298C069302805D0FFE702987E
:10E27000C069382801D1FFE708E045F22E60C0F6FA
:10E28000020040F247110FF023FCFFE70298006AFA
:10E2900028B1FFE70298006A802801D1FFE708E073
:10E2A00045F22E60C0F602004FF4A4710FF010FC8E
:10E2B000FFE70298406A28B1FFE70298406A1028F9
:10E2C00001D1FFE708E045F22E60C0F6020040F2FF
:10E2D00049110FF0FDFBFFE70298406A002863D167
:10E2E000FFE70298006928B1FFE702980069022859
:10E2F00001D1FFE708E045F22E60C0F602004FF4BE
:10E30000A6710FF0E5FBFFE70298406928B1FFE72F
:10E3100002984069012801D1FFE708E045F22E602C
:10E32000C0F6020040F24D110FF0D2FBFFE7029859
:10E330004068B0F5827F32D1FFE70298C06918B318
:10E34000FFE70298C06908281ED0FFE70298C0695D
:10E35000102819D0FFE70298C069182814D0FFE7E9
:10E360000298C06920280FD0FFE70298C0692828CA
:10E370000AD0FFE70298C069302805D0FFE702986D
:10E38000C069382801D1FFE708E045F22E60C0F6E9
:10E39000020040F251110FF09BFBFFE703E00299EE
:10E3A0000020C861FFE736E00298C06918B3FFE7B4
:10E3B0000298C06908281ED0FFE70298C06910289B
:10E3C00019D0FFE70298C069182814D0FFE7029817
:10E3D000C06920280FD0FFE70298C06928280AD01A
:10E3E000FFE70298C069302805D0FFE70298C069AE
:10E3F000382801D1FFE708E045F22E60C0F60200A0
:10E4000040F25B110FF064FBFFE702990020086106
:10E4100002994861FFE7029900208862029890F80B
:10E42000510040B9FFE70299002081F8500002989E
:10E4300000F052F8FFE70299022081F8510002989B
:10E440000168086820F040000860029A0192116893
:10E450005068D2F808C0D36800F482700CF4044C01
:10E46000604403F400631844136903F00203184482
:10E47000536903F001031844936903F400731844CB
:10E48000D36903F038031844136A03F08003184378
:10E49000926A02F4005210430860029A508B00F016
:10E4A00004001168526A02F0100210444860029899
:10E4B0000168C86920F40060C861029900204865BD
:10E4C000029A012182F851108DF80F00FFE79DF8A4
:10E4D0000F0004B080BD000080B592B01190002004
:10E4E00010900F900E900D900C901198006843F2D0
:10E4F0000001C4F20101884240F0B680FFE7FFE767
:10E5000000200B9043F64400C4F20200016841F47D
:10E5100080510160006800F480500B900B98FFE779
:10E52000FFE700200A9043F63000C4F202000168C1
:10E5300041F002010160006800F002000A900A98B0
:10E54000FFE7FFE70020099043F63000C4F2020025
:10E55000016841F001010160006800F001000990CC
:10E560000998FFE718200C90022001900D900120DF
:10E5700002900E90032003900F90052004901090BD
:10E5800040F20040C4F202000CA90591FCF70CFD1A
:10E59000DDF804C0029B039A049805994FF0800EA1
:10E5A000CDF830E0CDF834C00E930F9210900020DB
:10E5B000C4F20200FCF7F8FC41F68810C2F2000039
:10E5C000069046F24041C4F2020101604FF0C06182
:10E5D000416000218160C1604FF48062026141614D
:10E5E0008161C1614FF4403202624162FBF7F2FF88
:10E5F00018B1FFE7F8F7F8FCFFE7FFE7119841F6DD
:10E600008811C2F20001C16411988863FFE741F6E6
:10E61000E810C2F20000009046F25841C4F2020134
:10E6200001604FF0C0614160402181600021C16004
:10E630004FF48062026141618161C1614FF4003237
:10E6400002624162FBF7C6FF18B1FFE7F8F7CCFCA6
:10E65000FFE7FFE7119841F6E811C2F2000181647B
:10E6600011988863FFE73EE01198006843F60001C7
:10E67000C4F20001884235D1FFE7FFE7002008908F
:10E6800043F64000C4F20200016841F48041016099
:10E69000006800F4804008900898FFE7FFE700203A
:10E6A000079043F63000C4F20200016841F0020115
:10E6B0000160006800F0020007900798FFE74FF440
:10E6C00060400C9002200D9001200E9003200F90CE
:10E6D0000520109040F20040C4F202000CA9FCF7A3
:10E6E00063FCFFE7FFE712B080BD000080B588B093
:10E6F00006900591ADF81220039300208DF80700D5
:10E7000006984068B0F5827F16D1FFE706988068CA
:10E7100090B9FFE70699042081F851000698059A00
:10E72000BDF812300399EC46CCF80010114600F009
:10E7300089FB8DF81F00EDE0FFE7069890F8500088
:10E74000012804D1FFE702208DF81F00E2E00699BE
:10E75000012081F85000FFE7FFE7FDF71BF802906A
:10E76000069890F85100012804D0FFE702208DF8A8
:10E770000700C0E0059820B1FFE7BDF8120020B9FE
:10E78000FFE701208DF80700B5E00699042081F825
:10E7900051000699002048650599069A9163BDF8D5
:10E7A0001210069A9187BDF81210069AD187069921
:10E7B0000863069988860699C886069908640699AA
:10E7C000486406988068B0F5004F0DD1FFE70698C1
:10E7D0000168086820F04000086006980168086831
:10E7E00020F480400860FFE706980068006800F0A9
:10E7F0004000402807D0FFE706980168086840F00D
:10E8000040000860FFE70698C06880BBFFE7FFE7AD
:10E810000698C08F50B3FFE7069800688068C0076D
:10E8200078B1FFE706980068007B0699896B08704D
:10E830000699886B013088630699C88F0138C887AC
:10E8400013E0FCF7A7FF0299401A0399884204D30A
:10E85000FFE70398013018B9FFE7039820B9FFE7F5
:10E8600003208DF8070046E0FFE7D1E72FE0FFE740
:10E870000698C08F50B3FFE7069800688068C0070D
:10E8800078B1FFE706980068C0680699896B088030
:10E890000699886B023088630699C88F0138C8874B
:10E8A00013E0FCF777FF0299401A0399884204D3DA
:10E8B000FFE70398013018B9FFE7039820B9FFE795
:10E8C00003208DF8070016E0FFE7D1E7FFE7069881
:10E8D0000399029A07F070FF20B1FFE70699202004
:10E8E0004865FFE70698406D20B1FFE701208DF8ED
:10E8F0000700FFE7FFE70699012081F85100FFE7D5
:10E900000699002081F85000FFE79DF807008DF878
:10E910001F00FFE79DF81F0008B080BD80B584B0E0
:10E9200002900191ADF8022000208DF801000298BC
:10E93000C06C08B1FFE708E045F22E60C0F60200A7
:10E9400040F2CA610FF0C4F8FFE70298806810BB7C
:10E95000FFE702984068B0F5827F1CD1FFE702997B
:10E96000042081F851000298806C08B1FFE708E0AC
:10E9700045F22E60C0F6020040F2D1610FF0A8F817
:10E98000FFE70298019ABDF80230114600F01CFC26
:10E990008DF80F00A8E0FFE7029890F850000128DA
:10E9A00004D1FFE702208DF80F009DE002990120BD
:10E9B00081F85000FFE7FFE7029890F85100012826
:10E9C00004D0FFE702208DF8010082E0019820B119
:10E9D000FFE7BDF8020020B9FFE701208DF8010034
:10E9E00077E00299042081F85100029900204865DF
:10E9F0000199029A9163BDF80210029A9187BDF8BD
:10EA00000210029AD1870299086402994864029917
:10EA100088860299C88602988068B0F5004F0DD1AB
:10EA2000FFE702980168086820F04000086002983B
:10EA30000168086820F480400860FFE70298C16C14
:10EA400046F25D60C0F6010008640298C16C46F2AF
:10EA50008D60C0F60100C8630298C16C46F229605F
:10EA6000C0F60100C8640298C16C00200865029BD2
:10EA700019689A6BD86C0C31DB8FFCF747F860B1E2
:10EA8000FFE70299486D40F01000486501208DF8BD
:10EA90000100029981F851001BE0029800680068AB
:10EAA00000F04000402807D0FFE70298016808689E
:10EAB00040F040000860FFE702980168486840F0B5
:10EAC0002000486002980168486840F001004860F2
:10EAD000FFE7FFE70299002081F85000FFE79DF86B
:10EAE00001008DF80F00FFE79DF80F0004B080BD16
:10EAF00080B582B00190019807F022FF8DF80300E5
:10EB00009DF8030003281BD0FFE7019807F018FFCA
:10EB1000014640F29850C2F2000000EB41104068FC
:10EB200068B1FFE7019807F00BFF014640F29850EB
:10EB3000C2F2000000EB411040688047FFE7FFE7AA
:10EB400002B080BD80B582B00190019807F0F8FE58
:10EB50008DF803009DF8030003281BD0FFE7019800
:10EB600007F0EEFE014640F29850C2F2000000EBC2
:10EB70004110006968B1FFE7019807F0E1FE014626
:10EB800040F29850C2F2000000EB4110006980474B
:10EB9000FFE7FFE702B080BD80B588B00690059121
:10EBA000ADF81220039300208DF8070006988068C6
:10EBB00030B1FFE706988068B0F5004F01D1FFE75C
:10EBC00008E045F22E60C0F6020040F20A310EF075
:10EBD0007FFFFFE7FFE7069890F85000012804D177
:10EBE000FFE702208DF81F0028E10699012081F837
:10EBF0005000FFE7FFE7FCF7CDFD0290BDF81200E3
:10EC0000ADF80400069890F85100012804D0FFE701
:10EC100002208DF8070002E1059820B1FFE7BDF85A
:10EC2000120020B9FFE701208DF80700F7E00699F0
:10EC3000032081F851000699002048650599069A3D
:10EC40001163BDF81210069A9186BDF81210069A4B
:10EC5000D18606998863069988870699C887069998
:10EC600048640699086406988068B0F5004F0DD195
:10EC7000FFE706980168086820F0400008600698E1
:10EC80000168086840F480400860FFE70698006863
:10EC9000006800F04000402807D0FFE706980168B0
:10ECA000086840F040000860FFE70698C068B0F5CB
:10ECB000006F47D1FFE70698406828B1FFE7BDF82D
:10ECC000040001280ED1FFE706980168006B008858
:10ECD000C8600699086B023008630699C88E01382F
:10ECE000C886FFE7FFE70698C08E50B3FFE7069897
:10ECF00000688068800700280ED5FFE70698016845
:10ED0000006B0088C8600699086B0230086306999A
:10ED1000C88E0138C88613E0FCF73CFD0299401A02
:10ED20000399884204D3FFE70398013018B9FFE73D
:10ED3000039820B9FFE703208DF807006FE0FFE795
:10ED4000D1E746E00698406828B1FFE7BDF8040027
:10ED500001280ED1FFE706980168006B0078087360
:10ED60000699086B013008630699C88E0138C88679
:10ED7000FFE7FFE70698C08E50B3FFE706980068EC
:10ED80008068800700280ED5FFE706980168006BB1
:10ED9000007808730699086B013008630699C88EDD
:10EDA0000138C88613E0FCF7F5FC0299401A039974
:10EDB000884204D3FFE70398013018B9FFE70398AE
:10EDC00020B9FFE703208DF8070028E0FFE7D1E72F
:10EDD000FFE706980399029A07F060FD20B1FFE76C
:10EDE000069920204865FFE70698806870B9FFE71C
:10EDF000FFE70020009006980068C0680090069821
:10EE00000068806800900098FFE7FFE70698406D73
:10EE100020B1FFE701208DF80700FFE7FFE7069923
:10EE2000012081F85100FFE70699002081F8500089
:10EE3000FFE79DF807008DF81F00FFE79DF81F0012
:10EE400008B080BD80B58EB0DDF840C00C900B914D
:10EE50000A92ADF826300120059000208DF81300AD
:10EE60000C98806808B9FFE708E045F22E60C0F60C
:10EE7000020040F27E410EF02BFEFFE7FFE70C9808
:10EE800090F85000012804D1FFE702208DF83700E8
:10EE900095E10C99012081F85000FFE7FFE7FCF7AE
:10EEA00079FC06900C9890F851008DF81F000C9892
:10EEB00040680890BDF82600ADF824009DF81F00BA
:10EEC000012812D0FFE70898B0F5827F09D1FFE74B
:10EED0000C98806828B9FFE79DF81F00042804D02B
:10EEE000FFE702208DF813005AE10B9838B1FFE7D5
:10EEF0000A9820B1FFE7BDF8260020B9FFE70120FE
:10EF00008DF813004CE10C9890F85100042805D0BE
:10EF1000FFE70C99052081F85100FFE70C990020CC
:10EF200048650A990C9A9163BDF826100C9AD1870E
:10EF3000BDF826100C9A91870B990C9A1163BDF8B5
:10EF400026100C9AD186BDF826100C9A91860C9941
:10EF500008640C9948640C980068006800F0400050
:10EF6000402807D0FFE70C980168086840F040008F
:10EF70000860FFE70C98C068B0F5006F76D1FFE736
:10EF80000C98406828B1FFE7BDF8240001280ED195
:10EF9000FFE70C980168006B0088C8600C99086B4B
:10EFA000023008630C99C88E0138C886FFE7FFE776
:10EFB0000C98C18E0120029039B9FFE70C98C08FE0
:10EFC000002818BF01200290FFE70298C007002820
:10EFD0004BD0FFE70C98006880688007002818D5A0
:10EFE000FFE70C98C08EA0B1FFE70598012810D16B
:10EFF000FFE70C980168006B0088C8600C99086BEB
:10F00000023008630C99C88E0138C886002005902C
:10F01000FFE70C9800688068C007A8B1FFE70C986C
:10F02000C08F88B1FFE70C980068C0680C99896BA5
:10F0300008800C99886B023088630C99C88F01385E
:10F04000C88701200590FFE7FCF7A4FB0699401A4A
:10F050001099884208D3FFE71098013020B1FFE7EC
:10F0600003208DF813009BE0A2E778E00C9840683D
:10F0700028B1FFE7BDF8240001280ED1FFE70C9866
:10F080000168006B007808730C99086B0130086305
:10F090000C99C88E0138C886FFE7FFE70C98C18E2F
:10F0A0000120019039B9FFE70C98C08F002818BFE4
:10F0B00001200190FFE70198C00700284ED0FFE72C
:10F0C0000C98006880688007002818D5FFE70C9826
:10F0D000C08EA0B1FFE70598012810D1FFE70C987A
:10F0E0000168006B007808730C99086B01300863A5
:10F0F0000C99C88E0138C88600200590FFE70C984F
:10F1000000688068C007A8B1FFE70C98C08F88B17D
:10F11000FFE70C980068C0680C99896B08700C991F
:10F12000886B013088630C99C88F0138C88701202B
:10F130000590FFE7FCF72EFB0699401A10998842CC
:10F1400004D3FFE71098013018B9FFE7109820B9F1
:10F15000FFE703208DF8130022E09FE7FFE70C98FC
:10F160001099069A07F09AFB38B1FFE701208DF855
:10F1700013000C992020486512E00C98806870B943
:10F18000FFE7FFE7002003900C980068C068039039
:10F190000C980068806803900398FFE7FFE7FFE79B
:10F1A0000C99012081F85100FFE70C99002081F8AB
:10F1B0005000FFE79DF813008DF83700FFE79DF83A
:10F1C00037000EB080BD000080B588B00690059174
:10F1D0000492ADF80E3000208DF806000698C06C41
:10F1E00008B1FFE708E045F22E60C0F602004FF4D8
:10F1F000E8610EF06DFCFFE70698806C08B1FFE750
:10F2000008E045F22E60C0F6020040F241710EF0B7
:10F210005FFCFFE70698806808B9FFE708E045F261
:10F220002E60C0F6020040F244710EF051FCFFE780
:10F23000FFE7069890F85000012804D1FFE702206C
:10F240008DF81F00EFE00699012081F85000FFE7DC
:10F25000FFE7069890F851008DF80700069840687F
:10F2600002909DF80700012812D0FFE70298B0F540
:10F27000827F09D1FFE70698806828B9FFE79DF8EB
:10F280000700042804D0FFE702208DF80600BFE045
:10F29000059838B1FFE7049820B1FFE7BDF80E00EC
:10F2A00020B9FFE701208DF80600B1E0069890F83C
:10F2B0005100042805D0FFE70699052081F8510088
:10F2C000FFE70699002048650599069A1163BDF885
:10F2D0000E10069A9186BDF80E10069AD1860499F2
:10F2E000069A9163BDF80E10069A9187BDF80E102C
:10F2F000069AD1870699086406994864069890F89A
:10F30000510004280FD1FFE70698C16C46F25D60FA
:10F31000C0F6010008640698C16C46F28D60C0F624
:10F320000100C8630EE00698C16C46F27560C0F635
:10F33000010008640698C16C46F23170C0F6010005
:10F34000C863FFE70698C16C46F22960C0F6010069
:10F35000C8640698C16C00200865069B19689A6B02
:10F36000D86C0C31DB8FFBF7D1FB60B1FFE706995E
:10F37000486D40F01000486501208DF806000699A0
:10F3800081F8510044E006980168486840F00100A7
:10F3900048600698816C002008640699896CC863EF
:10F3A0000699896CC8640699896C0865069B1A6879
:10F3B000196B986C0C32DB8EFBF7A8FB60B1FFE792
:10F3C0000699486D40F01000486501208DF8060050
:10F3D000069981F851001BE006980068006800F06B
:10F3E0004000402807D0FFE706980168086840F011
:10F3F00040000860FFE706980168486840F0200078
:10F40000486006980168486840F002004860FFE7DD
:10F41000FFE70699002081F85000FFE79DF80600FD
:10F420008DF81F00FFE79DF81F0008B080BD0000A9
:10F4300080B582B00190019807F082FA8DF8030040
:10F440009DF8030003281BD0FFE7019807F078FA26
:10F45000014640F29850C2F2000000EB4110806873
:10F4600068B1FFE7019807F06BFA014640F2985047
:10F47000C2F2000000EB411080688047FFE7FFE721
:10F4800002B080BD80B582B00190019807F058FAB3
:10F490008DF803009DF8030003281BD0FFE70198B7
:10F4A00007F04EFA014640F29850C2F2000000EB1D
:10F4B0004110406968B1FFE7019807F041FA014641
:10F4C00040F29850C2F2000000EB411040698047C2
:10F4D000FFE7FFE702B080BD80B582B001900198E0
:10F4E00007F0DCFF02B080BD81B0009001B0704732
:10F4F00081B0009001B0704780B584B00290019156
:10F5000000200090029800680021C4F201018842A6
:10F5100009D0FFE70298006840F20041C4F20101FF
:10F52000884201D1FFE708E045F29E60C0F6020084
:10F5300040F2B4710EF0CCFAFFE701980068B0F524
:10F54000006F04D0FFE70198006808B9FFE708E002
:10F5500045F29E60C0F6020040F2B5710EF0B8FAB6
:10F56000FFE701984068B0F5806F04D0FFE701988D
:10F57000406808B9FFE708E045F29E60C0F6020067
:10F5800040F2B6710EF0A4FAFFE70198806890B1DE
:10F59000FFE701988068B0F5807F0CD0FFE7019805
:10F5A0008068B0F5007F06D0FFE701988068B0F56D
:10F5B000407F01D1FFE708E045F29E60C0F60200FF
:10F5C00040F2B7710EF084FAFFE70198C068FF2897
:10F5D00001D8FFE708E045F29E60C0F602004FF454
:10F5E000F7610EF075FAFFE701980069B0F5805FEA
:10F5F00004D0FFE70198006908B9FFE708E045F289
:10F600009E60C0F6020040F2B9710EF061FAFFE7A9
:10F610000198406930B1FFE701984069B0F5005F9B
:10F6200001D1FFE708E045F29E60C0F6020040F21B
:10F63000BA710EF04DFAFFE70198C069B0F5804F3E
:10F6400004D0FFE70198C06908B9FFE708E045F278
:10F650009E60C0F6020040F2BB710EF039FAFFE77F
:10F66000FFE7029890F83C00012804D1FFE7022050
:10F670008DF80F0044E00299012081F83C00FFE77B
:10F68000FFE7009820F0FF000199C9680843009047
:10F69000009820F440700199896808430090009810
:10F6A00020F480600199496808430090009820F494
:10F6B00000600199096808430090009820F4805088
:10F6C0000199096908430090009820F400500199BD
:10F6D000496908430090009820F480400199C96965
:10F6E000084300900098029909684864FFE702996E
:10F6F000002081F83C00FFE700208DF80F00FFE7B5
:10F700009DF80F0004B080BD80B586B004900391D1
:10F71000049800680021C4F2010188423CD0FFE750
:10F7200004980068B0F1804F36D0FFE70498006875
:10F7300040F20041C4F2000188422DD0FFE7049856
:10F74000006840F60001C4F20001884224D0FFE7BF
:10F750000498006840F60041C4F2000188421BD0C2
:10F76000FFE70498006841F20001C4F200018842FA
:10F7700012D0FFE70498006841F20041C4F2000192
:10F78000884209D0FFE70498006840F20041C4F2C3
:10F790000101884201D1FFE708E045F29E60C0F612
:10F7A000020040F277710EF093F9FFE703980068CA
:10F7B00018B3FFE70398006810281ED0FFE70398EE
:10F7C0000068202819D0FFE703980068302814D07B
:10F7D000FFE70398006840280FD0FFE70398006810
:10F7E00050280AD0FFE703980068602805D0FFE79B
:10F7F00003980068702801D1FFE708E045F29E6099
:10F80000C0F602004FF4EF610EF062F9FFE70398D3
:10F810004068802804D0FFE70398406808B9FFE7F4
:10F8200008E045F29E60C0F6020040F279710EF0E9
:10F830004FF9FFE7FFE7049890F83C00012804D156
:10F84000FFE702208DF817007EE00499012081F87F
:10F850003C00FFE7FFE70499022081F83D0004988F
:10F8600000684068029004980068806801900298DF
:10F8700020F07000029003980168029808430290FB
:10F880000298049909684860049800680021C4F24D
:10F89000010188423CD0FFE704980068B0F1804F36
:10F8A00036D0FFE70498006840F20041C4F200013E
:10F8B00088422DD0FFE70498006840F60001C4F2AA
:10F8C0000001884224D0FFE70498006840F6004118
:10F8D000C4F2000188421BD0FFE70498006840F2A0
:10F8E0000041C4F20101884212D0FFE70498006889
:10F8F00044F20001C4F20101884209D0FFE70498F4
:10F90000006841F60001C4F2000188420ED1FFE711
:10F91000019820F080000190039841680198084305
:10F9200001900198049909688860FFE70499012013
:10F9300081F83D00FFE70499002081F83C00FFE7D3
:10F9400000208DF81700FFE79DF8170006B080BD76
:10F9500080B582B00090009820B9FFE701208DF8B3
:10F96000070012E1009800680021C4F201018842FA
:10F9700072D0FFE700980068B0F1804F6CD0FFE7CD
:10F980000098006840F20041C4F20001884263D050
:10F99000FFE70098006840F60001C4F200018842C9
:10F9A0005AD0FFE70098006840F60041C4F2000119
:10F9B000884251D0FFE70098006841F20001C4F28C
:10F9C0000001884248D0FFE70098006841F20041FA
:10F9D000C4F2000188423FD0FFE70098006840F27F
:10F9E0000041C4F20101884236D0FFE70098006868
:10F9F00044F20001C4F2010188422DD0FFE70098D3
:10FA0000006844F20041C4F20101884224D0FFE7BB
:10FA10000098006844F60001C4F2010188421BD03E
:10FA2000FFE70098006841F60001C4F20001884237
:10FA300012D0FFE70098006841F60041C4F20001CF
:10FA4000884209D0FFE70098006842F20001C4F242
:10FA50000001884201D1FFE708E045F26660C0F688
:10FA6000020040F213110EF033F8FFE700988068AF
:10FA7000A0B1FFE70098806810280FD0FFE700983A
:10FA8000806820280AD0FFE700988068402805D0C9
:10FA9000FFE700988068602801D1FFE708E045F2A1
:10FAA0006660C0F602004FF48A710EF011F8FFE7AD
:10FAB0000098006960B1FFE700980069B0F5807FA9
:10FAC00006D0FFE700980069B0F5007F01D1FFE79D
:10FAD00008E045F26660C0F6020040F215110DF034
:10FAE000F7FFFFE70098806928B1FFE70098806979
:10FAF000802801D1FFE708E045F26660C0F6020009
:10FB00004FF48B710DF0E4FFFFE7009890F83D0093
:10FB100040B9FFE70099002081F83C00009800F010
:10FB200039F8FFE70099022081F83D00009951F86B
:10FB3000040B07F067FD0099012081F84600FFE7FC
:10FB40000099012081F83E00009981F83F0000995A
:10FB500081F84000009981F84100FFE7FFE7009934
:10FB6000012081F84200009981F84300009981F852
:10FB70004400009981F84500FFE70099012081F8D1
:10FB80003D0000208DF80700FFE79DF8070002B058
:10FB900080BD000080B58AB00990099800680021F6
:10FBA000C4F2010188421BD1FFE7FFE70020089063
:10FBB00043F64400C4F20200016841F00101016013
:10FBC000006800F0010008900898FFE718200190F5
:10FBD00005210022FCF7FAF90198FCF7DFF9B0E003
:10FBE0000998006840F20041C4F20001884212D135
:10FBF000FFE7FFE70020079043F64000C4F2020051
:10FC0000016841F002010160006800F00200079005
:10FC10000798FFE794E00998006840F60001C4F2F5
:10FC20000001884212D1FFE7FFE70020069043F66B
:10FC30004000C4F20200016841F004010160006864
:10FC400000F0040006900698FFE778E00998006845
:10FC500040F60041C4F20001884212D1FFE7FFE7FD
:10FC60000020059043F64000C4F20200016841F014
:10FC700008010160006800F0080005900598FFE7A2
:10FC80005CE00998006841F20041C4F2000188423A
:10FC90001BD1FFE7FFE70020049043F64000C4F2C9
:10FCA0000200016841F020010160006800F02000BE
:10FCB00004900498FFE73720009005210022FCF70C
:10FCC00085F90098FCF76AF937E00998006840F276
:10FCD0000041C4F20101884212D1FFE7FFE7002092
:10FCE000039043F64400C4F20200016841F00201AF
:10FCF0000160006800F0020003900398FFE71BE03A
:10FD00000998006844F20041C4F20101884212D10E
:10FD1000FFE7FFE70020029043F64400C4F2020030
:10FD2000016841F400310160006800F40030029085
:10FD30000298FFE7FFE7FFE7FFE7FFE7FFE7FFE7DF
:10FD4000FFE70AB080BD000080B584B00290029841
:10FD500000680021C4F20101884272D0FFE70298D6
:10FD60000068B0F1804F6CD0FFE70298006840F265
:10FD70000041C4F20001884263D0FFE702980068A6
:10FD800040F60001C4F2000188425AD0FFE7029811
:10FD9000006840F60041C4F20001884251D0FFE7FC
:10FDA0000298006841F20001C4F20001884248D084
:10FDB000FFE70298006841F20041C4F20001884266
:10FDC0003FD0FFE70298006840F20041C4F2010111
:10FDD000884236D0FFE70298006844F20001C4F27E
:10FDE000010188422DD0FFE70298006844F20041EB
:10FDF000C4F20101884224D0FFE70298006844F66B
:10FE00000001C4F2010188421BD0FFE7029800689C
:10FE100041F60001C4F20001884212D0FFE70298C7
:10FE2000006841F60041C4F20001884209D0FFE7B2
:10FE30000298006842F20001C4F20001884201D138
:10FE4000FFE708E045F26660C0F6020040F2CF111D
:10FE50000DF03EFEFFE7029890F83D00012804D027
:10FE6000FFE701208DF80F006AE00299022081F877
:10FE70003D0002980168C86840F00100C86002981F
:10FE800000680021C4F2010188423CD0FFE70298DB
:10FE90000068B0F1804F36D0FFE70298006840F26A
:10FEA0000041C4F2000188422DD0FFE702980068AB
:10FEB00040F60001C4F20001884224D0FFE7029816
:10FEC000006840F60041C4F2000188421BD0FFE701
:10FED0000298006840F20041C4F20101884212D049
:10FEE000FFE70298006844F20001C4F20101884271
:10FEF00009D0FFE70298006841F60001C4F2000152
:10FF0000884212D1FFE702980068806800F007007D
:10FF100001900198062807D0FFE702980168086859
:10FF200040F001000860FFE706E0029801680868F9
:10FF300040F001000860FFE700208DF80F00FFE7A8
:10FF40009DF80F0004B080BD80B586B00490039189
:10FF5000FFE7049890F83C00012805D1FFE7022054
:10FF60008DF8170000F069BC0499012081F83C006D
:10FF7000FFE7FFE70499022081F83D00039800683D
:10FF8000B0F5805F2DD0FFE703980068B0F5005F03
:10FF900027D0FFE70398006818B3FFE703980068CD
:10FFA00010281ED0FFE703980068202819D0FFE72B
:10FFB00003980068302814D0FFE7039800684028B1
:10FFC0000FD0FFE70398006850280AD0FFE7039896
:10FFD0000068602805D0FFE703980068702801D109
:10FFE000FFE708E045F26660C0F6020041F22241F8
:10FFF0000DF06EFDFFE7049800688068029002989B
:020000040801F1
:1000000020F077000290029820F47F40029002983E
:10001000049909688860039800680190002800F03E
:10002000A883FFE70198102800F0A383FFE7019859
:10003000202800F09E83FFE70198302800F0998384
:10004000FFE70198402800F00883FFE70198502857
:1000500000F0EB81FFE70198602800F07282FFE773
:100060000198702800F09180FFE70198B0F5805F5B
:1000700006D0FFE70198B0F5005F00F03A81CDE3CC
:10008000049800680021C4F20101884272D0FFE7A1
:1000900004980068B0F1804F6CD0FFE704980068C6
:1000A00040F20041C4F20001884263D0FFE70498A7
:1000B000006840F60001C4F2000188425AD0FFE710
:1000C0000498006840F60041C4F20001884251D013
:1000D000FFE70498006841F20001C4F20001884281
:1000E00048D0FFE70498006841F20041C4F20001E3
:1000F00088423FD0FFE70498006840F20041C4F214
:100100000101884236D0FFE70498006844F20001FC
:10011000C4F2010188422DD0FFE70498006844F240
:100120000041C4F20101884224D0FFE7049800682E
:1001300044F60001C4F2010188421BD0FFE7049895
:10014000006841F60001C4F20001884212D0FFE7C6
:100150000498006841F60041C4F20001884209D0C9
:10016000FFE70498006842F20001C4F200018842EF
:1001700001D1FFE708E045F26660C0F6020041F2F7
:100180002E410DF0A5FCFFE749E30498006800212B
:10019000C4F2010188423CD0FFE704980068B0F146
:1001A000804F36D0FFE70498006840F20041C4F267
:1001B000000188422DD0FFE70498006840F6000156
:1001C000C4F20001884224D0FFE70498006840F69A
:1001D0000041C4F2000188421BD0FFE70498006888
:1001E00040F20041C4F20101884212D0FFE70498B6
:1001F000006844F20001C4F20101884209D0FFE71F
:100200000498006841F60001C4F20001884201D15F
:10021000FFE708E045F26660C0F6020041F23541B2
:100220000DF056FCFFE70398806890B1FFE7039854
:100230008068B0F5805F0CD0FFE703988068B0F568
:10024000005F06D0FFE703988068B0F5405F01D1FA
:10025000FFE708E045F26660C0F6020041F238416F
:100260000DF036FCFFE703984068B0F5004F12D060
:10027000FFE70398406870B1FFE70398406850B10A
:10028000FFE703984068022805D0FFE7039840681D
:100290000A2801D1FFE708E045F26660C0F60200D7
:1002A00041F239410DF014FCFFE70398C0680F28B4
:1002B00001D8FFE708E045F26660C0F6020041F2AF
:1002C0003A410DF005FCFFE704980068039B5A686B
:1002D0009968DB6807F004FB049800688068029066
:1002E000029840F0770002900298049909688860AB
:1002F00095E2049800680021C4F2010188422AD0E6
:10030000FFE704980068B0F1804F24D0FFE704981D
:10031000006840F20041C4F2000188421BD0FFE7B0
:100320000498006840F60001C4F20001884212D02F
:10033000FFE70498006840F60041C4F200018842DB
:1003400009D0FFE70498006840F20041C4F20101BF
:10035000884201D1FFE708E045F26660C0F602007E
:1003600041F24D410DF0B4FBFFE70398806890B176
:10037000FFE703988068B0F5805F0CD0FFE7039833
:100380008068B0F5005F06D0FFE703988068B0F59D
:10039000405F01D1FFE708E045F26660C0F6020069
:1003A00041F250410DF094FBFFE703984068B0F52F
:1003B000004F12D0FFE70398406870B1FFE7039841
:1003C000406850B1FFE703984068022805D0FFE776
:1003D000039840680A2801D1FFE708E045F266600B
:1003E000C0F6020041F251410DF072FBFFE70398A5
:1003F000C0680F2801D8FFE708E045F26660C0F644
:10040000020041F252410DF063FBFFE704980068DF
:10041000039B5A689968DB6807F062FA04980168E0
:10042000886840F480408860F9E104980068002101
:10043000C4F2010188423CD0FFE704980068B0F1A3
:10044000804F36D0FFE70498006840F20041C4F2C4
:10045000000188422DD0FFE70498006840F60001B3
:10046000C4F20001884224D0FFE70498006840F6F7
:100470000041C4F2000188421BD0FFE704980068E5
:1004800040F20041C4F20101884212D0FFE7049813
:10049000006844F20001C4F20101884209D0FFE77C
:1004A0000498006841F60001C4F20001884201D1BD
:1004B000FFE708E045F26660C0F6020041F26141E4
:1004C0000DF006FBFFE703984068B0F5004F12D02F
:1004D000FFE70398406870B1FFE70398406850B1A8
:1004E000FFE703984068022805D0FFE703984068BB
:1004F0000A2801D1FFE708E045F26660C0F6020075
:1005000041F264410DF0E4FAFFE70398C0680F2858
:1005100001D8FFE708E045F26660C0F6020041F24C
:1005200065410DF0D5FAFFE704980068039A516819
:10053000D26807F08BFC04980068502107F0EAF9B4
:100540006DE1049800680021C4F2010188423CD0AA
:10055000FFE704980068B0F1804F36D0FFE70498B9
:10056000006840F20041C4F2000188422DD0FFE74C
:100570000498006840F60001C4F20001884224D0CB
:10058000FFE70498006840F60041C4F20001884289
:100590001BD0FFE70498006840F20041C4F201015B
:1005A000884212D0FFE70498006844F20001C4F2C8
:1005B0000101884209D0FFE70498006841F6000174
:1005C000C4F20001884201D1FFE708E045F266600D
:1005D000C0F6020041F271410DF07AFAFFE703988C
:1005E0004068B0F5004F12D0FFE70398406870B143
:1005F000FFE70398406850B1FFE70398406802287E
:1006000005D0FFE7039840680A2801D1FFE708E01A
:1006100045F26660C0F6020041F274410DF058FAEE
:10062000FFE70398C0680F2801D8FFE708E045F20C
:100630006660C0F6020041F275410DF049FAFFE72D
:1006400004980068039A5168D26807F027FC049860
:100650000068602107F05EF9E1E00498006800217D
:10066000C4F2010188423CD0FFE704980068B0F171
:10067000804F36D0FFE70498006840F20041C4F292
:10068000000188422DD0FFE70498006840F6000181
:10069000C4F20001884224D0FFE70498006840F6C5
:1006A0000041C4F2000188421BD0FFE704980068B3
:1006B00040F20041C4F20101884212D0FFE70498E1
:1006C000006844F20001C4F20101884209D0FFE74A
:1006D0000498006841F60001C4F20001884201D18B
:1006E000FFE708E045F26660C0F6020041F2814192
:1006F0000DF0EEF9FFE703984068B0F5004F12D017
:10070000FFE70398406870B1FFE70398406850B175
:10071000FFE703984068022805D0FFE70398406888
:100720000A2801D1FFE708E045F26660C0F6020042
:1007300041F284410DF0CCF9FFE70398C0680F281F
:1007400001D8FFE708E045F26660C0F6020041F21A
:1007500085410DF0BDF9FFE704980068039A5168E0
:10076000D26807F073FB04980068402107F0D2F8C4
:1007700055E0049800680021C4F2010188423CD091
:10078000FFE704980068B0F1804F36D0FFE7049887
:10079000006840F20041C4F2000188422DD0FFE71A
:1007A0000498006840F60001C4F20001884224D099
:1007B000FFE70498006840F60041C4F20001884257
:1007C0001BD0FFE70498006840F20041C4F2010129
:1007D000884212D0FFE70498006844F20001C4F296
:1007E0000101884209D0FFE70498006841F6000142
:1007F000C4F20001884201D1FFE708E045F26660DB
:10080000C0F6020041F294410DF062F9FFE704984E
:1008100000680399096807F07DF800E0FFE7049994
:10082000012081F83D00FFE70499002081F83C0099
:10083000FFE700208DF81700FFE79DF8170006B0CE
:1008400080BD000081B0009001B0704780B582B0DB
:10085000019001980068006900F002010020B0EBEF
:10086000510F28D0FFE701980068C06800F002012E
:100870000020B0EB510F1DD0FFE7019801686FF029
:1008800002000861019901200877019800688069D9
:10089000800720B1FFE70198FFF7D4FF06E0019839
:1008A00000F04CFA019800F0A3FDFFE70199002049
:1008B0000877FFE7FFE701980068006900F004018E
:1008C0000020B0EB910F29D0FFE701980068C068C5
:1008D00000F004010020B0EB910F1ED0FFE701985B
:1008E00001686FF0040008610199022008770198FF
:1008F0000068806910F4407F04D0FFE70198FFF79B
:10090000A1FF06E0019800F019FA019800F070FDCF
:10091000FFE7019900200877FFE7FFE701980068EB
:10092000006900F008010020B0EBD10F28D0FFE7EC
:1009300001980068C06800F008010020B0EBD10FFA
:100940001DD0FFE7019801686FF008000861019968
:100950000420087701980068C069800720B1FFE78C
:100960000198FFF76FFF06E0019800F0E7F90198A2
:1009700000F03EFDFFE7019900200877FFE7FFE761
:1009800001980068006900F010010020B0EB111F11
:1009900029D0FFE701980068C06800F0100100202E
:1009A000B0EB111F1ED0FFE7019801686FF0100037
:1009B000086101990820087701980068C06910F45F
:1009C000407F04D0FFE70198FFF73CFF06E0019865
:1009D00000F0B4F9019800F00BFDFFE70199002049
:1009E0000877FFE7FFE7019800680069C00780B15A
:1009F000FFE701980068C068C00748B1FFE70198A9
:100A000001686FF001000861019801F057F8FFE7F5
:100A1000FFE7019800680069C1B20020B0EBD11F68
:100A200013D0FFE701980068C068C1B20020B0EBA6
:100A3000D11F09D0FFE7019801686FF080000861BD
:100A40000198FEF751FDFFE7FFE701980068006994
:100A500000F040010020B0EB911F14D0FFE7019897
:100A60000068C06800F040010020B0EB911F09D081
:100A7000FFE7019801686FF040000861019801F0FC
:100A800033F8FFE7FFE701980068006900F02001F4
:100A90000020B0EB511F14D0FFE701980068C06838
:100AA00000F020010020B0EB511F09D0FFE70198B2
:100AB00001686FF0200008610198FEF719FDFFE75B
:100AC000FFE702B080BD000080B592B01190002019
:100AD00010900F900E900D900C90119800680021CE
:100AE000C4F20101884222D1FFE7FFE700200B900A
:100AF00043F63000C4F20200016841F010010160C9
:100B0000006800F010000B900B98FFE74FF4D44002
:100B10000C9002210D9101200E900F91109041F246
:100B20000000C4F202000CA9FAF73EFA03E11198A2
:100B3000006840F20041C4F20001884222D1FFE780
:100B4000FFE700200A9043F63000C4F2020001687B
:100B500041F004010160006800F004000A900A9866
:100B6000FFE74FF480700C9002200D9001210E9150
:100B70000F90109040F60000C4F202000CA9FAF7A2
:100B800013FAD7E01198006840F60001C4F20001A2
:100B9000884223D1FFE7FFE70020099043F63000A9
:100BA000C4F20200016841F008010160006800F031
:100BB000080009900998FFE74FF480400C9002204C
:100BC0000D9001210E9103210F91109040F60040ED
:100BD000C4F202000CA9FAF7E7F9AAE0119800683C
:100BE00040F60041C4F20001884222D1FFE7FFE74E
:100BF0000020089043F63000C4F20200016841F082
:100C000080010160006800F0800008900898FFE70C
:100C10004FF4E0500C9002200D9001210E910F90A6
:100C2000109041F60040C4F202000CA9FAF7BCF99A
:100C30007EE01198006840F20041C4F20101884250
:100C40004AD1FFE7FFE70020079043F63000C4F2E7
:100C50000200016841F480710160006800F4807056
:100C600007900798FFE7FFE70020069043F6300063
:100C7000C4F20200016841F004010160006800F064
:100C8000040006900698FFE7402000900C90022098
:100C900002900D90012101910E910F90032003907D
:100CA000109042F20000C4F202000CA90491FAF77D
:100CB0007BF9DDF800C0019B029A03980499CDF8F6
:100CC00030C00D920E930F92109040F60000C4F2C7
:100CD0000200FAF769F92AE01198006844F200412D
:100CE000C4F20101884221D1FFE7FFE7002005900F
:100CF00043F63000C4F20200016841F020010160B7
:100D0000006800F0200005900598FFE740200C9057
:100D100002200D900E900F900320109041F20040A1
:100D2000C4F202000CA9FAF73FF9FFE7FFE7FFE77B
:100D3000FFE7FFE7FFE712B080BD000081B0009041
:100D400001B0704780B586B004900391029202987A
:100D500080B1FFE7029804280CD0FFE7029808282A
:100D600008D0FFE702980C2804D0FFE702983C283F
:100D700001D1FFE708E045F26660C0F6020041F2EB
:100D800017010CF0A5FEFFE703980068602805D066
:100D9000FFE703980068702801D1FFE708E045F2FB
:100DA0006660C0F6020041F218010CF091FEFFE708
:100DB0000398806828B1FFE703988068022801D172
:100DC000FFE708E045F26660C0F6020041F2190153
:100DD0000CF07EFEFFE70398006928B1FFE7039857
:100DE0000069042801D1FFE708E045F26660C0F61B
:100DF000020041F21A010CF06BFEFFE7FFE70498D6
:100E000090F83C00012804D1FFE702208DF817007C
:100E1000C3E10499012081F83C00FFE7FFE7029855
:100E200001900C2800F2AE810199DFE811F00D006D
:100E3000AB01AB01AB019800AB01AB01AB01000111
:100E4000AB01AB01AB015501049800680021C4F26D
:100E50000101884260D0FFE704980068B0F1804F3C
:100E60005AD0FFE70498006840F20041C4F2000144
:100E7000884251D0FFE70498006840F60001C4F2B0
:100E80000001884248D0FFE70498006840F600411E
:100E9000C4F2000188423FD0FFE70498006840F2A6
:100EA0000041C4F20101884236D0FFE7049800688F
:100EB00044F20001C4F2010188422DD0FFE70498FA
:100EC000006844F20041C4F20101884224D0FFE7E7
:100ED0000498006844F60001C4F2010188421BD066
:100EE000FFE70498006841F60001C4F2000188425F
:100EF00012D0FFE70498006841F60041C4F20001F7
:100F0000884209D0FFE70498006842F20001C4F269
:100F10000001884201D1FFE708E045F26660C0F6B3
:100F2000020041F224010CF0D3FDFFE704980068B1
:100F3000039906F005FD04980168886940F00800EF
:100F4000886104980168886920F00400886103982A
:100F500002690498016888691043886113E1049864
:100F600000680021C4F2010188423CD0FFE70498E8
:100F70000068B0F1804F36D0FFE70498006840F277
:100F80000041C4F2000188422DD0FFE704980068B8
:100F900040F60001C4F20001884224D0FFE7049823
:100FA000006840F60041C4F2000188421BD0FFE710
:100FB0000498006840F20041C4F20101884212D056
:100FC000FFE70498006844F20001C4F2010188427E
:100FD00009D0FFE70498006841F60001C4F200015F
:100FE000884201D1FFE708E045F26660C0F60200E2
:100FF00041F235010CF06CFDFFE70498006803999D
:1010000006F050FD04980168886940F4006088612A
:1010100004980168886920F48060886103980269F7
:1010200004980168886940EA02208861ABE004986E
:1010300000680021C4F2010188422AD0FFE7049829
:101040000068B0F1804F24D0FFE70498006840F2B8
:101050000041C4F2000188421BD0FFE704980068F9
:1010600040F60001C4F20001884212D0FFE7049864
:10107000006840F60041C4F20001884209D0FFE751
:101080000498006840F20041C4F20101884201D195
:10109000FFE708E045F26660C0F6020041F2460153
:1010A0000CF016FDFFE704980068039906F0B0FD08
:1010B00004980168C86940F00800C8610498016894
:1010C000C86920F00400C8610398026904980168A7
:1010D000C8691043C86156E0049800680021C4F252
:1010E000010188422AD0FFE704980068B0F1804FE0
:1010F00024D0FFE70498006840F20041C4F20001E8
:1011000088421BD0FFE70498006840F60001C4F253
:101110000001884212D0FFE70498006840F60041C1
:10112000C4F20001884209D0FFE70498006840F249
:101130000041C4F20101884201D1FFE708E045F215
:101140006660C0F6020041F257010CF0C1FCFFE7F7
:1011500004980068039906F011FE04980168C869B4
:1011600040F40060C86104980168C86920F4806098
:10117000C8610398026904980168C86940EA0220BE
:10118000C86100E0FFE7FFE70499002081F83C0018
:10119000FFE700208DF81700FFE79DF8170006B065
:1011A00080BD000080B582B00090009820B9FFE7B4
:1011B00001208DF8070012E1009800680021C4F2B8
:1011C0000101884272D0FFE700980068B0F1804FBB
:1011D0006CD0FFE70098006840F20041C4F20001C3
:1011E000884263D0FFE70098006840F60001C4F22F
:1011F000000188425AD0FFE70098006840F600419D
:10120000C4F20001884251D0FFE70098006841F223
:101210000001C4F20001884248D0FFE7009800684E
:1012200041F20041C4F2000188423FD0FFE700983C
:10123000006840F20041C4F20101884236D0FFE765
:101240000098006844F20001C4F2010188422DD0E8
:10125000FFE70098006844F20041C4F201018842AF
:1012600024D0FFE70098006844F60001C4F20101B1
:1012700088421BD0FFE70098006841F60001C4F2E5
:101280000001884212D0FFE70098006841F6004153
:10129000C4F20001884209D0FFE70098006842F2DA
:1012A0000001C4F20001884201D1FFE708E045F2E5
:1012B0006660C0F6020040F20E510CF009FCFFE738
:1012C00000988068A0B1FFE70098806810280FD0D0
:1012D000FFE70098806820280AD0FFE70098806820
:1012E000402805D0FFE700988068602801D1FFE71B
:1012F00008E045F26660C0F6020040F20F510CF0C3
:10130000E7FBFFE70098006960B1FFE7009800691C
:10131000B0F5807F06D0FFE700980069B0F5007F48
:1013200001D1FFE708E045F26660C0F602004FF425
:10133000A2610CF0CDFBFFE70098806928B1FFE7C0
:1013400000988069802801D1FFE708E045F26660D7
:10135000C0F6020040F211510CF0BAFBFFE7009812
:1013600090F83D0040B9FFE70099002081F83C006B
:10137000009800F039F8FFE70099022081F83D005D
:10138000009951F8040B06F03DF90099012081F80D
:101390004600FFE70099012081F83E00009981F89E
:1013A0003F00009981F84000009981F84100FFE773
:1013B000FFE70099012081F84200009981F843007D
:1013C000009981F84400009981F84500FFE70099F1
:1013D000012081F83D0000208DF80700FFE79DF80F
:1013E000070002B080BD000081B0009001B07047DE
:1013F00081B0009001B0704780B58CB00A9009911F
:101400000A9800680021C4F20101884214D1FFE764
:101410000998002800F0E780FFE70998042800F009
:10142000E280FFE70998082800F0DD80FFE70998CF
:101430000C2800F0D880FFE70A980068B0F1804FD0
:1014400014D1FFE70998002800F0CD80FFE7099844
:10145000042800F0C880FFE70998082800F0C3803E
:10146000FFE709980C2800F0BE80FFE70A980068A3
:1014700040F20041C4F20001884214D1FFE709980C
:10148000002800F0B080FFE70998042800F0AB8046
:10149000FFE70998082800F0A680FFE709980C28C4
:1014A00000F0A180FFE70A98006840F60001C4F24E
:1014B0000001884214D1FFE70998002800F09380CA
:1014C000FFE70998042800F08E80FFE709980828B4
:1014D00000F08980FFE709980C2800F08480FFE77E
:1014E0000A98006840F60041C4F20001884210D119
:1014F000FFE70998002876D0FFE70998042872D002
:10150000FFE7099808286ED0FFE709980C286AD0F1
:10151000FFE70A98006840F20041C4F201018842E6
:1015200010D1FFE7099800285DD0FFE7099804284B
:1015300059D0FFE70998082855D0FFE709980C28EB
:1015400051D0FFE70A98006844F20001C4F201019B
:10155000884208D1FFE70998002844D0FFE709989E
:10156000042840D0FFE70A98006844F20041C4F222
:101570000101884203D1FFE70998A0B3FFE70A9869
:10158000006844F60001C4F20101884203D1FFE77C
:10159000099840B3FFE70A98006841F60001C4F2D9
:1015A0000001884207D1FFE70998E0B1FFE70998F9
:1015B000042818D0FFE70A98006841F60041C4F2F9
:1015C0000001884203D1FFE7099860B1FFE70A985C
:1015D000006842F20001C4F20001884204D1FFE732
:1015E000099808B9FFE708E045F26660C0F6020016
:1015F00040F294510CF06CFAFFE7099828B9FFE724
:101600000A9890F83E0007901CE00998042805D13C
:10161000FFE70A9890F83F00069010E00998082824
:1016200005D1FFE70A9890F84000059004E00A9879
:1016300090F841000590FFE705980690FFE70698AF
:101640000790FFE70798012804D0FFE701208DF8F5
:101650002F00AFE0099828B9FFE70A99022081F826
:101660003E001EE00998042806D1FFE70A990220EF
:1016700081F83F00049012E00998082806D1FFE79E
:101680000A99022081F84000039005E00A9902209F
:1016900081F841000390FFE703980490FFE7049866
:1016A000FFE70A98006809990122019206F078F88C
:1016B00001980A9909680022C4F20102914202903D
:1016C0000CD0FFE70A9800684FF60041CBF6FE7198
:1016D0000844B0FA80F040090290FFE70298C00782
:1016E00038B1FFE70A980168486C40F4004048644C
:1016F000FFE70A9800680021C4F2010188423CD04B
:10170000FFE70A980068B0F1804F36D0FFE70A98EB
:10171000006840F20041C4F2000188422DD0FFE78A
:101720000A98006840F60001C4F20001884224D003
:10173000FFE70A98006840F60041C4F200018842C1
:101740001BD0FFE70A98006840F20041C4F2010193
:10175000884212D0FFE70A98006844F20001C4F200
:101760000101884209D0FFE70A98006841F60001AC
:10177000C4F20001884212D1FFE70A98006880682D
:1017800000F0070008900898062807D0FFE70A989D
:101790000168086840F001000860FFE706E00A9869
:1017A0000168086840F001000860FFE700208DF83C
:1017B0002F00FFE79DF82F000CB080BD80B586B0EC
:1017C00005900491059800680021C4F20101884247
:1017D00014D1FFE70498002800F0E780FFE70498A1
:1017E000042800F0E280FFE70498082800F0DD807C
:1017F000FFE704980C2800F0D880FFE70598006800
:10180000B0F1804F14D1FFE70498002800F0CD809C
:10181000FFE70498042800F0C880FFE70498082830
:1018200000F0C380FFE704980C2800F0BE80FFE7BB
:101830000598006840F20041C4F20001884214D1CA
:10184000FFE70498002800F0B080FFE70498042820
:1018500000F0AB80FFE70498082800F0A680FFE7BF
:1018600004980C2800F0A180FFE70598006840F676
:101870000001C4F20001884214D1FFE70498002857
:1018800000F09380FFE70498042800F08E80FFE7C3
:101890000498082800F08980FFE704980C2800F0DD
:1018A0008480FFE70598006840F60041C4F200011B
:1018B000884210D1FFE70498002876D0FFE704980B
:1018C000042872D0FFE7049808286ED0FFE7049838
:1018D0000C286AD0FFE70598006840F20041C4F286
:1018E0000101884210D1FFE7049800285DD0FFE78E
:1018F0000498042859D0FFE70498082855D0FFE73A
:1019000004980C2851D0FFE70598006844F20001C4
:10191000C4F20101884208D1FFE70498002844D0AE
:10192000FFE70498042840D0FFE70598006844F2D8
:101930000041C4F20101884203D1FFE70498A0B33B
:10194000FFE70598006844F60001C4F201018842EF
:1019500003D1FFE7049840B3FFE70598006841F61C
:101960000001C4F20001884207D1FFE70498E0B10A
:10197000FFE70498042818D0FFE70598006841F6AF
:101980000041C4F20001884203D1FFE7049860B12E
:10199000FFE70598006842F20001C4F200018842A6
:1019A00004D1FFE7049808B9FFE708E045F2666054
:1019B000C0F602004FF4B9610CF08AF8FFE7059811
:1019C00000680499002205F0EBFE059801680120EB
:1019D0000022C4F20102914203900CD0FFE7059867
:1019E00000684FF60041CBF6FE710844B0FA80F073
:1019F00040090390FFE70398C007D8B1FFE7FFE76E
:101A000005980068006A41F21111084210D1FFE701
:101A100005980068006A40F24441084207D1FFE798
:101A200005980168486C20F400404864FFE7FFE730
:101A3000FFE7FFE7FFE705980068006A41F2111130
:101A4000084210D1FFE705980068006A40F244415F
:101A5000084207D1FFE705980168086820F00100F7
:101A60000860FFE7FFE7FFE7049828B9FFE705995B
:101A7000012081F83E001EE00498042806D1FFE70B
:101A80000599012081F83F00029012E0049808288F
:101A900006D1FFE70599012081F84000019005E09B
:101AA0000599012081F841000190FFE7019802901B
:101AB000FFE70298FFE7002006B080BD81B00090EC
:101AC0000098006841F20041C4F20001884208D148
:101AD000FFE741F62451C2F20001086801300860B6
:101AE000FFE701B07047000081B0009001B070477F
:101AF00082B00190ADF8021002B0704780B582B09C
:101B00000190019807F0CCFE8DF803009DF80300CA
:101B100004281BD0FFE79DF8030000EBC00140F252
:101B20001860C2F2000000EB8100C06968B1FFE7F5
:101B30009DF8030000EBC00140F21860C2F2000003
:101B400000EB8100C0698047FFE7FFE702B080BD7E
:101B500080B582B0019001980168C86820F4907047
:101B6000C86001980168486920F001004861019847
:101B7000006B012807D1FFE701980168C86820F0D1
:101B80001000C860FFE7019800684069400600281F
:101B90002BD5FFE701980168486920F040004861B3
:101BA0000198806B98B1FFE70198816B49F28D70C5
:101BB000C0F6010008650198806BF8F759FB28B161
:101BC000FFE70198806B016D8847FFE70CE0019902
:101BD0000020C885019A202182F83E1001990863EF
:101BE0000198FFF78BFFFFE70CE001990020C88503
:101BF000019A202182F83E10019908630198FFF7AD
